:020000040800F2
:1000000030C901203D03000899550008074B00083E
:1000100095550008251E00084F5B000800000000F1
:10002000000000000000000000000000F959000876
:10003000291E0008000000009D550008FB5900081B
:100040005703000857030008570300085703000828
:100050005703000857030008570300085703000818
:100060005703000857030008570300085703000808
:1000700057030008570300085703000857030008F8
:1000800057030008570300085703000857030008E8
:1000900057030008570300085703000857030008D8
:1000A00057030008570300085703000857030008C8
:1000B000570300085703000800000000570300081A
:1000C00057030008570300085703000857030008A8
:1000D0005703000857030008570300085703000898
:1000E000570300085703000800000000000000004C
:1000F0000000000000000000000000000000000000
:10010000000000005703000800000000570300082B
:100110005703000800000000895A00080000000092
:100120005703000857030008570300085703000847
:100130005703000857030008570300080000000099
:100140005703000857030008570300085703000827
:100150005703000857030008570300085703000817
:100160005703000857030008570300080000000069
:10017000000000005703000800000000000000001D
:1001800057030008570300085703000857030008E7
:100190005703000800F002F800F0C0F80AA090E849
:1001A000000C82448344AAF10107DA4501D100F032
:1001B000B5F8AFF2090EBAE80F0013F0010F18BF3F
:1001C000FB1A43F00103184748A8050088A805005A
:1001D0000A444FF0000C10F8013B13F0070408BF6D
:1001E00010F8014B1D1108BF10F8015B641E05D00B
:1001F00010F8016B641E01F8016BF9D113F0080FC0
:100200001EBF10F8014BAD1C0C1B09D16D1E58BF51
:1002100001F801CBFAD505E014F8016B01F8016B88
:100220006D1EF9D59142D6D370470000103A24BF15
:1002300078C878C1FAD8520724BF30C830C144BF4B
:1002400004680C607047000000230024002500268D
:10025000103A28BF78C1FBD8520728BF30C148BF29
:100260000B6070476E2900F05983702900F0A38459
:1002700066293BF07A8765293BF0778767293BF051
:10028000748761293BF0738703681B0A28BF41F01C
:100290008001692900F0A880642900F0A5807529F3
:1002A00000F0A2806F2900F03184782900F06F847B
:1002B000E92900F0CB83E42900F0C883F52900F098
:1002C000C583EF2900F02E84F82900F06E840368BE
:1002D000DB0928BF41F08001632901F057807329B1
:1002E00001F05C80E32901F06780F32901F06C8064
:1002F000002070471FB53BF02EFF01F0B7F8040057
:10030000002000213BF0E4F9401C60600020002147
:100310003BF0C8F9E0601FBD10B510BD01F079F8E1
:100320001146FFF7E7FF30F0FBF801F051F903B495
:10033000FFF7F2FF03BC00F049FC000009488047CA
:1003400009480047FEE7FEE7FEE7FEE7FEE7FEE7B7
:10035000FEE7FEE7FEE7FEE704480549054A064BCF
:1003600070470000755A00089501000830B7012059
:1003700030C9012030B9012030B901207CB51D46BB
:1003800016460C00009001D02044401E074B7B44D1
:100390002A4669460190304600F0D9FA05461CB15C
:1003A0000020694600F0E6FA28467CBDED05000015
:1003B0000FB47CB50C0009AA009001D02044401E67
:1003C000084B7B4469460190089800F0C0FA054646
:1003D0001CB10020694600F0CDFA28467CBC5DF8CF
:1003E00014FB0000B90500002DE9F0410646002489
:1003F00010687529314616A510D000F0FBF90028C9
:1004000002DA404213A507E031688A0701D512A538
:1004100002E0490704D511A5012401E000F0F3F939
:1004200000210A2206F1240709E0B0FBF2FCB0FB30
:10043000F2F302FB1C00303078541846491C0028A7
:10044000F3D123462A463046BDE8F04100F00DBA0C
:10045000000000002D0000002B0000002000000024
:100460002DE9F05F894604464FF0000ADFF874B1C9
:10047000FB44C0F820A02046E1688847002874D0DB
:10048000252806D0D4E901219047206A401C20622B
:10049000F1E700265F462046E168884720280546A8
:1004A00007DB312D05D2781910F8200C08B106436E
:1004B000F1E7B00701D526F00406C4F81CA0002718
:1004C000C4F818A02A2D09D0284605F081FB38B3BE
:1004D00004EB8708303DC8F8185019E059F8041BA0
:1004E000204604EB87029161E1688847012F0546A9
:1004F00018D1E069002820DA26F020061DE0D8F89F
:10050000180000EB800005EB40003038C8F81800F8
:100510002046E1688847054605F05AFB0028EED1E1
:10052000012F0AD02E2D08D12046E16888477F1C74
:100530000546022F46F02006C4DBA069002803DA36
:10054000404246F00106A061F00701D026F01006F7
:100550006C2D0BD0682D09D04C2D39D06A2D35D09B
:10056000742D35D07A2D33D016E038E0E1682F466F
:1005700020468847B842054609D16C2F26D04FF453
:100580008060E168064320468847054604E06C2FFA
:100590001AD04FF4807006430DB3A5F1410019281D
:1005A00002D8203546F400664A4629462046266091
:1005B0004E46FFF757FE80B101280BD0F61D26F0FE
:1005C000070000F1080956E74020E4E78020D8E75B
:1005D0000020D6E706F104094DE7284652E7206AD5
:1005E000BDE8F09FC49F050040EA0103024630B514
:1005F0009B0710D14FF0013400E008C208C91D1B51
:100600009D4315EAC41FF8D013F0FF0102F8011B47
:100610000DD01B0AF8E711F8013B002B02F8013B53
:1006200005D011F8013B002B02F8013BF3D130BD9E
:1006300010B5431C02E010F8011B71B18107FAD11B
:100640004FF0013202C88C1A8C4314EAC211F9D05F
:10065000C01A0A0603D0C01E10BDC01A10BD0A047D
:1006600001D0801E10BD0902FCD0401E10BD10B587
:10067000203AC0F00B80B1E81850203AA0E818509A
:10068000B1E81850A0E81850BFF4F5AF5FEA027C5B
:1006900024BFB1E81850A0E8185044BF18C918C0CA
:1006A000BDE810405FEA827C24BF51F8043B40F86B
:1006B000043B08BF7047D20728BF31F8023B48BF50
:1006C00011F8012B28BF20F8023B48BF00F8012B8E
:1006D00070474FF0000200B5134694469646203905
:1006E00022BFA0E80C50A0E80C50B1F12001BFF4EB
:1006F000F7AF090728BFA0E80C5048BF0CC05DF851
:1007000004EB890028BF40F8042B08BF704748BF9E
:1007100020F8022B11F0804F18BF00F8012B704712
:100720004FF0013C50F8042B51F8043B9A4221D180
:10073000A2EB0C03934313EACC1317D150F8042B0C
:1007400051F8043B9A4215D1A2EB0C03934313EAF0
:10075000CC130BD150F8042B51F8043B9A4209D129
:10076000A2EB0C03934313EACC13DBD04FF0000051
:10077000704700BFD01A01BAB1FA81F101F0180137
:1007800022FA01F0CB40C1F12001DBB2C0B2C01AA5
:100790002CFA01F3D11A914311EAC311E6D1704743
:1007A00070477047704770B5044685690068C10698
:1007B00001D5302600E02026C00707D070BDD4E95F
:1007C000012130469047206A401C20626D1EF6D5FC
:1007D00070BD70B5044685690078C00707D170BD4B
:1007E000D4E9012120209047206A401C20626D1E20
:1007F000F6D570BD09684A0501D540B27047C905F4
:10080000FCD500B2704709684A0501D5C0B27047EF
:10081000C905FCD580B2704770B50C460546012A63
:1008200005D02878800600D5EA69002302E001237C
:1008300005E05B1C934202D2E05C0028F9D1A86974
:10084000E618C01AA861286A184428622846FFF7EB
:10085000AAFF04E0D5E9012114F8010B9047B44246
:10086000F8D32846FFF7B5FF70BD2DE9F0470D46D8
:1008700099469246044600F124080168880604D58A
:10088000E06921F01001216000E00120A84201DDB3
:10089000471B00E00027A1697A1902EB0900081A3A
:1008A000A0612078C00602D42046FFF77CFF002616
:1008B00008E0D4E901211AF806009047206A401C9C
:1008C000761C20624E45F4DB2078C0060AD520460F
:1008D000FFF769FF06E0D4E9012130209047206A44
:1008E000401C2062381EA7F10107F4DC07E0D4E9C0
:1008F000012118F805009047206A401C2062281E3C
:10090000A5F10105F3DC2046FFF763FF2078000620
:1009100002D50220BDE8F0870120FBE711680268DC
:10092000006A530501D508700AE0D30501D5088097
:1009300006E0130603D5C217C1E9000200E0086013
:100940000120704701694A1C02610878704700B5B0
:100950008FB0CDE901310021059105497944CDE9F8
:10096000031011466846FFF77BFD0FB000BD000085
:10097000E5FFFFFF0A6802F8010B0A607047D1E942
:1009800000239A4202D2531C0B6010707047000083
:100990002DE9FF5F15468A460446DFF8AC80F8442F
:1009A0000027D8E900103E46CDE9001010E03AF8E3
:1009B00016106A4602A800F00BFD411C07D02178F2
:1009C000890603D5E269391891420DD80744761C8F
:1009D0002078800602D5E069B84205DDAE42E6DB4C
:1009E0003AF816000028E2D1A069C01BA061204699
:1009F000FFF7D9FED8E90010CDE90010002017E07C
:100A00003AF818106A4602A800F0E2FCB0F1FF3F85
:100A100081460BD000250DF1080B05E0D4E901213A
:100A20001BF8050090476D1C4D45F7D308F10100F8
:100A3000B0428046E4DB206A384420622046FFF75B
:100A4000C8FEBDE8FF9F0000AA9A05002DE9F0410D
:100A50008046D21D22F007020025D2E90002F529C6
:100A600015A614D0011E72F1000106DA0023D0EBA6
:100A7000030063EB020211A608E0D8F800108B0710
:100A800001D50FA602E0490701D50EA601251146A2
:100A9000002408F1240704E000F09EF830323A55B3
:100AA000641C50EA0102F7D12B46324621464046EB
:100AB000BDE8F041FFF7D9BE000000002D000000A6
:100AC0002B0000002000000030B4002100F12404BD
:100AD00008E002F00705D208303542EA4372DB082D
:100AE0006554491C52EA0305F3D10468002310A29F
:100AF000250708D504F020040C4304D0C469012361
:100B00000CA2641EC46130BCFFF7AFBE10B5044632
:100B100021461068FFF777FE02462046BDE81040E8
:100B20000023D1E7D21D22F00701D1E90023CBE752
:100B30000000000030000000F0B40D4601880905F7
:100B400002D5214C7C4402E01F4C7C440E34002131
:100B500000F1240608E002F00F071209E75D42EAFF
:100B600003721B097754491C52EA0307F3D1027838
:100B70000023120704D5702D06D009B102231134C9
:100B80002246F0BCFFF771BE01231034F8E770B5C0
:100B900004460D4621461068FFF735FE02462946F9
:100BA0002046BDE870400023C6E7D21D22F00703AF
:100BB000D3E90023C0E70368126843F02003036011
:100BC0000823C3610023B7E70C99050001491820E9
:100BD000ABBEFEE72600020030B5B0F10A024FEAD4
:100BE000900E71F100034EEA817EB0EB0E0061EBD6
:100BF00091014FEA101E4EEA017E10EB0E0041EB10
:100C000011114FEA102E4EEA016E10EB0E0041EB6F
:100C100011214FEA104E4EEA014E10EB0E0041EB4F
:100C20001141401841F100014FEAD00040EA417003
:100C30004FEAD10110EB80054FEA810444EA907439
:100C400044EB01046D1944EB0404521BA3414FF023
:100C5000000348BF0A3200D530BD401C41F10001FD
:100C600030BD70472DE9FF4F0C461E464FF0FF3751
:100C70008BB0D2E90001DDF860800A908A46C1F3AA
:100C80000A5505B93D46002108464FF00000BAF16B
:100C9000000F00F4400005DA00EB80004FF4400143
:100CA00001EA50004FEA9059B9F1010F00DDB94651
:100CB0000A9850EA4A000ED044F61050A5F2FF35CB
:100CC00045432F14B8F1000F1ED07542291E1EDDBA
:100CD000C9F100021CE0B8F1010F4FF0000001D093
:100CE000302103E0F24305E02154401CB042FBDB1D
:100CF00030460022002121540B99C1F80880C1E937
:100D000000200FB0BDE8F08FBD1B6D1CDEE74A462A
:100D100000DA694206A800F0EDFB06AB93E8070095
:100D200003AB83E8070050460A9900F05BFC8DE8AE
:100D30000700A0F500501F3800900398002D09DD32
:100D400042F21F014A46084403A90390684600F096
:100D5000BAFE08E0A0F500504A461F3803A90390E8
:100D6000684600F0C4FE8DE807000004000C03D0C4
:100D70004FF0FF30410800E01046B8F1000F03D0FB
:100D80000022009215461EE0751E05D4FFF724FFD1
:100D9000303262556D1EF9D5B3460122084302D0A8
:100DA00000227F1C04E02078302801D100227F1E21
:100DB000002A099786D01DE0112D07DAFFF70CFFF6
:100DC000303262556D1C50EA0102F5D1084302D061
:100DD0000098C8B10EE00021681E05E0235C625C4B
:100DE00063542254401E491C8142F7DBAB46A81BCA
:100DF000401E0990002004F80B000B98099AC0F8D7
:100E00000880C0E9002B7CE711264FF0000859E765
:100E10002DE9F04F88460446D21D22F0070191B01B
:100E2000D1E90001CDE90A0104F093FE02460B98D6
:100E3000C00F01D02D2007E02068810701D52B20AD
:100E400002E0202101EAC000032A099001D0072A0C
:100E500005DB03464146204600F00CFB0BE1207801
:100E6000800601D5E06900E00620B8F1650F8146F3
:100E700006D0B8F1660F18D0B8F1670F70D131E025
:100E80000020B9F1110F009001DB112301E009F1FD
:100E900001030AAA01A90CA8FFF7E4FEDDE90C7022
:100EA000002609F10105834647E001204B460090EA
:100EB0004FF000470AAA01A90CA8FFF7D3FEDDE90D
:100EC0000DB00C995D46002610B909F101000D180E
:100ED000B9EB050003D4C0F1FF3609F10105A5EB1C
:100EE00009002BE0B9F1010F01DA4FF001090020F0
:100EF000B9F1110F0090484601DD112300E00346CF
:100F00000AAA01A90CA8FFF7ADFEDDE90C704D4659
:100F100000268346207800070AD4AB4500DA5D46F8
:100F200001A8012D04DD411911F8011C302907D059
:100F30004F4502DA17F1040F04DA012082460FE070
:100F40006D1EEEE7002F02DCED1B3E4403E0781C33
:100F5000A84200DD7D1CB81B00F1010A4FF00047DC
:100F60002078000703D4AA4501DB4FF0FF3A0021A7
:100F7000B7F1004F0DF143088DF8431024D0022043
:100F80002B23002F01DA7F422D230A21021EA0F11C
:100F9000010000DC5FB197FBF1FC97FBF1F201FB74
:100FA0001C7C17460CF1300C08F801CDEEE7A8F1D7
:100FB000010003702188090501D5452100E0652164
:100FC000A0F1010800F8011C09980FA9A1EB08077E
:100FD000FF1D00B10120411901EBEA70A1693844FD
:100FE000081A401EA0612078C00602D42046FFF7F0
:100FF000DAFB099828B1D4E901219047206A401C06
:1010000020622078C00622D52046FFF7CCFB1EE0E8
:10101000002E04DBB34502DD01A8805D00E0302036
:10102000D4E901219047206A401C2062761CAAF175
:1010300001005FEA000A0AD100F018FAC0680168EE
:10104000405CD4E901219047206A401C2062281EA0
:10105000A5F10105DCDC07E0D4E9012118F8010B5A
:101060009047206A401C2062381EA7F10107F3DC7C
:101070002046FFF7AEFB032011B043E62DE9F04F09
:1010800004460D46D21D22F0070089B0D0E9009237
:1010900048461746394604F05CFD0246F80F01D079
:1010A0002D2307E02068810701D52B2302E02021B2
:1010B00001EAC0038DF820300BB1012000E00020D0
:1010C000032A824601D0072A04DB2946204600F085
:1010D000D1F93DE12078800601D40D2500E0E569D5
:1010E000C7F30A560D2D49DA00214FEA175B08466F
:1010F0004FF00000002F00F4400007DA00EB800002
:101100004FF4400100EBD07001EA60008115012925
:1011100001DD4FF0FF3100224FEA850CBCF1180FC2
:1011200006D31346ACF118004FF08052C24003E0E2
:101130004FF4801323FA0CF30CF10C0CBCF1200FCC
:1011400004D3ACF1200C09FA0CF001E007FA0CF022
:1011500000294FF0004801DD18B90FE00ED14045DD
:101160000CD319EB02095F4121B9404502D19F43DD
:1011700029EA0209BBEB175F00D0761C2088000526
:1011800002D57B48784402E079487844193808AAA7
:10119000302302F80A30037C0AF10101002E0AF123
:1011A000020A53546A4602DC4FF0300101E04FF06E
:1011B00031014FF001088DF8001002D0A6F2FF3681
:1011C00003E059EA470100D06A4E002D02DC217885
:1011D000090704D54FF002082E218DF80110C446EE
:1011E00000210BE0C7F303433F01C35C491C6D1EA4
:1011F00002F80830052908F1010801DA002DF1DCB8
:1012000000210CE000EB1973491C1B786D1E0829A6
:1012100002F808304FEA091908F1010801DA002D37
:10122000F0DC2178890602D514E0A8F10108E04538
:1012300005DD02EB080111F8011C3029F5D0B8F1E9
:10124000000F07DD02EB080111F8011C2E2901D166
:10125000A8F10108002D05DD3E2102F808106D1EE1
:1012600008F10108407C002E02F8080008F101088E
:1012700004DA2D20764202F8080002E02B2002F862
:1012800008000A214FF47A70864208F101080BDB4E
:1012900096FBF0F3303302F8083096FBF0F308F1D8
:1012A000010800FB136601E0642E0CDB642096FB52
:1012B000F0F3303302F8083096FBF0F308F1010840
:1012C00000FB136601E00A2E06DB96FBF1F03030DE
:1012D00002F8080008F1010896FBF1F001FB10602C
:1012E000303002F80800A16908F1010808EB050296
:1012F00002EB0A00081AA0612078C00602D420463A
:10130000FFF751FA216A08AE01EB0A00206204E0FF
:10131000D4E9012116F8010B9047BAF1010AF7D27E
:101320002078C00602D52046FFF73DFA6E4609E058
:1013300016F8010B3E280FD0D4E901219047206A0E
:10134000401C2062B8F10108F2D22046FFF741FAB2
:1013500009B00320BDE8F08F206A2844206203E032
:10136000D4E90121302090476D1EEBD3F8E700004F
:101370000793050002FCFFFF10B5436913B1AFF3FB
:10138000008001E0FFF748FA012010BD127800F15B
:1013900024010A7000224A700122EDE711684FF023
:1013A000FF32E9E710B5436913B1AFF3008001E004
:1013B000FFF7EEFA012010BD128800F124018284AB
:1013C0000022C2840122EDE711684FF0FF32E9E705
:1013D00070B516460C46054600F040F8036893F8D1
:1013E0000101012806D0FF2C0FD8185D68B101203B
:1013F0002C7070BDD3F807013246214603F2071363
:1014000003442846BDE8704018474FF0FF3070BDD8
:101410007047754600F0E2F8AE460500694653464F
:1014200020F00700854618B020B5FEF795FFBDE80F
:1014300020404FF000064FF000074FF000084FF03B
:10144000000B21F00701AC46ACE8C009ACE8C009CC
:10145000ACE8C009ACE8C0098D46704710B500F093
:1014600005F8001D10BD00BF69A2030000487047C9
:10147000F0B601202DE9F0411F460446032601681D
:10148000072A01F4006004DB08B116A505E016A5E3
:1014900003E008B115A500E015A521F010002060BB
:1014A000A069C01EA0610FB1401EA0612046FFF7D9
:1014B0007AF94FB1D4E9012138469047206A401C9F
:1014C0002062C01C206206E0206AFAE7D4E901210C
:1014D00015F8010B9047761EF8D22046FFF779F9F0
:1014E000BDE8F0814E414E006E616E00494E4600EF
:1014F000696E66002DE9F047814616468AB033488A
:1015000078440DC88DE80D0030487844801C03AC49
:101510000DC884E80D0041F69B300844372190FB4C
:10152000F1F290FBF1F5A5F1800501FB12041B3CE3
:1015300002D56442012000E00020DFF890A0804640
:101540000027FA44AAF1BE0A0DE0E00709D03246AE
:10155000684607EB47010AEB810100F0C8FA8DE805
:10156000070064107F1C002CEFD1184F7F44AC3F64
:1015700018E0E80714D007EB04100DF1180A90E802
:101580000E008AE80E00C068F04201D19819089058
:10159000324606A903A800F0AAFA03AB83E80700C5
:1015A0006D10641C002DE4D132466946B8F1000F7D
:1015B00003A802D000F087FA01E000F098FAC9E928
:1015C0000001C9F808200AB0BDE8F0871C900500AA
:1015D0000446AFF300802046FEF7A9FE004870479E
:1015E000D0B601205FEA400C08BF91F0000F4FEA2F
:1015F0008C234FEAC12243EA51514FEA1C5018BFD5
:1016000000F5F0404FEA300018BF41F000415FEABA
:101610006C5C00F02980BCF1FF3F08BF40F08040C7
:101620007047130C06BF12044FF0100C4FF0000C63
:10163000130E04BF12020CF1080C130F04BF1201A9
:101640000CF1040C930F04BF92000CF1020CD30FA9
:1016500004BF52000CF1010C11464FF00002A0F142
:101660001F00A0EB0C00704711F0004F08BF70473F
:1016700031F000413FF4D5AF0B0C06BF09044FF029
:10168000100C4FF0000C0B0E04BF09020CF1080CFB
:101690000B0F04BF09010CF1040C8B0F04BF890070
:1016A0000CF1020CCB0F04BF49000CF1010CCCF182
:1016B0002003A0EB0C0022FA03F302FA0CF241EA39
:1016C000030100F10100704720F07F4C80EA030025
:1016D00023F07F47ACEB070303F57C5300F0004099
:1016E00003F1FF032DE980494FEA154B09B44FEA96
:1016F000144325EA0B4E24EA03480FF2042606EBB6
:10170000132749083E785FEA320203FB0667C7F5F4
:10171000000707FB06F64FEA54374FEAD64606F1B4
:10172000020607FB066CCCF1005C4FEA1C472CEA72
:10173000074C07FB06F40CFB06F504EB15464FEAD5
:10174000961634BF00204FF000404FEAD13706FB19
:1017500007FC4FEA1C4C0CFB0BF7D21B03FB0CF7EE
:1017600061EB07010CFB0EF7B0EB074072EB174281
:101770000CFB08F734BFA2EB0742B2EB074261EB68
:1017800017414FEA0C444FEA910706FB07FC4FEA6A
:101790001C4C0CFB0BF7B0EBC74072EB573203FB52
:1017A0000CF734BFA2EBC742B2EBC74261EB573133
:1017B0000CFB0EF7B0EBC70072EB57720CFB08F78F
:1017C00034BFA2EBC702B2EBC70261EB5771039FB4
:1017D0004FEA816141EA921104EBCC044FEAD13720
:1017E0004FEA826206FB07FC42EA90124FEA8060F1
:1017F0004FEA1C4C0CFB0BF7D21B03FB0CF761EB05
:1018000007010CFB0EF7B0EB074072EB17420CFB25
:1018100008F734BFA2EB0742B2EB074261EB174176
:101820004FEA8C554FEA910704EB9C2406FB07FC1A
:101830004FEA1C4C0CFB0BF7B0EBC74072EB573276
:1018400003FB0CF734BFA2EBC742B2EBC74261EB1C
:1018500057310CFB0EF7B0EBC70072EB57720CFB65
:1018600008F734BFA2EBC702B2EBC70261EB5771B6
:1018700015EB4C254FEA816141EA92114FEA8262F1
:101880004FEAD13742EA901206FB07FC44F100040C
:101890004FEA80604FEA1C4C0CFB0BF7D21B03FB9A
:1018A0000CF761EB07010CFB0EF7B0EB074072EB96
:1018B00017420CFB08F734BFA2EB0742B2EB07421A
:1018C00061EB174115EB1C154FEA813141EA92415A
:1018D0004FEA823242EA90424FEA80304FEA0C7679
:1018E00044F1000448EA03434EEA0B484FF0000E6F
:1018F000B2EB080C71EB030724BF624639464EEB8E
:101900000E0E4FF0000B0018524149414BEB0B0BF0
:10191000B2EB080C71EB03077BF1000B24BF6246AE
:1019200039464EEB0E0E4FF0000B00185241494164
:101930004BEB0B0BB2EB080C71EB03077BF1000BCD
:1019400024BF624639464EEB0E0E51EA020718BF1D
:1019500046F0010616EB0E7655F1000254F1000137
:1019600003D5BDE88901BDE80088BDE88901BDE86F
:101970000048B619524141EB0101A3F10103704740
:1019800080807F7E7D7C7B7A7978777676757473BC
:10199000727171706F6E6E6D6C6C6B6A6A6968687B
:1019A000676666656464636362616160605F5F5E11
:1019B0005E5D5D5C5C5B5B5A5A5959585857575687
:1019C00056555555545453535252525151505050EC
:1019D0004F4F4F4E4E4D4D4D4C4C4C4B4B4B4A4A3E
:1019E0004A49494948484847474747464646454582
:1019F00045444444444343434342424242414141BB
:101A0000002B26D4770021D01CB54FEA370703B44A
:101A10004FF010004FF010014FF000000FBCBDE878
:101A200010400BF1010BBBF1010F08BF5FEA170774
:101A300022BF12F1010211F101014FF0004143F107
:101A4000000300F0004043EA00007047F9D3570854
:101A5000DAE746EA064613F1400F4FEA16461FDD65
:101A600013F1200FDFBF16430A46002120335B42EB
:101A7000C8D0C3F1200746EA064602FA07F74FEA44
:101A8000164646EA0706C3F1200722FA03F201FAD6
:101A900007F721FA03F14FF0000342EA0702B1E72A
:101AA00046EA020646EA06464FEA164646EA0106B6
:101AB000BCBF46EA0646360C4FF000034FF000026A
:101AC0004FF000019EE72DE9C048934630B491E8FD
:101AD000380007C831EA400C48BF34EA430C03D54C
:101AE000FFF7F2FDFFF78CFFF0BCBDE800882DE9A1
:101AF000C048934630B491E8380007C810F0804FD2
:101B000008BF13F0804F03D100F005F8FFF778FF0E
:101B1000F0BCBDE8008820F07F4780EA030023F096
:101B20007F4C07EB0C03A3F57C5300F00040A3F1BE
:101B3000FE0392F0000F00F0B38095F0000F00F06C
:101B400077802DE901494FEA11404FEA144621EA16
:101B5000004800FB06FC24EA064708FB06F607FBE4
:101B600008F800FB07F718EB06484CEB164C4FEA59
:101B7000124B18EB07484FEA15464CEB174022EA88
:101B80000B4E0BFB06FC25EA06470EFB06F607FB91
:101B90000EFE0BFB07F71EEB064E4CEB164C4FF000
:101BA00000061EEB074E4CEB174B18EB0B0840F1F1
:101BB000000018EB0E0B58EB000840F100008F1AE4
:101BC0004FF000013CBFC943661B14BFB5EB040CCA
:101BD00000213CBFC943F61B4FEA17444EEA8E0E64
:101BE00027EA04454FEA1C4704FB07622CEA074C2E
:101BF00005FB07F70CFB05F604FB0CFC16EB074690
:101C000042EB174216EB0C4642EB1C421BEB06065E
:101C100058EB0202414146EA9E0601D5BDE8018922
:101C2000B619524141EB0101A3F10103BDE801895D
:101C30004FEA14454FEA114724EA054621EA074CCA
:101C400005FB07F406FB07F70CFB06F105FB0CFC94
:101C500011EB074144EB17444FEA124711EB0C41DB
:101C600044EB1C4422EA074C05FB07F206FB07F78E
:101C70000CFB06F605FB0CFC16EB074642EB174285
:101C800016EB0C4642EB1C456A1854F1000148BFA4
:101C90007047B619524141EB0101A3F101037047AE
:101CA00095F0000F37D04FEA11424FEA144721EA6E
:101CB000024624EA074C02FB07F106FB07F70CFB80
:101CC00006F402FB0CFC14EB074441EB17414FEA0E
:101CD000154714EB0C4441EB1C4125EA074C02FB71
:101CE00007F506FB07F70CFB06F602FB0CFC16EBF0
:101CF000074645EB174516EB0C4645EB1C421219FF
:101D000051F1000148BF7047B619524141EB010142
:101D1000A3F1010370474FEA14454FEA114724EA43
:101D2000054621EA074C05FB07F106FB07F70CFB0C
:101D300006F24FF0000605FB0CFC12EB074241EBEC
:101D4000174112EB0C4251EB1C4148BF70479218EF
:101D500041EB0101A3F101037047000038B50446CF
:101D600000200090206803F045FA00284FD1206839
:101D700080682849084048B1A06D40F01000A06577
:101D8000E06D40F00100E065012038BD206803F0FF
:101D90001BFA00BF2048806800F0E07000F40000EB
:101DA00080B11E4800681E49B0FBF1F0401C00EBFA
:101DB00040008000009002E00098401E00900098D3
:101DC0000028F9D100F042FD05461AE0206803F032
:101DD00011FA10B9206803F0F7F900F037FD401B45
:101DE00002280ED92068006800F0010048B9A06DF3
:101DF00040F01000A065E06D40F00100E0650120BA
:101E0000C3E72068006800F001000028DED0002051
:101E1000BBE700003F000080000304500C000020DE
:101E2000400D030000BFFEE7704772B67047000028
:101E30002DE9FC5F05460C46002001900090FE490C
:101E4000E068884200D000E000BF00BF95F8540071
:101E5000012802D10220BDE8FC9F012085F8540032
:101E600000BF286803F0D0F900287DD1676860685A
:101E7000052815D86068022806D0032806D0042853
:101E800006D0052809D105E00C2708E0122706E056
:101E9000182704E04FF4807701E0062700BF00BF59
:101EA0002868216800F13003C7F3012C03EB8C0292
:101EB000136807F01F0B4FF01F0C0CFA0BFC23EA02
:101EC0000C0307F01F0CC1F3846B0BFA0CFB43EA05
:101ED0000B03136000BF286803F096F98246286858
:101EE00003F083F98146BAF1000F3FD1B9F1000F39
:101EF000FBD1A068B0F1004F0AD121680022286808
:101F000003F090F94FF00041286803F0B0F908E0C1
:101F1000A2682168286803F085F90021286803F089
:101F2000A6F960692968C968C1F3C101490000FACE
:101F300001F8206904281AD028682268216900F174
:101F4000600C0CEB8103D3F800C0DFF8F0B20CEAB0
:101F50000B0C02F0F84B4BF0004B4BEA080B4CEA31
:101F60000B0CC3F800C000E0B7E100BFA7E0002100
:101F7000286803F031F9C0F3120030B90021286855
:101F800003F02AF9C0F3846007E00021286803F019
:101F900023F990FAA0F0B0FA80F02168C1F31201A1
:101FA00019B92168C1F3846104E0216891FAA1F1B3
:101FB000B1FA81F1884204D100221146286803F069
:101FC0004BF90121286803F007F9C0F3120030B97A
:101FD0000121286803F000F9C0F3846007E00121C3
:101FE000286803F0F9F890FAA0F0B0FA80F02168C0
:101FF000C1F3120119B92168C1F3846104E02168B9
:1020000091FAA1F1B1FA81F1884204D100220121B3
:10201000286803F021F90221286803F0DDF8C0F3F5
:10202000120030B90221286803F0D6F8C0F38460AA
:1020300007E00221286803F0CFF890FAA0F0B0FA88
:1020400080F02168C1F3120119B92168C1F38461DC
:1020500004E0216891FAA1F1B1FA81F1884204D13A
:1020600000220221286803F0F7F80321286803F012
:10207000B3F8C0F3120030B90321286803F0ACF8BC
:10208000C0F3846007E00321286803F0A5F890FA04
:10209000A0F0B0FA80F02168C1F3120119B92168EB
:1020A000C1F3846104E0216891FAA1F1B1FA81F1F0
:1020B000884204D100220321286803F0CDF8286863
:1020C00003F098F8002872D12868E2682168D0F8F7
:1020D000B030C1F3120C23EA0C0302F0180BDFF846
:1020E00060C12CFA0BFC0CEA010C43EA0C03C0F8AB
:1020F000B03000BF5049E068884258D12368C3F32C
:1021000012031BB92368C3F3846304E0236893FAC2
:10211000A3F3B3FA83F35B1C03F01F03092B3ED830
:102120002368C3F312031BB92368C3F3846304E079
:10213000236893FAA3F3B3FA83F35B1C03F01F0342
:102140004FF0010C0CFA03FC2368C3F312031BB914
:102150002368C3F3846304E0236893FAA3F3B3FA18
:1021600083F35B1C03F01F034CEA836C2368C3F307
:1021700012031BB92368C3F3846304E0236893FA52
:10218000A3F3B3FA83F35B1C03F01F0303EB4303D6
:102190004FF0000B4BEA03534CEA03033FE0236884
:1021A000C3F3120323B92368C3F3846305E03BE060
:1021B000236893FAA3F3B3FA83F35B1C03F01F03C2
:1021C0004FF0010C0CFA03FC2368C3F312031BB994
:1021D0002368C3F3846304E0236893FAA3F3B3FA98
:1021E00083F35B1C03F01F034CEA836C2368C3F387
:1021F00012031BB92368C3F3846304E0236893FAD2
:10220000A3F3B3FA83F35B1C03F01F030A3B03EB56
:1022100043034FF0007B4BEA03534CEA0303194698
:10222000A268286802F0FEFF06492068084088B3CB
:1022300000BF0548806809E000007F4000F0FF0310
:10224000FFFF0700000008800003045000F0E07664
:1022500000BF2849206888421DD106F40000D0B98B
:1022600025492868884237D146F40001234802F006
:10227000EDFF234800682349B0FBF1F0401C00EB60
:1022800040008000009002E00098401E00900098FE
:102290000028F9D120E01C49206888420CD106F0C2
:1022A000807048B914492868884215D146F0807179
:1022B000124802F0CBFF0FE01449206888420BD18E
:1022C00006F4800040B90C492868884204D146F4DD
:1022D00080010A4802F0BAFF05E0A86D40F0200036
:1022E000A8650120019000BF002085F8540000BFC0
:1022F0000198B0E5000052C70000045000030450EC
:102300000C000020400D0300000084CB0100008081
:1023100001460868006C70472DE9F84304464FF009
:1023200000080020009014B90120BDE8F88320695E
:1023300020B12020005D012800D100BFA06D30B980
:10234000204600F0E3F80020E06584F8540020689F
:102350008168C1F3407131B120688168644A1140DD
:10236000816000BF00BF206802F049FFB0B920685B
:102370008168604A114041F08051816000BF5E4831
:1023800000685E49B0FBF1F0401C4000009002E0A4
:102390000098401E009000980028F9D1206802F0B3
:1023A0002EFF48B9A06D40F01000A065E06D40F030
:1023B0000100E0654FF00108206802F025FF0646A5
:1023C000A06D00F0100000287BD1002EFCD1A06D84
:1023D00020F4807040F00200A065206802F00AFF3F
:1023E00068B9474802F006FF48B9606845498968FE
:1023F00021F47C110143434A916000BF00BF607E1D
:10240000616B41EA4030E1680843A168084320213C
:10241000095D40EA01452020005D012803D1A08C20
:10242000401E45EA4045A06A28B1208D00F4707036
:10243000E16A084305432068C068334908402843DF
:102440002168C860206802F0D0FE07462EBB27BB7B
:10245000207EE16C41EA803194F8300041EA400589
:102460002068C06844F20601884328432168C86098
:1024700094F83800012811D1E06B40F00101206C84
:102480000843616C0843A16C08432168096940F264
:10249000FC72914308432168086105E020680069E7
:1024A00020F0010021680861206901280AD1206814
:1024B000006B20F00F00E169491E084321680863A2
:1024C00006E00CE02068006B20F00F002168086334
:1024D000A06D20F0020040F00100A06505E0A06DB5
:1024E00040F01000A0654FF0010840461DE70000D5
:1024F000C0FFFF5FC0FFFF7F0C000020400D030006
:10250000000004500003045007C0F0FF10B5A0B055
:10251000044614211BA8FEF7DCF8682101A8FEF789
:10252000D8F82249206888423DD14FF4804001907C
:102530008003189003200290012103910821049147
:1025400007210591022106910791C905089101A86B
:1025500000F05CFD08B1FFF768FC00BF1448C06CD8
:1025600040F400501249C8640846C06C00F40050A2
:10257000009000BF00BF00BF0846C06C40F00100E3
:10258000C8640846C06C00F00100009000BF00BFA6
:1025900020201B900B201C9000201D901BA94FF0A9
:1025A000904000F065F820B010BD0000000004501D
:1025B0000010024070B50446206802F025FE002895
:1025C0003FD100BF94F85400012801D1022070BD12
:1025D000012084F8540000BF2046FFF7BFFB0546EA
:1025E00055BBA06D40F60161884340F48070A06542
:1025F000A06D00F48050B0F5805F04D1E06D20F054
:102600000600E06501E00020E0651C20216808600C
:1026100000BF002084F8540000BF2068C06800F0AC
:10262000007028B1A06D20F4005040F48050A065E7
:10263000206802F0EFFD05E000BF002084F85400A0
:1026400000E002252846C2E770B5044600F0FEF817
:1026500006462546681C10B104480078054400BFB2
:1026600000F0F4F8801BA842FAD370BD08000020E7
:1026700078B503460A460021C5E001268E4015685C
:1026800005EA0604002C73D0157905F00305012D29
:1026900004D0157905F00305022D13D198684E007A
:1026A0000325B540A8434E00D568B540284398603F
:1026B000586801258D40A8431579C5F300158D4054
:1026C00028435860157905F00305032D09D0D86813
:1026D0004E000325B540A8434E009568B5402843F9
:1026E000D860157905F00305022D13D1CE0803F14A
:1026F000200555F826004D07EE0E0F25B540A843DE
:102700004E07F60E1569B5402843CE0803F12005A3
:1027100045F8260018684E000325B540A8431579F2
:1027200005F003054E00B54028431860556805F4D0
:102730004035002D66D000BF364D2D6E45F00105A9
:10274000344E356635462D6E05F00105009500BF07
:1027500000BF4FEAB6358E0855F826008D072E0FBC
:102760000F25B540A843B3F1904F02D1002515E0E5
:1027700048E0294DAB4201D101250FE0274DAB4286
:1027800001D102250AE0264DAB4201D1032505E027
:10279000244DAB4201D1042500E007258E07360FFA
:1027A000B5402843204D8E0845F826001F4D286867
:1027B000A043556805F4801505B120431B4D2860E2
:1027C0002D1D2868A043556805F4001505B1204368
:1027D000164D2D1D2860154D2D1F2868A0435568E6
:1027E00005F4003505B12043104D2D1F28602D1F25
:1027F0002868A043556805F4803505B120430B4D8A
:10280000083D2860491C1568CD40002D7FF435AF88
:1028100078BD000000100240000400480008004895
:10282000000C004800100048080001400804014066
:10283000024613690B400BB1012000E000207047F5
:102840000AB1816100E081627047000001480068C0
:102850007047000000000020024692F84100202846
:102860002DD100BF92F84000012801D1022070470D
:10287000012082F8400000BF242082F84100106847
:10288000006820F00100136818601068006820F4E8
:102890008050136818601068006808431368186057
:1028A0001068006840F0010013681860202082F86A
:1028B000410000BF002082F8400000BFD7E702209F
:1028C000D5E710B502460B4692F8410020282AD1E0
:1028D00000BF92F84000012801D1022010BD012064
:1028E00082F8400000BF242082F841001068006890
:1028F00020F00100146820601068016821F4706104
:1029000041EA0321106801601068006840F001008E
:1029100014682060202082F8410000BF002082F867
:10292000400000BFDAE70220D8E7000010B50446F7
:102930000CB9012010BD94F8410028B9002084F89A
:102940004000204600F0FAF9242084F84100206875
:10295000006820F0010021680860606820F0706065
:10296000216808612068806820F400402168886040
:10297000E068012805D1A06840F400402168886023
:1029800004E0A06840F4044021688860E068022800
:1029900006D12068406840F400602168486005E086
:1029A0002068406820F40060216848602068406822
:1029B00013490843216848602068C06820F400403B
:1029C0002168C860D4E904010843A16940EA0120F4
:1029D0002168C860D4E907010843216808602068BD
:1029E000006840F001002168086000206064202039
:1029F00084F841000020206384F8420000BF99E77A
:102A0000008000022DE9FC5F0446894692469B4601
:102A1000DDE90C780E9E94F8410020287ED117B194
:102A2000B8F1000F05D14FF4007060640120BDE8DB
:102A3000FC9F00BF94F84000012801D10220F6E776
:102A4000012084F8400000BFFFF700FF054619236E
:102A50000122D1032046009502F09CF908B1012023
:102A6000E5E7222084F84100402084F8420000205D
:102A700060646762A4F82A8060635B4652464946F8
:102A80002046CDE9006502F0EDF830B100BF00202E
:102A900084F8400000BF0120C9E7608DFF280CD9F1
:102AA000012020853D48009094F828204FF0807345
:102AB0004946204602F052F90BE0608D20853748E8
:102AC000009094F828204FF000734946204602F009
:102AD00045F900BF3346002204212046009502F04C
:102AE00059F908B10120A2E72068406A616A0870BC
:102AF000606A401C6062208D401E2085608D401EF3
:102B00006085608D48B3208D38BB3346002280211C
:102B10002046009502F03EF918B100E03CE00120AB
:102B200085E7608DFF280CD90120208500200090CA
:102B300094F828204FF080734946204602F00EF9A1
:102B40000BE0608D20850020009094F828204FF045
:102B500000734946204602F001F9608D0028B9D182
:102B60002A463146204602F056F908B101205EE7B8
:102B700020202168C8612068406809490840216810
:102B80004860202084F84100002084F8420000BF03
:102B900084F8400000BF4AE7022048E70024008094
:102BA00000E800FE2DE9FC5F0446894692469B46FC
:102BB000DDE90C780E9E94F8410020287DD117B1F4
:102BC000B8F1000F05D14FF4007060640120BDE83A
:102BD000FC9F00BF94F84000012801D10220F6E7D5
:102BE000012084F8400000BFFFF730FE054619239E
:102BF0000122D1032046009502F0CCF808B1012053
:102C0000E5E7212084F84100402084F842000020BC
:102C100060646762A4F82A8060635B465246494656
:102C20002046CDE9006502F05BF830B100BF00201E
:102C300084F8400000BF0120C9E7608DFF280CD94F
:102C4000FF2020850020009094F828204FF080730A
:102C50004946204602F082F80BE0608D2085002076
:102C6000009094F828204FF000734946204602F067
:102C700075F800BF2A463146204602F0FCF808B13C
:102C80000120A4E7606A007821688862606A401CBD
:102C90006062608D401E6085208D401E2085608DA5
:102CA00040B3208D30BB3346002280212046009562
:102CB00002F070F810B1012089E73AE0608DFF283A
:102CC0000CD9FF2020850020009094F828204FF098
:102CD00080734946204602F041F80BE0608D208564
:102CE0000020009094F828204FF0007349462046B9
:102CF00002F034F8608D0028BCD12A4631462046C7
:102D000002F089F808B1012061E720202168C8613C
:102D1000206840680849084021684860202084F8FD
:102D20004100002084F8420000BF84F8400000BF4A
:102D30004DE702204BE7000000E800FE10B5A0B010
:102D4000044614211BA8FDF7C4FC682101A8FDF767
:102D5000C0FC1D492068884234D14FF48010019096
:102D60000020119001A800F051F908B1FFF75DF8BB
:102D700000BF1648C06C40F002001449C864084601
:102D8000C06C00F00200009000BF00BF4FF4406034
:102D90001B9012201C9000201D9003201E901F905D
:102DA0001BA90B48FFF764FC00BF0848C06D40F04A
:102DB00002000649C8650846C06D00F00200009098
:102DC00000BF00BF20B010BD0084004000100240D2
:102DD0000004004803480068034909780844014991
:102DE00008607047000000200800002010B5002493
:102DF000032000F0A9F80F2000F008F808B1012422
:102E000001E000F02FF8204610BD000070B5044628
:102E1000002511480078D8B10F4800784FF47A7136
:102E2000B1FBF0F00D490968B1FBF0F6304601F056
:102E30003DFB58B9102C07D200222146501E00F04D
:102E400045F80748046004E0012502E0012500E0A0
:102E50000125284670BD0000080000200C0000205D
:102E60000400002008B500BF0D48006E40F00100CE
:102E70000B4908660846006E00F00100009000BF94
:102E800000BF00BF0846806D40F08050886508464E
:102E9000806D00F08050009000BF00BF08BD0000B2
:102EA000001002400146084600280DDB00BF00BFAD
:102EB00000F01F0301229A4043099B0003F1E02325
:102EC000C3F8002100BF00BF00BF70472DE9F05FCD
:102ED00080460D461646002702F054FE0746394646
:102EE0002A46334601F00700C0F1070ABAF1040F81
:102EF00002D94FF0040A01E0C0F1070AD14600F1FF
:102F0000040ABAF1070F02D24FF0000A01E0A0F163
:102F1000030AD4464FF0010A0AFA09FAAAF1010A93
:102F20000AEA020A0AFA0CFA4FF0010B0BFA0CFB40
:102F3000ABF1010B0BEA030B4AEA0B0421464046B6
:102F400002F028FEBDE8F09F00BF00F00702064B2C
:102F500019684FF6FF031940044B0B4343EA022163
:102F6000014B196000BF70470CED00E00000FA054E
:102F70000246B2F5007F2AD11D48006800F4C06007
:102F8000B0F5007F32D01A48006820F4C06040F4E9
:102F90000070174B18601748006832235843164BCF
:102FA000B0FBF3F0411C00E0491E1148406900F4F9
:102FB0008060B0F5806F01D10029F5D10C484069DF
:102FC00000F48060B0F5806F10D10320704708488E
:102FD000006800F4C060B0F5806F07D00448006856
:102FE00020F4C06040F48060014B18600020EDE7E1
:102FF000007000400C00002040420F0002480068B2
:1030000000F4C06070470000007000402DE9F843F4
:1030100004460025A846208800F40060B0F5006F43
:1030200026D1E06C68B1B0F5000F03D0B0F5400FC9
:103030000ED10CE0F748C06840F48030F549C86014
:1030400008E00021201D02F0ABFA054602E001E095
:10305000012500BF00BF55B9EE488830006820F454
:103060004000E16C0843EB49C1F8880000E0A84645
:10307000206800F40030B0F5003F75D14FF0000932
:10308000E448806D012121EA107078B100BFE14869
:10309000806D40F08050DF4988650846806D00F003
:1030A0008050009000BF00BF4FF00109DA4800686F
:1030B00040F48070D8490860FFF7C8FB074606E077
:1030C000FFF7C4FBC01B022801D9032505E0D24845
:1030D000006800F480700028F2D000BF7DBBCD48AE
:1030E0009030006800F44076CEB1606EB04216D0E9
:1030F000C8489030006820F44076C648D0F8900068
:1031000040F48030C349C1F890000846D0F89000E0
:1031100020F48030C1F890000846C0F8906006F0B6
:103120000100A8B1FFF792FB074609E0FFF78EFB0D
:10313000C01B41F28831884202D9032507E016E01E
:10314000B4489030006800F002000028EED000BFC4
:103150005DB9B0489030006820F44070616E08435B
:10316000AC49C1F8900003E00CE0A84600E0A84696
:10317000B9F1010F05D1A748806D20F08050A54915
:10318000886500BF207800F0010048B1A148883070
:10319000006820F00300216A08439E49C1F88800B6
:1031A000207800F00200022809D19A48883000688F
:1031B00020F00C00616A08439649C1F88800207825
:1031C00000F00400042809D192488830006820F0FB
:1031D0003000A16A08438F49C1F88800207800F0C8
:1031E0000800082809D18B488830006820F0C0000A
:1031F000E16A08438749C1F88800207800F0200080
:10320000202809D183488830006820F44060216B71
:1032100008438049C1F88800208800F40070B0F5A8
:10322000007F09D17B488830006820F44020616C21
:1032300008437849C1F88800208800F48060B0F520
:10324000806F09D173488830006820F44010A16C69
:1032500008437049C1F88800207800F040004028F9
:1032600009D16C488830006820F44050616B0843F5
:103270006849C1F88800207800F08000802809D1D2
:1032800064488830006820F44040A16B08436149DD
:10329000C1F88800208800F48070B0F5807F09D1E3
:1032A0005C488830006820F44030E16B084359499D
:1032B000C1F88800206800F48010B0F5801F09D1A3
:1032C00054489C30006820F00300216C08435149A9
:1032D000C1F89C00208800F40050B0F5005F1FD1B9
:1032E0004C488830006820F04060216D084349490F
:1032F00088310860206DB0F1006F06D14548C06884
:1033000040F480104349C8600AE0206DB0F1806F3E
:1033100006D10121201D02F043F9054605B1A8465A
:10332000206800F40020B0F5002F1FD13948883004
:10333000006820F04060616D0843364988310860BC
:10334000606DB0F1006F06D13248C06840F4801063
:103350003049C8600AE0606DB0F1806F06D101218C
:10336000201D02F01DF9054605B1A846206800F4AD
:103370008020B0F5802F1FD126488830006820F0CB
:103380004060A16D0843234988310860A06DB0F109
:10339000006F06D11F48C06840F480101D49C86006
:1033A0000AE0A06DB0F1806F06D10121201D02F06E
:1033B000F7F8054605B1A846208800F48040B0F52E
:1033C000804F14D113488830006820F04050E16DE0
:1033D0000843104988310860E06DB0F1805F06D184
:1033E0000221201D02F0DCF8054605B1A846206840
:1033F00000F48030B0F5803F09D10648883000687D
:1034000020F00040216E08430249C1F88800404680
:10341000BDE8F88300100240007000402DE9F04143
:1034200004460D4614B90120BDE8F08163480068E8
:1034300000F00700A8420ED26048006820F00700A4
:1034400028435E4908600846006800F00700A8426B
:1034500001D00120E8E7207800F0020002280ED118
:103460005749A068896801F0F001884207D954489B
:10347000806820F0F000A1680843514988602078F6
:1034800000F0010078B36068032806D14C4800685A
:1034900000F00070D8B90120C6E76068022806D1A4
:1034A0004748006800F4003088B90120BCE7606834
:1034B00030B94348006800F0020040B90120B3E78A
:1034C0003F48006800F4806008B90120ACE73C4840
:1034D000806820F003006168084339498860FFF77D
:1034E000B5F9064609E010E0FFF7B0F9801B41F29C
:1034F0008831884201D9032096E73148806800F07E
:103500000C006168B0EB810FEED1207800F0020072
:1035100002280ED12A49A068896801F0F00188428A
:1035200007D22748806820F0F000A16808432449AA
:1035300088602248006800F00700A8420ED91F48A2
:10354000006820F0070028431C490860084600680E
:1035500000F00700A84201D0012065E7207800F0C4
:103560000400042807D11648806820F4E060E16870
:10357000084313498860207800F00800082808D123
:103580000F48806820F46050216940EAC1000C496E
:10359000886000F01DF80A498968C1F30311094ADF
:1035A000515C01F01F01C8400749086007480068E6
:1035B000FFF72CFC0746384636E7000000200240A3
:1035C0000010024074C103080C0000200400002019
:1035D000F0B500230020DFF8D4C0DCF808C00CF000
:1035E0000C01DFF8C8C0DCF80CC00CF0030719B1FF
:1035F0000C291ED1012F1CD1DFF8B0C0DCF800C0AF
:103600000CF0080CBCF1000F06D1DFF8A0C0DCF80C
:1036100094C0CCF3032305E0DFF890C0DCF800C0D1
:10362000CCF30313DFF888C05CF8233041B91846A7
:1036300006E0042901D11F4802E0082900D11E48F4
:103640000C2932D1DFF864C0DCF80CC00CF00304A4
:10365000012C09D0022C02D0032C04D101E0154A20
:1036600004E0154A02E000BF1A4600BF00BFDFF8C1
:103670003CC0DCF80CC0CCF3021C0CF10106DFF8F6
:103680002CC0DCF80CC0CCF3062C0CFB02FCBCFB01
:10369000F6F2DFF818C0DCF80CC0CCF3416C0CF18A
:1036A000010C4FEA4C05B2FBF5F0F0BD00100240F2
:1036B0008CC103080024F40000127A002DE9F843BD
:1036C000044614B90120BDE8F883F948806800F089
:1036D0000C06F748C06800F00307207800F01000DF
:1036E000102877D11EB10C2E76D1012F74D1F0485D
:1036F000006800F0020018B1A06908B90120E2E7F3
:10370000EB48216A006800F0080020B1E848006832
:1037100000F0F00005E0E6489430006800F47060C6
:10372000000981421FD9206A01F0FEFF08B1012083
:10373000C9E700BFDE48006840F00800DC490860C7
:103740000846006820F0F000216A0843D849086064
:1037500000BF0846406820F47F40E16940EA01204C
:10376000D34948601FE000BFD148006840F008001E
:10377000CF4908600846006820F0F000216A08433D
:10378000CB49086000BF0846406820F47F40E169EB
:1037900040EA0120C64948602EB9206A01F0C4FF02
:1037A00008B101208FE7FFF713FFC1498968C1F312
:1037B0000311C04A515C01F01F01C840BE490860B6
:1037C000BE480068FFF722FB8046B8F1000F4ED0DC
:1037D000404678E74BE0FFE7A06980B3B448006853
:1037E00040F00100B2490860FFF730F8054606E0F6
:1037F000FFF72CF8401B022801D9032063E7AC48EF
:10380000006800F002000028F2D000BFA84800685D
:1038100040F00800A64908600846006820F0F00063
:10382000216A0843A249086000BF0846406820F4A6
:103830007F40E16940EA01209D49486017E0FFE7C9
:103840009B48006820F0010099490860FEF7FEFFE0
:10385000054606E0FEF7FAFF401B022801D90320C7
:1038600031E79348006800F002000028F2D1207888
:1038700000F0010000285CD0082E03D00C2E0AD1E5
:10388000032F08D18A48006800F4003088B36068CC
:1038900078BB012017E700BF6068B0F5803F06D114
:1038A0008348006840F48030814908601AE060680D
:1038B000B0F5A02F0BD17E48006840F480207C49F1
:1038C00008600846006840F4803008600AE07848E4
:1038D000006820F48030764908600846006820F4CB
:1038E0008020086000BF606890B1FEF7AFFF05461A
:1038F00007E01EE0FEF7AAFF401B642801D9032061
:10390000E1E66B48006800F400300028F2D010E0D7
:10391000FEF79CFF054606E0FEF798FF401B642873
:1039200001D90320CFE66248006800F40030002887
:10393000F2D1207800F00200022852D1042E03D0E8
:103940000C2E14D1022F12D15948006800F4806067
:1039500018B1E06808B90120B5E65548406820F084
:10396000FE40217C40EA01605149486039E0E0684E
:1039700000B34F48006840F480704D490860FEF77E
:1039800065FF054606E0FEF761FF401B022801D9EE
:10399000032098E64648006800F480600028F2D0D2
:1039A0004348406820F0FE40217C40EA01604049E5
:1039B000486016E03E48006820F480703C4908608A
:1039C000FEF744FF054606E0FEF740FF401B0228D5
:1039D00001D9032077E63648006800F480600028AB
:1039E000F2D1207800F00800082836D16069D0B103
:1039F0002F489430006840F001002D49C1F8940030
:103A0000FEF724FF054606E0FEF720FF401B0228D4
:103A100001D9032057E626489430006800F00200E0
:103A20000028F1D019E022489430006820F001000D
:103A30001F49C1F89400FEF709FF054606E0FEF7AE
:103A400005FF401B022801D903203CE618489430AA
:103A5000006800F002000028F1D1207800F0040096
:103A6000042872D14FF000091148806D00F0805099
:103A700078B900BF0E48806D40F080500C498865D1
:103A80000846806D00F08050009000BF00BF4FF0EE
:103A900001090B48006800F4807000BB084800680A
:103AA00040F4807006490860FEF7D0FE054610E03D
:103AB0000010024074C103080C0000200400002024
:103AC00000700040FEF7C2FE401B022801D903200F
:103AD000F9E5CA48006800F480700028F2D000BF01
:103AE000A068012808D1C648006840F00100C44918
:103AF0009039C1F8900021E0A06805280FD1C04896
:103B0000006840F00400BE499039C1F890000846B2
:103B1000D0F8900040F00100C1F890000EE0B848E5
:103B2000006820F00100B6499039C1F890000846BD
:103B3000D0F8900020F00400C1F8900000BFA06809
:103B4000A0B1FEF783FE054609E02EE0FEF77EFEFB
:103B5000401B41F28831884201D90320B3E5A848CF
:103B6000006800F002000028F0D012E0FEF76EFEC0
:103B7000054608E0FEF76AFE401B41F288318842A4
:103B800001D903209FE59E48006800F0020000284C
:103B9000F0D1B9F1010F07D199489038806D20F02C
:103BA000805097499039886500BF207800F0200048
:103BB000202838D1606AD8B191480830006840F0B8
:103BC00001008F499039C1F89800FEF73FFE054685
:103BD00006E0FEF73BFE401B022801D9032072E5F8
:103BE00087480830006800F002000028F1D01AE091
:103BF00083480830006820F0010081499039C1F8FD
:103C00009800FEF723FE054606E0FEF71FFE401B68
:103C1000022801D9032056E579480830006800F0F1
:103C200002000028F1D1A06A00287DD0A06A0228F5
:103C30007BD173489038C76807F00301E06A81427E
:103C400025D107F07001206B401EB1EB001F1ED183
:103C500007F4FE41606BB1EB002F18D107F07841FB
:103C60003820005DB1EBC06F11D107F4C001A08F07
:103C70000122C2EB5000B1EB405F08D107F0C061F8
:103C80004020005DC2EB5000B1EB406F66D00C2EBF
:103C900062D05B489038006800F0806008B1012075
:103CA00011E557489038006820F0807054499039E9
:103CB0000860FEF7CBFD054606E0FEF7C7FD401B9A
:103CC000022801D90320FEE44D489038006800F036
:103CD00000700028F1D1D4E90B10401E41EA001118
:103CE000606B41EA0021A08F0122C2EB500041EA43
:103CF00040514020005DC2EB500041EA4061382055
:103D0000005D41EAC0603E499039C9683D4A1140B2
:103D100008433B499039C8600846006840F080700D
:103D200008600846C06801E053E03DE040F0807064
:103D3000C860FEF78BFD054606E0FEF787FD401BD9
:103D4000022801D90320BEE42D489038006800F015
:103D500000700028F1D04FE00120B4E428489038EA
:103D6000006800F00070A0BB25489038006840F063
:103D700080702349903908600846C06840F0807020
:103D8000C860FEF763FD054606E0FEF75FFD401BD9
:103D9000022801D9032096E419489038006800F001
:103DA00000700028F1D027E00C2E23D01448903862
:103DB000006820F08070124990390860FEF746FDD7
:103DC000054607E0FEF742FD401B022802D903200A
:103DD00079E411E00A489038006800F0007000288B
:103DE000F0D107489038C068074908400449903925
:103DF000C86001E0012066E4002064E40070004037
:103E0000901002408C809D01FCFFEEFE70B50446D0
:103E10000CB9012070BD606A38B96068B0F5827F66
:103E200000D105E00021E16102E000212161616132
:103E30000021A16294F85D0028B9002084F85C009C
:103E4000204600F05BF8022084F85D0020680068DE
:103E500020F0400021680860E068B0F5E06F01D90B
:103E6000002501E04FF48055E068B0F5706F05D093
:103E7000E068B0F5E06F01D00021A162A08800F4F5
:103E80008270218901F404410843217C01F0020180
:103E90000843217D01F001010843218B01F40071E9
:103EA0000843217F01F0380108432021095D01F01A
:103EB00080010843218D01F4005108432168086006
:103EC0000421A06901EA104094F8241001F01001C7
:103ED000084394F8341001F008010843A18901F463
:103EE0007061084305F48051084321684860002050
:103EF0002066012084F85D0000208BE710B586B0B5
:103F00000446142101A8FCF7E4FB2F4920688842ED
:103F10002AD100BF2D48006E40F480502B4908661E
:103F20000846006E00F48050009000BF00BF00BF44
:103F30000846C06C40F00100C8640846C06C00F040
:103F40000100009000BF00BFC2200190022002903B
:103F500000200390032004900520059001A94FF054
:103F60009040FEF785FB2DE019492068884229D151
:103F700000BF1648806D40F48040144988650846AB
:103F8000806D00F48040009000BF00BF00BF084675
:103F9000C06C40F00200C8640846C06C00F002002B
:103FA000009000BF00BF4FF46040019002200290DB
:103FB00000200390032004900520059001A90548E6
:103FC000FEF756FB06B010BD003001400010024065
:103FD00000380040000400482DE9F84304460F462D
:103FE00016461D46FEF732FC8046B14694F85D0049
:103FF000012802D00220BDE8F88307B10EB90120E4
:10400000F9E700BF94F85C00012801D10220F2E733
:10401000012084F85C0000BF032084F85D000020CC
:104020002066A763A687E6872064A4F84400A4F866
:1040300046002065E064A068B0F5004F0BD1206811
:10404000006820F04000216808602068006840F4A3
:104050008040216808602068006800F04000402827
:1040600005D02068006840F0400021680860E068E2
:10407000B0F5E06F37D9606810B1B9F1010F09D11F
:10408000A06B00882168C860A06B801CA063E08FD3
:10409000401EE08723E02068806800F002000228CC
:1040A0000AD1A06B00882168C860A06B801CA06347
:1040B000E08F401EE08712E0FEF7C8FBA0EB08008F
:1040C000A84201D3681C00B94DB9012084F85D00F5
:1040D00000BF002084F85C0000BF03208BE7E08F66
:1040E0000028D8D152E0606810B1B9F1010F17D1A2
:1040F000E08F01280AD9A06B00882168C860A06BF6
:10410000801CA063E08F801EE08709E0A06B007830
:1041100021680873A06B401CA063E08F401EE087FD
:1041200031E02068806800F00200022818D1E08F9A
:1041300001280AD9A06B00882168C860A06B801C88
:10414000A063E08F801EE0871DE0A06B00782168EF
:104150000873A06B401CA063E08F401EE08712E054
:10416000FEF774FBA0EB0800A84201D3681C00B95D
:104170004DB9012084F85D0000BF002084F85C0088
:1041800000BF032037E7E08F0028CAD14246294606
:10419000204601F017FB08B120202066A06850B926
:1041A00000BF002000902068C068009020688068F0
:1041B000009000BF00BF012084F85D0000BF002018
:1041C00084F85C0000BF206E08B1012013E70020D6
:1041D00011E72DE9FE4F04460F4690461D460C9E02
:1041E00001200090FEF732FB824694F85DB06068D3
:1041F0000190A9460295BBF1010F0BD00198B0F5D3
:10420000827F04D1A06810B9BBF1040F02D0022054
:10421000BDE8FE8F1FB1B8F1000F00D00DB901202D
:10422000F6E700BF94F85C00012801D10220EFE717
:10423000012084F85C0000BF94F85D00042802D0DF
:10424000052084F85D0000202066C4F84080A4F8B2
:104250004650A4F84450A763E587A587E06420652D
:10426000E068B0F5E06F02D80298012806D920680E
:10427000406820F480502168486005E0206840686C
:1042800040F48050216848602068006800F04000D9
:10429000402805D02068006840F040002168086090
:1042A000E068B0F5E06F56D9606810B1B9F1010F60
:1042B00009D1A06B00882168C860A06B801CA06336
:1042C000E08F401EE0873EE02068806800F002003A
:1042D000022810D1E08F70B1009801280BD1A06B9B
:1042E00000882168C860A06B801CA063E08F401E1E
:1042F000E087002000902068806800F0010080B115
:10430000B4F8460068B12068C068216C0880206C51
:10431000801C2064B4F84600401EA4F8460001202A
:104320000090FEF793FAA0EB0A00B0420BD3701C8A
:1043300048B1012084F85D0000BF002084F85C00D3
:1043400000BF032064E7E08F0028BDD1B4F8460029
:104350000028B9D18DE0606810B1B9F1010F17D113
:10436000E08F01280AD9A06B00882168C860A06B83
:10437000801CA063E08F801EE08709E0A06B0078BE
:1043800021680873A06B401CA063E08F401EE0878B
:1043900068E02068806800F0020002281ED1E08FEB
:1043A000E0B10098012819D1E08F01280AD9A06B4B
:1043B00000882168C860A06B801CA063E08F801E0D
:1043C000E08709E0A06B007821680873A06B401CAF
:1043D000A063E08F401EE087002000902068806886
:1043E00000F0010058B3B4F8460040B3B4F84600FA
:1043F000012816D92068C068216C0880206C801CB8
:104400002064B4F84600801EA4F84600B4F84600C4
:10441000012812D82068406840F480502168486024
:104420000BE02068007B216C0870206C401C20642D
:10443000B4F84600401EA4F8460001200090FEF7A4
:1044400005FAA0EB0A00B04201D3701C00B94EB9C6
:10445000012084F85D0000BF002084F85C0000BFEC
:104460000320D5E6E08F002893D1B4F84600002859
:104470008FD152463146204601F0A4F940B12020A8
:10448000206600BF002084F85C0000BF0120BFE66A
:10449000012084F85D0000BF002084F85C0000BFAC
:1044A000206E08B10120B3E60020B1E670B50446E5
:1044B0002546681EB0F1807F01D301200FE0681E01
:1044C0004FF0E02148610F214FF0FF3001F062FB17
:1044D00000204FF0E021886107200861002070BDB6
:1044E000704770477047000030B502460B4600BF6A
:1044F00092F83C00012801D1022030BD012082F851
:104500003C0000BF022082F83D001068416810683E
:104510008468174D1068A84203D121F470015868CF
:10452000014321F070011868014310684160104D8B
:104530001068A8420BD01068B0F1804F07D00D4D25
:104540001068A84203D00C4D1068A84205D124F091
:1045500080049868044310688460012082F83D005C
:1045600000BF002082F83C0000BF00BFC5E700008C
:10457000002C0140000400400040014010B50446FA
:104580000CB9012010BD94F83D0028B9002084F832
:104590003C00204600F02AF8022084F83D00211D4E
:1045A000206801F079FA012084F8480000BF84F8FF
:1045B0003E0001213F200155402001554120015579
:1045C000422001554320015500BF00BF012084F85F
:1045D000440045200155462001554720015500BFA4
:1045E000012084F83D000020CCE7000038B50446E7
:1045F0000D492068884215D100BF0C48806D40F0FD
:1046000010000A4988650846806D00F0100000908F
:1046100000BF00BF002211463620FEF757FC3620AF
:10462000FEF740FC38BD00000010004000100240C2
:10463000014691F83D00012801D001207047022079
:1046400081F83D000868C06840F001000B68D86040
:10465000144B086898420BD00868B0F1804F07D01F
:10466000114B0868984203D0104B0868984210D14B
:10467000086880680E4B00EA0302062A0FD0B2F5E4
:10468000803F0CD00868006840F001000B6818609B
:1046900005E00868006840F001000B681860002021
:1046A000CCE70000002C0140000400400040014025
:1046B000070001002DE9F04104460D4614B9012020
:1046C000BDE8F08194F83D0028B9002084F83C0052
:1046D000204600F055F8022084F83D0020688068EC
:1046E0002649084021688860211D206801F0D4F91E
:1046F0002068D0F80880206886692068076A2868E2
:1047000040EA080840F203308643A969A86840EAF5
:104710000120064340F60C4086434FF2F0008643EA
:10472000E969E86840EA0120064328690001296A2E
:1047300040EA0130064327F0220727F0880769691D
:10474000686840EA011007432068C0F808802068C4
:10475000866120680762012084F8480084F83E00E2
:1047600001213F200155012084F8440045200155D6
:10477000012084F83D000020A2E70000F8BFFEFF02
:1047800010B586B00446142101A8FBF7A2FF184912
:10479000206888422AD100BF1648006E40F40060AD
:1047A000144908660846006E00F40060009000BFDF
:1047B00000BF00BF0846C06C40F00100C864084656
:1047C000C06C00F00100009000BF00BF4FF44070CB
:1047D0000190022002900120039002200490012009
:1047E000059001A94FF09040FDF742FF06B010BDC3
:1047F000002C0140001002402DE9F04304460D4614
:1048000094F83E603F20075D94F84480452010F8FE
:1048100004906DB9012E02D1B8F1010F02D0012030
:10482000BDE8F083022084F83E0084F8440025E0CF
:10483000042D0CD1012F02D1B9F1010F01D00120BB
:10484000EEE702213F2001554520015516E0012EDB
:1048500007D1012F05D1B8F1010F02D1B9F1010F34
:1048600001D00120DCE7022084F83E0002213F2035
:104870000155022084F844004520015515B1042D4E
:104880000CD105E001220021206801F04FF910E071
:1048900001220421206801F049F90AE001220021E7
:1048A000206801F043F901220421206801F03EF95B
:1048B00000BF00BF2068006840F001002168086068
:1048C0000020ADE7704770B504462068C6682068D0
:1048D000056905F00200022819D106F0020002283D
:1048E00015D1401F21680861012020772068806968
:1048F00000F0030018B12046FFF7E4FF05E0204672
:1049000000F0ADF8204600F0ABF80020207705F06D
:104910000400042819D106F00400042815D1C0436E
:1049200021680861022020772068806900F44070C7
:1049300018B12046FFF7C6FF05E0204600F08FF8CB
:10494000204600F08DF80020207705F008000828A8
:1049500019D106F00800082815D1C0432168086164
:10496000042020772068C06900F0030018B12046B9
:10497000FFF7A8FF05E0204600F071F8204600F0A0
:104980006FF80020207705F01000102819D106F0EC
:104990001000102815D1C043216808610820207735
:1049A0002068C06900F4407018B12046FFF78AFF04
:1049B00005E0204600F053F8204600F051F80020B2
:1049C000207705F0010048B106F0010030B16FF02A
:1049D000010021680861204600F044F805F08000DD
:1049E000802804D005F40050B0F5005F0AD106F02D
:1049F0008000802806D16FF40250216808612046AB
:104A0000FFF76FFD05F48070B0F5807F0AD106F0E6
:104A10008000802806D16FF48070216808612046EC
:104A2000FFF75EFD05F04000402809D106F0400088
:104A3000402805D1C04321680861204600F062F893
:104A400005F02000202809D106F02000202805D1FB
:104A5000C043216808612046FFF744FD70BD7047E0
:104A60007047000010B504461D48844237D101202C
:104A70002AF0C2FE02F02CFE1A48006801282ED14E
:104A800019480068406A194908600FF075FF184915
:104A90000968022923D115490968164A1268881A3B
:104AA000002801DB014600E041420E2917DD0F48D6
:104AB0000068104908600D4801680F480268A0F5B9
:104AC000805040F822100D4801680B4800680C4ADD
:104AD00042F8201008480068401C0749086010BDD3
:104AE0003406002008030020E805002038000020DC
:104AF0000C0300203C0000200420001010000020C7
:104B000004000010704700BFFEE701688969C1F327
:104B1000400111B10021026891620168896901F0C8
:104B2000010129B90168896941F0010102689161B7
:104B3000704700002DE9F74F04460E460027206815
:104B4000D0F818800025DDF8089008F01000102833
:104B500045D12168C86134E0701C90B3FDF776FE42
:104B6000A0EB0900B04200D85EBB2068406800F4AA
:104B7000804A94F842B020688069C0F3C03070B1B8
:104B8000BAF5804F0BD0BBF1200F08D020684068E9
:104B900040F4804021684860FDF758FE814609E0F6
:104BA000FDF754FEA0EB0900192803D945F02005B4
:104BB000012705E020688069C0F340100028EFD08D
:104BC00000BF20688069C0F3401008B9002FC3D02F
:104BD00017B920202168C86145F004050127206825
:104BE000D0F8188008F48070B0F5807F06D145F0C9
:104BF00001054FF480702168C861012708F48060C6
:104C0000B0F5806F06D145F008054FF4806021684B
:104C1000C861012708F40070B0F5007F06D145F0A7
:104C200002054FF400702168C8610127AFB120462A
:104C3000FFF76BFF20684068094908402168486019
:104C4000606C28436064202084F84100002084F8D0
:104C5000420000BF84F8400000BF3846BDE8FE8F28
:104C600000E800FE2DE9F8430446894615461E4635
:104C7000DDE908781948F2B2002349460090204641
:104C800000F06CF842463946204600F0F4F810B1C6
:104C90000120BDE8F883012E03D1E8B221688862C3
:104CA0000EE0C5F307202168886242463946204657
:104CB00000F0E1F808B10120EBE7E8B22168886272
:104CC0003B46002240212046CDF8008000F062F8EB
:104CD00008B10120DDE70020DBE7000000200080B4
:104CE0002DE9F8430446894615461E46DDE9087855
:104CF0001948F2B2C30249460090204600F02EF84F
:104D000042463946204600F0B6F810B10120BDE811
:104D1000F883012E03D1E8B2216888620EE0C5F362
:104D200007202168886242463946204600F0A3F8F1
:104D300008B10120EBE7E8B2216888623B46002217
:104D400080212046CDF8008000F024F808B1012031
:104D5000DDE70020DBE7000000200080F0B5059CC7
:104D6000C1F309064FF47F0707EA02473E431E439B
:104D7000264326F00045066876684FF4806707EA08
:104D8000545767F0FC2747F4C047BE432E430768DB
:104D90007E60F0BD2DE9F04104460D4617461E46E3
:104DA000DDF818802BE0424631462046FFF7C2FE70
:104DB00010B10120BDE8F081701C00B3FDF746FD85
:104DC000A0EB0800B04200D8CEB920688069284026
:104DD000A84201D1012000E00020B8420FD1606C50
:104DE00040F020006064202084F84100002084F816
:104DF000420000BF84F8400000BF0120DAE72068CD
:104E000080692840A84201D1012000E00020B8427A
:104E1000C9D00020CEE770B504460D46164622E004
:104E2000324629462046FFF785FE08B1012070BDB5
:104E3000FDF70CFD801BA84200D8A5B92068806949
:104E4000C0F3401078B9606C40F02000606420200E
:104E500084F84100002084F8420000BF84F840003C
:104E600000BF0120E3E720688069C0F340100028FC
:104E7000D6D00020DBE770B504460D46164624E088
:104E8000324629462046FFF755FE08B1012070BD85
:104E9000681CD0B1FDF7DAFC801BA84200D8A5B988
:104EA00020688069C0F3400078B9606C40F0200051
:104EB0006064202084F84100002084F8420000BF94
:104EC00084F8400000BF0120E1E720688069C0F35A
:104ED00040000028D4D00020D9E72DE9F041074652
:104EE0000C4615461E462A2000F028F9384600F0E8
:104EF00016F9284600F013F92B2000F01FF904F1F1
:104F0000220188B200F00BF906F1220188B200F00C
:104F100006F92C2000F012F9BDE8F08100B587B049
:104F200000BF1048C06C40F002000E49C86408463B
:104F3000C06C00F00200019000BF00BF4FF42040A1
:104F400002900120039004900220059002A90648D7
:104F5000FDF78EFB012260210348FDF771FC07B0CD
:104F600000BD0000001002400004004810B5FFF72B
:104F7000D5FF002208214FF09040FDF761FC1E2074
:104F800005F075FD012208214FF09040FDF758FC17
:104F9000642005F06CFD642005F069FD112000F02F
:104FA000CDF8362000F0CAF8702000F0C1F83A20A1
:104FB00000F0C4F8052000F0BBF8B22000F0BEF805
:104FC0000C2000F0B5F80C2000F0B2F8002000F042
:104FD000AFF8332000F0ACF8332000F0A9F8B72088
:104FE00000F0ACF8352000F0A3F8BB2000F0A6F8E4
:104FF000352000F09DF8C02000F0A0F82C2000F033
:1050000097F8C22000F09AF8012000F091F8C32030
:1050100000F094F8132000F08BF8C42000F08EF814
:10502000202000F085F8C62000F088F80F2000F05E
:105030007FF8D02000F082F8A42000F079F8A120B9
:1050400000F076F8D62000F079F8A12000F070F892
:10505000E02000F073F8F02000F06AF8002000F083
:1050600067F8042000F064F8042000F061F80420E0
:1050700000F05EF8052000F05BF8292000F058F8F9
:10508000332000F055F83E2000F052F8382000F0B0
:105090004FF8122000F04CF8122000F049F82820B8
:1050A00000F046F8302000F043F8E12000F046F828
:1050B000F02000F03DF8072000F03AF80A2000F058
:1050C00037F80D2000F034F80B2000F031F80720FD
:1050D00000F02EF8282000F02BF8332000F028F8FC
:1050E0003E2000F025F8362000F022F8142000F0D1
:1050F0001FF8142000F01CF8292000F019F83220C5
:1051000000F016F8212000F019F8112000F016F830
:10511000782005F0ACFC292000F010F810BD10B587
:105120000446201200F01CF8E0B200F019F810BD9F
:1051300010B50446204600F013F810BD10B5044623
:10514000002204214FF09040FDF77AFB204600F04A
:1051500007F8012204214FF09040FDF771FB10BDCC
:1051600070B50446002201214FF09040FDF768FB26
:1051700000251DE000224FF400511248FDF760FBAE
:1051800004F0800028B10122D1030E48FDF758FB3E
:1051900005E000224FF400410A48FDF751FB0122CF
:1051A00051030848FDF74CFB6006040E681CC5B2AD
:1051B000082DDFDB012211464FF09040FDF740FB48
:1051C00070BD0000000400488168024A1140491C7B
:1051D00081607047C0FFFF7F024602F1600000EB74
:1051E0008103186800F0F840704701468868C0F3F2
:1051F000C00070470146886800F001007047014612
:105200008868C0F30070704701468868C0F380006A
:10521000704700008168024A1140091D8160704793
:10522000C0FFFF7F70B500F11404C1F3406504EBCB
:1052300085031C68C1F304560725B540AC43C1F390
:10524000045502FA05F52C431C6070BD826822F0FB
:10525000E0720A438260704710B500F1600404EB0D
:1052600081031C6824F0004414431C6010BD426993
:1052700022F000420A4342617047000000B587B047
:10528000182101A8FBF725FA1A481B4908600020DD
:105290004860002118488160C160016104214161BA
:1052A0000021017641760121C161002180F82010A2
:1052B0008162C16280F83010416380F83810FDF7D8
:1052C0002BF808B1FCF7B1FD0C48019006200290C4
:1052D000032003907F200490042005900020069076
:1052E00001A90548FCF7A4FD08B1FCF79EFD07B035
:1052F00000BD000000000450640400200004002AE7
:1053000000B587B0142102A8FBF7E3F900BF2E48CF
:10531000C06C40F080002C49C8640846C06C00F0A6
:105320008000019000BF00BF00BF0846C06C40F085
:105330000100C8640846C06C00F00100019000BF85
:1053400000BF00BF0846C06C40F00200C8640846B9
:10535000C06C00F00200019000BF00BF01220D21CF
:105360004FF09040FDF76CFA012211031748FDF74A
:1053700067FA00224FF4E0711448FDF761FA0D203E
:1053800002900120039000200490059002A94FF0A4
:105390009040FDF76DF940F2232002900020039029
:1053A000049002A90948FDF763F94FF48E5002906A
:1053B0000120039000200490059002A90348FDF706
:1053C00057F907B000BD000000100240000400487B
:1053D00010B5124812490860124848600021104870
:1053E00081600121C1600021016141618161C16170
:1053F0000162FDF79BFA08B1FCF717FD0021084890
:10540000FDF72AFA08B1FCF710FD00210448FDF76A
:1054100058FA08B1FCF709FD10BD000000840040F7
:10542000CC040020EC9C901010B511481149086084
:105430004FF48270486000210E4881604FF4E061B3
:10544000C160002101610121416149028161302176
:10545000C16100210162416281620721C1620021B4
:1054600001634163FEF7D2FC08B1FCF7DEFC10BD1E
:10547000003001402005002010B511481149086096
:105480004FF48270486000210E4881604FF44071F3
:10549000C160022101610121416149028161202134
:1054A000C16100210162416281620721C162002164
:1054B00001634163FEF7AAFC08B1FCF7B6FC10BD1E
:1054C000003800408405002000B58DB0242104A8D8
:1054D000FBF7FFF80020019002900390184819494B
:1054E0000860002048600021164881604FF6FF7177
:1054F000C1600021016141618161032004900020AD
:105500000590012006900020079008900990012046
:105510000A9000200B900C9004A90A48FFF7CAF8E3
:1055200008B1FCF782FC002001900290039001A9D1
:105530000448FEF7D9FF08B1FCF777FC0DB000BDB9
:10554000002C0140E80500200EB5002000900190DD
:1055500002900E480E4908604F20486000210C4818
:10556000816040F2E731C16000218161FFF706F8F8
:1055700008B1FCF75AFC00200090029069460448EC
:10558000FEF7B2FF08B1FCF750FC0EBD0010004062
:105590003406002000BFFEE700BFFEE770470000B2
:1055A0002DE9F04104460F4600255B48C06800F035
:1055B000030090B15848C06800F003002168884299
:1055C00009D1206838B15448C068C0F30210401CAB
:1055D0006168884233D0012531E02068012804D079
:1055E000022809D003281AD10DE04B48006800F0CA
:1055F000020000B9012514E04748006800F480600B
:1056000000B901250DE04448006800F4003028B9D5
:105610004148006800F4802000B9012501E001251F
:1056200000BF00BF5DB9D4E90010401E41EA001080
:105630003949C96821F0730108433749C860002D12
:1056400067D13548006820F0806033490860FDF775
:10565000FDF8064606E0FDF7F9F8801B022801D99F
:10566000032505E02C48006800F000600028F2D116
:1056700000BFC5BB67B9A0680002217B40EAC160DA
:1056800025490969254A114008432349086120E05A
:10569000012F0FD1A0680002218A0122C2EB510123
:1056A00040EA41501C4909691D4A114008431A4902
:1056B00008610EE0A0680002217D0122C2EB5101C9
:1056C00040EA416014490969164A114008431249E9
:1056D00008611148006840F080600F490860FDF7DC
:1056E000B5F8064607E014E0FDF7B0F8801B022885
:1056F00001D9032505E00848006800F00060002893
:10570000F2D000BF2DB904480069A16908430249DD
:1057100008612846BDE8F08100100240FF80FF07C5
:10572000FF809FFFFF80FFF9F8B50446002623485D
:10573000806D00F0805018B1FDF760FC054616E062
:1057400000BF1E48806D40F080501C4988650846A7
:10575000806D00F08050009000BF00BFFDF74EFC50
:1057600005461648806D20F0805014498865B5F5CF
:10577000007F07D1802C10D9A02C01D902260CE083
:1057800001260AE0802C01D9032606E0802C01D1F5
:10579000022602E0702C00D101260948006820F0A2
:1057A00007003043064908600846006800F007001B
:1057B000B04201D00120F8BD0020FCE700100240FB
:1057C00000200240F8B504460E4615463346002236
:1057D0004FF4C0512046009500F026F828B1206E05
:1057E00040F0200020660320F8BD334600228021CF
:1057F0002046009500F094F828B1206E40F020007B
:1058000020660320F0E7334600224FF4C0612046B3
:10581000009500F009F828B1206E40F020002066C5
:105820000320E1E70020DFE72DE9FC5F04460D4699
:1058300016461F46DDF8309000200090FDF706F870
:10584000A0EB0900A7EB0008FDF700F882462068EE
:1058500000F10C0B31480068C0EBC00000EB800089
:10586000000D00FB08F0019050E0B5F5C06F05D1C8
:1058700026B99BF8000000909DF80000781C0028D5
:1058800044D0FCF7E3FFA0EB0A00404502D2B8F198
:10589000000F34D12068406820F0E00021684860A3
:1058A0006068B0F5827F0DD1A068B0F5004F03D0DD
:1058B000A068B0F5806F05D12068006820F0400036
:1058C00021680860A06AB0F5005F0DD100BF2068B4
:1058D000006820F40050216808602068006840F4E7
:1058E00000502168086000BF012084F85D0000BFFF
:1058F000002084F85C0000BF0320BDE8FC9F0198F5
:1059000008B94FF000080198401E01902068806897
:105910002840B042A9D10020EFE700000C00002091
:105920002DE9F84F04460D4690461E46DDF82890B6
:10593000FCF78CFFA0EB0900371AFCF787FF8246C3
:105940002C480068C0F3CB307843009045E0701CD1
:10595000002842D0FCF77AFFA0EB0A00B84200D240
:10596000A7BB2068406820F0E000216848606068BC
:10597000B0F5827F0DD1A068B0F5004F03D0A068CC
:10598000B0F5806F05D12068006820F040002168E4
:105990000860A06AB0F5005F0DD100BF2068006804
:1059A00020F40050216808602068006840F400502E
:1059B0002168086000BF012084F85D0000BF00205E
:1059C00084F85C0000BF0320BDE8F88FFFE7009873
:1059D00000B900270098401E009020688068284089
:1059E000A84201D1012000E000204045AFD10020B5
:1059F000EAE700000C000020704710B5FDF7EAF957
:105A000010BD00B597B0442106A8FAF762FE142134
:105A100001A8FAF75EFE4FF40070FDF7A9FA08B18D
:105A2000FCF703FA01200690000407900220109072
:105A30000321119101211291142113910721149135
:105A400002211591169106A8FDF738FE08B1FCF762
:105A5000ECF90F20019003200290002003900490A5
:105A60000590042101A8FDF7D9FC08B1FCF7DDF988
:105A700017B000BD0348006840F470000149086099
:105A80007047000088ED00E010B50248FEF71BFFEC
:105A900010BD00003406002010B502681F4B98426C
:105AA00005D0B0F1804F02D01D4B984203D122F0B7
:105AB00070024B681A43194B98420BD0B0F1804FDB
:105AC00008D0174B984205D0164B984202D0164B7F
:105AD000984203D122F44072CB681A4322F080032B
:105AE0004C6943EA040202608B68C3620B688362FC
:105AF0000A4B984205D00B4B984202D00A4B984271
:105B000001D10B69036301234361036903F00103BE
:105B10001BB1036923F00103036110BD002C014098
:105B200000040040004001400044014030B501F055
:105B30001F05012404FA05F3046A9C430462046A05
:105B400001F01F0502FA05F52C43046230BD00BFC9
:105B5000FEE703B401984100009850EAC12018BF45
:105B600004204A0D18BF40F0010040F2FF72B2EB72
:105B7000515F08BF40F00200012808BF052002B0B5
:105B80007047000002480068C0F302207047000020
:105B90000CED00E010B5002804DB0A07130E054ADF
:105BA000135406E00A07140E034A00F00F031B1FEC
:105BB000D45410BD00E400E018ED00E02DED020B20
:105BC000019820F0004001909DED000B02B070475D
:105BD00030380A2801D201207047002070470000A9
:105BE00010B54421074801F02AF800221E2106487A
:105BF00029F06AFE0549086002F0A6F80020044971
:105C0000087010BD04350020297E0008180200200D
:105C1000140200202DE9F04F87B007460C461546C8
:105C20002946204600F066F920B94FF0FF3007B052
:105C3000BDE8F08F00222946204600F0FDF808B1AB
:105C40000020F4E70026204614F080FB401E00B23E
:105C50000490204614F0EBFA401E00B203906888CE
:105C60006188401A0FFA80FABAF1000F16DD208819
:105C7000ADF814006088ADF81600A088ADF81800E3
:105C80006088504400B2ADF81A003046711C4EB224
:105C900007EBC0000599016006994160E8886188BA
:105CA000411A0398401A0FFA80FBBBF1000F1CDD6C
:105CB000B5F90600B4F90610884216DA2088ADF866
:105CC0001400E888ADF81600A088ADF81800E88840
:105CD000584400B2ADF81A003046711C4EB207EBC2
:105CE000C0000599016006994160B5F90200B4F958
:105CF0000210884202DDB5F9020001E0B4F90200A9
:105D00008046B5F90600B4F90610884202DAB5F902
:105D1000060001E0B4F9060002900298A0EB08002A
:105D20000FFA80F928882188401A00B20190019862
:105D300000281BDDB9F1000F18DD2088ADF8140034
:105D4000ADF8168021880198084400B2ADF818001B
:105D500008EB090000B2ADF81A003046711C4EB2D3
:105D600007EBC0000599016006994160A888218869
:105D7000411A0498401A00B200900098002818DDDB
:105D8000A888ADF81400ADF81680A98800980844DA
:105D900000B2ADF8180008EB090000B2ADF81A0027
:105DA0003046711C4EB207EBC000059901600699A0
:105DB000416030463BE730B50346B1F90040B2F9E7
:105DC0000050AC4202DDB1F9004001E0B2F9004000
:105DD0001C80B1F90240B2F90250AC4202DDB1F9C7
:105DE000024001E0B2F902405C80B1F90440B2F92E
:105DF0000450AC4202DAB1F9044001E0B2F90440C7
:105E00009C80B1F90640B2F90650AC4202DAB1F911
:105E1000064001E0B2F90640DC800120B3F9004001
:105E2000B3F90450AC4205DCB3F90240B3F90650B3
:105E3000AC4200DD002030BDF8B504460D461646E4
:105E40000027B4F90000B5F90010884212DBB4F95C
:105E50000200B5F9021088420CDBB4F90400B5F970
:105E60000410884206DCB4F90600B5F90610884231
:105E700000DC01270FB90020F8BD0EB90120FBE7B7
:105E80002088ADF800006088ADF80200324669460F
:105E9000284600F0A7F808B90020EDE7A088ADF883
:105EA00000006088ADF8020032466946284600F0DE
:105EB00099F808B90020DFE72088ADF80000E088F5
:105EC000ADF8020032466946284600F08BF808B962
:105ED0000020D1E7A088ADF80000E088ADF802000E
:105EE00032466946284600F07DF808B90020C3E72D
:105EF0000120C1E70246B2F90000B1F9043098422E
:105F000013DCB2F90400B1F9003098420DDBB2F9AC
:105F10000200B1F90630984207DCB2F90600B1F987
:105F20000230984201DB012070470020FCE7F8B501
:105F300004460D461646B4F90400B5F9001088422F
:105F400011DBB4F90600B5F9021088420BDBB4F995
:105F50000000B5F90410884205DCB4F90200B5F977
:105F60000610884201DD0120F8BD0EB90020FBE7D4
:105F70002088ADF800006088ADF80200324669461E
:105F8000284600F02FF808B10020EDE7A088ADF812
:105F900000006088ADF8020032466946284600F0ED
:105FA00021F808B10020DFE72088ADF80000E08884
:105FB000ADF8020032466946284600F013F808B1F1
:105FC0000020D1E7A088ADF80000E088ADF802001D
:105FD00032466946284600F005F808B10020C3E7BC
:105FE0000120C1E72DE9FC5F05460E4614464FF03F
:105FF000000AB6F90000B5F90010884213DBB6F9C3
:106000000000B5F9041088420DDCB6F90200B5F9BC
:106010000210884207DBB6F90200B5F90610884283
:1060200001DC4FF0010ABAF1000F02D10020BDE8F7
:10603000FC9F002C01DC0120F9E7284614F086F9CA
:10604000834600EBDB704710284614F0F0F88346D7
:1060500000EBDB704FEA6008474501DA384600E0A4
:10606000404681464C4500DD4C462888ADF800008E
:106070002888204400B2ADF804006888ADF802001A
:106080006888204400B2ADF8060000223146684618
:10609000FFF7A8FF80B1BDF80400204400B2ADF8BE
:1060A0000400BDF80600204400B2ADF806003146F9
:1060B000684626F023F8BAE7E888001B00B2ADF87E
:1060C0000200E888ADF80600002231466846FFF776
:1060D00089FF80B1BDF80400204400B2ADF804008F
:1060E000BDF80200001B00B2ADF802003146684660
:1060F00026F004F89BE7A888001B00B2ADF800006A
:10610000A888ADF80400002231466846FFF76AFF10
:1061100080B1BDF80000001B00B2ADF80000BDF872
:106120000200001B00B2ADF802003146684625F0BF
:10613000E5FF7CE76888ADF802006888204400B27B
:10614000ADF80600002231466846FFF74BFF80B1EC
:10615000BDF80000001B00B2ADF80000BDF806005D
:10616000204400B2ADF806003146684625F0C6FF6F
:106170005DE701205BE710B5B1F90030B2F90040EE
:10618000A34202DAB1F9003001E0B2F90030038035
:10619000B1F90230B2F90240A34202DAB1F9023099
:1061A00001E0B2F902304380B1F90430B2F90440A1
:1061B000A34202DDB1F9043001E0B2F9043083807A
:1061C000B1F90630B2F90640A34202DDB1F906305A
:1061D00001E0B2F90630C38010BD0000F8B50546F5
:1061E00029F0FAFA07460020009035B14C49E868DA
:1061F0000860284629F080FC03E017F02BFA484994
:10620000086047490968086925F00CFE44480068A1
:10621000406920B142490968486925F003FE4049B8
:106220000968C86925F0FEFD3D490968086A25F03E
:10623000F9FD3B480068006938B900203849096811
:10624000A1F8500100BF00BFF8BD26F021F82CF0E6
:106250002DF92BF065FD32480068B0F85001002898
:1062600056D02F4800680068007C00F0010040B361
:106270002B4800680068C068406810B3002419E02B
:106280002748006800F59870005D00B110E02448D0
:10629000006800F5AC7000F034FD06462048006848
:1062A000303000EBC400016831604068706000BFAE
:1062B000601C84B21A480068B0F85001A042DFDCCC
:1062C00000BF4FF480711648006830301FF05CFC4E
:1062D00020211348006800F598701FF055FC00203D
:1062E0000F490968A1F85001384629F067FA009073
:1062F0000B4800680068406A50B10949096808689D
:106300000749096809684B6A06490A68009998476D
:106310001FF0B2F900F03EF800F006F800BF93E776
:10632000D4000020D000002010B5002416E0C4EBFB
:10633000C4000C4951F8200030B1C4EBC401094A33
:1063400052F821001FF04AFAC4EBC401054A02EBDF
:1063500081001C211FF018FC601CC4B2042CE6DB79
:1063600010BD0000E03500200146094A10680BE02E
:1063700042688A4202D002688A4204D1027E22F038
:106380000102521C027640690028F1D170470000DA
:10639000A80000207047000010B50421014800F05B
:1063A0004EFC10BDF834002010B52021014800F04B
:1063B00046FC10BD103500202DE9FF4704460D4670
:1063C00016461F46DDE90C896FB9B8F5807F0AD102
:1063D000002020806080681E00B2A080701E00B285
:1063E000E080BDE8FF8700200090019002900390BC
:1063F000ADF80450ADF80A60ADF80C50ADF80E6081
:106400004B4642463946684625F0AEFD4B4642466D
:10641000394601A825F0A8FD4B464246394602A858
:1064200025F0A2FD4B464246394603A825F09CFDC7
:10643000BDF90000BDF90410884202DABDF9000080
:1064400001E0BDF90400BDF90810BDF90C2091422E
:1064500002DABDF9081001E0BDF90C1088420BDA30
:10646000BDF90000BDF90410884202DABDF9000050
:106470000DE0BDF904000AE0BDF90800BDF90C10FB
:10648000884202DABDF9080001E0BDF90C00801E67
:1064900000B22080BDF90000BDF90410884202DD81
:1064A000BDF9000001E0BDF90400BDF90810BDF917
:1064B0000C20914202DDBDF9081001E0BDF90C107D
:1064C00088420BDDBDF90000BDF90410884202DDF1
:1064D000BDF900000DE0BDF904000AE0BDF90800B7
:1064E000BDF90C10884202DDBDF9080001E0BDF9DC
:1064F0000C00801C00B2A080BDF90210BDF906009E
:10650000814202DABDF9020001E0BDF90600BDF9E1
:106510000A20BDF90E108A4202DABDF90A1001E024
:10652000BDF90E1088420BDABDF90210BDF9060064
:10653000814202DABDF902000DE0BDF906000AE071
:10654000BDF90A10BDF90E00814202DABDF90A0058
:1065500001E0BDF90E00801E00B26080BDF902109E
:10656000BDF90600814202DDBDF9020001E0BDF97E
:106570000600BDF90A20BDF90E108A4202DDBDF900
:106580000A1001E0BDF90E1088420BDDBDF90210C2
:10659000BDF90600814202DDBDF902000DE0BDF942
:1065A00006000AE0BDF90A10BDF90E00814202DDC5
:1065B000BDF90A0001E0BDF90E00801C00B2E080C8
:1065C00000BF0EE72DE9F743054616460024134C9D
:1065D00029F002F98046334629462046019A1CF0EC
:1065E00029FC07465FB900BF00BF2C2120461FF0E1
:1065F000CBFA4FF00040A0620020BDE8FE830020EF
:10660000A062E06918B9404629F0D8F8E061E06975
:1066100008B90120E0612046EFE700003435002092
:1066200010B51421114800F00AFB1CF0B5FB04461C
:1066300000BF1CB900BF00BF00BFFEE700BF14B918
:1066400000BF00BF10BD0A4920461CF08DFC09495F
:1066500020461CF08BFC084920461CF089FC0749A9
:1066600020461CF07FFC00BFECE700001C3500203A
:10667000492502081D2A0208A52C02081125020836
:1066800070B504460D46102128461FF07DFA20689B
:106690000078012804D1A08A2880E08A68800CE074
:1066A00020680078022802D1E068686005E0206870
:1066B0000078042801D10A2068602068406820B171
:1066C000206829464268904701E000BF00BF70BDC6
:1066D0002DE9FE4F0446A08A18B9E08A08B9BDE842
:1066E000FE8FE66A96B920460DF05AF8064606B9BE
:1066F000F5E7204611F030FA0022092130461AF061
:106700003DFF6078C0F3400000B1E8E700274FF498
:106710008078B14616E00021484622F091FE3844C8
:1067200007B20021484622F0C7FE8246C0170AEB96
:106730001060001200FB08F00FFA80F8484621F0C4
:1067400015FA8146B9F1000FE5D117B9B8F5807F88
:1067500011D0784207B24FF4803090FBF8F00FFA76
:1067600080F8002000906B464246394604F1140040
:1067700025F0FAFB00BF00200290019094F8400041
:1067800000F00F00032812D1304621F00DFB8246A5
:10679000304621F091FA834603200090B4F914109A
:1067A00053465A4630460CF02BFA029012E030461F
:1067B00021F07CFB8246304621F0F0F983460C2024
:1067C0000090B4F916105B46524630460CF018FAA9
:1067D000019000BF304621F041FA054605F0010066
:1067E00028B9BDF90800002801DD0020029005F05D
:1067F000020028B9BDF90800002801DA0020029043
:1068000005F0040028B9BDF90400002801DD0020CE
:10681000019005F0080028B9BDF90400002801DA4C
:106820000020019001AA02A920462CF01FFBBDF90F
:106830000420BDF90810304600F0FCFA6078C0F37F
:10684000400000B14BE7208BBDF80810084401B2AE
:106850002183608BBDF80410084401B2618300BF3E
:106860003DE72DE9F84F0446D4F82CB0BBF1000FFA
:1068700001D1BDE8F88F94F8400000F00F0000B996
:10688000F7E71CF02BFF06463068477E402158464C
:1068900022F0CCFF10B90021E183A183584621F0FA
:1068A000F1FA8046584621F0F7FA054694F8400080
:1068B00000F00F000C2843D10021A1831DBBB4F9C7
:1068C0001E00C7F164014843642190FBF1F001B25E
:1068D000E183584621F062F98146584621F0E6FAF4
:1068E00082460C200090B4F91E104B465246584682
:1068F0000CF086F9E083B4F91E20002319465846AF
:1069000024F03EFB69E020462CF007FB00900021BC
:10691000E1836A4620462CF0A9FABDF9003041F621
:10692000FF72514258460DF02DF98146BDF8000026
:10693000484402B201230021584624F021FB4CE0D8
:1069400094F8400000F00F00032846D10021E183B5
:10695000B8F1000F23D1B4F91C00C7F1640148431A
:10696000642190FBF1F001B2A183584621F0A4F913
:106970008146584621F018FA824603200090B4F967
:106980001C1053464A4658460CF03AF9A083B4F915
:106990001C1000231A46584624F0F2FA1DE0204647
:1069A0002CF0A0FA00900021A18300226946204625
:1069B0002CF05CFABDF9003041F6FF7251425846A6
:1069C0000DF046F88146BDF80000484401B20123AD
:1069D0000022584624F0D4FA00BFA08B002860D1D2
:1069E000E08B00285DD11DBB584621F05FFA81463F
:1069F000584621F0D3F88246B9F1000F02DCBAF113
:106A0000000F14DDB9F1000F06DA01234A46002118
:106A1000584624F0B5FA0AE0BAF1000F07DA01236C
:106A2000CAF1000002B20021584624F0A9FA00BFC2
:106A3000B8F1000F23D1584621F03EF9814658465F
:106A400021F0B2F98246B9F1000F02DCBAF1000F71
:106A500014DDB9F1000F06DA012300224946584639
:106A600024F08EFA0AE0BAF1000F07DA01230022BF
:106A7000CAF1000001B2584624F082FA00BF324643
:106A80000A2158461AF07AFD6078C0F3400000B140
:106A9000EFE694F8400020F00F0184F84010002148
:106AA000E16200BFE5E62DE9FF4104460F4614B957
:106AB00016F0D0FD04460CB9BDE8FF81204616F063
:106AC00062FE00B9F8E794F82800C0F3800010B126
:106AD00000BF00BFF0E71FB90020A4F85001EBE7AA
:106AE0000020ADF80800ADF80A00204616F0CAFDF7
:106AF000401E00B2ADF80C00204616F029FE401EE4
:106B000000B2ADF80E0002AA39466846FFF753F905
:106B1000064606B9D0E72068007CC0F3400060B1AB
:106B200002982063039860630120A4F85001606814
:106B300010B1606828F0ECFFBEE72068806918B1EA
:106B4000206869468269904700250BE004F1300017
:106B500000EBC50100226846FFF76EF900B1ABE714
:106B6000681C85B2B4F85001A842EFDCB4F85001BB
:106B7000202809DAB4F8502104F1300101EBC200F9
:106B8000694613F0BBFA0BE00020A4F85001B4F8FA
:106B9000502104F1300101EBC20002A913F0AEFA5A
:106BA000B4F85001401CA4F85001606810B160684E
:106BB00028F0AEFF00BF7FE770B50546284600F01D
:106BC00013F8044600260CE02146284600F024F87D
:106BD00006462146284600F0C0F820461EF0FEFD7D
:106BE0003446002CF0D170BD014609B90020704731
:106BF0004868FCE770B5064600243046FFF7F4FF0E
:106C0000054605E0641C2946304600F005F80546B7
:106C1000002DF7D1204670BD02460B461068001DBE
:106C200003441868704702460B461068034418680E
:106C30007047014609B9002070478868FCE70022C8
:106C400042608260CA1C22F003010160704770B587
:106C50000446216801F108001EF0E2FC0546A5B1DA
:106C60000022294620462AF01BFB2946204662685E
:106C70002AF008FB606820B12A46204661682AF0A5
:106C80000FFB6560A06800B9A560284670BD2DE9BE
:106C9000F04106460D4606B115B90020BDE8F08169
:106CA0003046FFF7A1FFA84206D13046FFF7CFFFDD
:106CB000044624BB0020F1E7316801F108001EF012
:106CC000AFFC04460CB90020E8E729463046FFF740
:106CD000AAFF07462246394630462AF0D3FA3A46FA
:106CE000214630462AF0DCFA2246294630462AF070
:106CF000D7FA2A46214630462AF0C4FA00BF204679
:106D0000CCE770B50446216801F108001EF088FC4C
:106D10000546A5B10022294620462AF0B3FA2946A5
:106D20002046A2682AF0BCFAA06820B12A46204674
:106D3000A1682AF0A7FAA560606800B965602846D6
:106D400070BD014609B901207047486818B98868C4
:106D500008B90120F8E70020F6E72DE9F0410446E4
:106D60000D460CB9BDE8F0812046FFF73DFFA84273
:106D70000FD129462046FFF74FFF6060606810B9C9
:106D80000020A0602FE00022204661682AF088FAE7
:106D900029E02046FFF74DFFA8420FD129462046A3
:106DA000FFF741FFA060A06810B9002060601AE002
:106DB00000222046A1682AF065FA14E02946204600
:106DC000FFF731FF064629462046FFF725FF074615
:106DD0003A46314620462AF055FA32463946204690
:106DE0002AF05EFA00BF00BFBCE710B50446206879
:106DF000806818B120682146826890472068006842
:106E000028B12068006820602046FFF7EEFF10BD23
:106E10000146886818B18868B0F9160070470020EC
:106E2000FCE70146886818B18868807E8009704751
:106E30000020FCE72DE9F04104460D4616461DB939
:106E400016B90120BDE8F08120461FF0B1FDA06811
:106E5000008A284400B2A1680882A068408A3044B1
:106E600001B2A0684182012332462946204623F020
:106E700077F900220B2120461AF080FB0746012FEC
:106E800001D03846DEE7204623F093F80120D9E709
:106E9000F7B582B004460E4614B9049805B0F0BDAB
:106EA00000BF62223146204622F050F90190019D38
:106EB00000BFBDB12868A8B100BF6322314620469B
:106EC00022F044F901900198C0B207464FB13A460A
:106ED0002B682846049998470190BDF80400ADF846
:106EE000100000BF0498D9E72DE9F04F95B0044693
:106EF0008B4691469A461E9D608C20F00400001D32
:106F00006084A4F820902A895946204622F01EF970
:106F10001490A4F820A02A895946204622F016F998
:106F20001390608C20F004006084DDE91310884227
:106F30000CD1DDE91310884208D1BDF85000BDF82E
:106F40004C10884202D115B0BDE8F08FA4F8209013
:106F50002A895946204622F0F9F81490A4F820A076
:106F6000594620460EF01EFE12902989129A10688A
:106F7000149A27F0FFF828890B2833D147F6FF71C0
:106F80001498884202D0139888422BD1204622F0D0
:106F9000F0FB009000EBD0704710204620F096FDEB
:106FA000009000EBD0704FEA600847F6FF7114982C
:106FB000884208D1781C08F10101884200DA01E01A
:106FC00008F10100149047F6FF711398884208D128
:106FD000781C08F10101884200DA01E008F10100A3
:106FE000139000BF2348FFF732FE064600BF1EB9CC
:106FF00000BF00BF00BFFEE700BF06B9A3E71498BB
:10700000F0601398306134602889B080C6F808B009
:1070100001A812F027FA314601A812F0E2FA164947
:1070200001A812F0A7FA1548039000BF144901A85F
:1070300012F0AEFAFF22002101A812F0C0FA29884E
:1070400001A812F0AEFA698801A812F08CFAE8687B
:10705000089000BF01A8002190F8422061F30002CF
:1070600080F8422000BF2869079001A812F0D0FAEA
:1070700000BF68E7283500209DAC030845AF030832
:1070800075AE030810B514210148FFF7D8FD10BDF7
:10709000283500202DE9FE4F04460F4690464FF05C
:1070A000000900254CE1E06800EBC5004068C0F332
:1070B000406000B143E1E16801EBC501496821F09E
:1070C0007F4024F075FE064626EA070008B9012035
:1070D00000E00020029026EA080008B9012000E044
:1070E00000200190DDE90101814270D0E06850F894
:1070F00035A04FF0000B6A461021504626F012FCD6
:1071000010B14FF0010B98E06A461121504626F06D
:1071100009FC10B14FF0010B8FE06A461221504676
:1071200026F000FC10B14FF0010B86E06A461321F7
:10713000504626F0F7FB10B14FF0010B7DE06A4698
:107140001521504626F0EEFB10B14FF0010B74E014
:107150006A461421504626F0E5FB10B14FF0010BB2
:107160006BE06A460A21504626F0DCFB10B14FF076
:10717000010B62E06A466B21504626F0D3FB10B14A
:107180004FF0010B59E06A466C21504626F0CAFBCD
:1071900010B14FF0010B50E06A460121504626F035
:1071A000C1FB10B14FF0010B47E06A460421504685
:1071B00026F0B8FB10B14FF0010B3EE06A46022109
:1071C000504626F0AFFB18B14FF0010B35E0B5E0AB
:1071D0006A460321504626F0A5FB10B14FF0010B83
:1071E0002BE06A460521504626F09CFB10B14FF07B
:1071F000010B22E06A460621504626F093FB10B1AF
:107200004FF0010B19E06A463221504626F08AFB06
:1072100010B14FF0010B10E06A466E21504626F087
:1072200081FB10B14FF0010B07E06A466D2150461B
:1072300026F078FB08B14FF0010BBBF1000F02D034
:107240000320BDE8FE8F6A466921504626F06AFB9E
:1072500010B14FF0020970E06A466A21504626F0EC
:1072600061FB10B14FF0020967E06A466E2150469B
:1072700026F058FB10B14FF002095EE06A466D211E
:10728000504626F04FFB10B14FF0020955E06A4618
:107290003721504626F046FB10B14FF002094CE072
:1072A0006A463821504626F03DFB10B14FF00209E6
:1072B00043E06A463521504626F034FB10B14FF0CA
:1072C00002093AE06A464021504626F02BFB10B1F5
:1072D0004FF0020931E06A464521504626F022FB74
:1072E00010B14FF0020928E06A464121504626F0CD
:1072F00019FB10B14FF002091FE06A4642215046C7
:1073000026F010FB10B14FF0020916E06A46432147
:10731000504626F007FB10B14FF002090DE06A4617
:107320004921504626F0FEFA10B14FF0020904E060
:10733000B9F1000F01D14FF0010900BF00BF6D1C72
:10734000608CC0F3C500A8423FF6ADAE484678E772
:107350000148006870470000D400002070470146D3
:10736000C1F30412072A00DD0722D0B270470000E3
:1073700001464FF6FF70814201D11F20704709B9C5
:107380000020FBE7712902DA0948405CF6E7A1F129
:10739000710081B20748006838B10748006881422F
:1073A00003D204480068405CE8E70020E6E70000FC
:1073B0005C0104083C0200205002002010B5182196
:1073C0000348FFF73CFC012028F0BAFA10BD00008A
:1073D000D43400202DE9F04105460F4616460DB97C
:1073E000BDE8F0812846F9F723F98046394628465A
:1073F0000A4A126890470746E8193146074A126858
:10740000904706463C4603E0A019285C2855641CBA
:10741000A8EB0600A042F7D200BFE1E780020020FF
:107420002DE9F04106460C4617461D4629463046D2
:10743000084A126890472060206830B1296888198E
:107440000021044A1268904700E000203860BDE83F
:10745000F0810000780200202DE9F04F87B004464B
:107460000F4692469846DDE910560DB1002028805F
:107470001CB9002007B0BDE8F08F207808B90020C3
:10748000F8E70FB90020F5E74FF0000906F0020019
:1074900010B906F0040098B1002000E0401C215C07
:1074A0000A2905D0215C0D2902D0215C0029F5D1E3
:1074B000215C01B1401C15B14FF0FF312980D9E7A3
:1074C00006F0020008B141F6FF7800200690059012
:1074D00038E000200490059808B9012000E0002061
:1074E00006A904AACDE90062CDE902100599601849
:1074F00043465246394628F08BFC83460498A8EB55
:1075000000000FFA80F8049848440FFA80F9BBF1A4
:10751000000F00D11CE005985844059020780A28F7
:1075200002D020780D2800D112E00598205C0A28AE
:1075300003D00598205C0D2803D10598401C0590C8
:1075400006E000BF0598205C10B1B8F1000FC0DC68
:1075500000BF059870B905A92046094A12689047EE
:10756000834635B10022594638461AF08BF90FFA96
:1075700080F900BF0DB1A5F8009005987AE70000EA
:10758000780200202DE9F04706468846174606B1E6
:107590000FB9BDE8F0873046F9F74AF8814638461A
:1075A000F9F746F8044604B9F3E704EB090A414643
:1075B00030460B4A126890478046554603E0281B28
:1075C000305C70556D1E08EB0400A842F7D906EB3D
:1075D0000800224639461EF091FA00BFD9E70000A4
:1075E00080020020024600200FA31B788B4211D19D
:1075F00013781BB90123137001200BE01378012BC2
:1076000002D10023137005E01378022B02D100236E
:10761000137001201378012B04D1202901D10223FA
:1076200013700120704700002300000073B582B082
:10763000064603980190324600210846019BF8F760
:107640009DFE0546002001900024681C1DF0E8FF07
:10765000044600BF1CB900BF00BF00BFFEE700BF6B
:1076600014B9002004B070BD002060553246691C7A
:107670002046039BF8F782FE2046F3E72DE9F0470A
:1076800081460E4614461F46DDF820A035461BE015
:10769000600800FB075529464846D047B0F100086E
:1076A00009DD04F0010080F00100C0EB5404E8198A
:1076B0000546064608E0B8F1000F02DA64083546D0
:1076C00002E02846BDE8F087002CE1D10020F9E770
:1076D00010B52DED068B2948FAF71AFE28490880C7
:1076E0000846008834F08EFA41EC1A0B9FED250B0A
:1076F00053EC102B34F0E8F841EC190B9FED230B01
:1077000053EC102B34F0CEFA41EC180B33F0F6FFAB
:10771000204908601948FAF74DFF1E4890ED000A0D
:10772000BCEEC00A10EE100A1B491C4A126841F850
:10773000220008461949096850F8210018490968CB
:1077400008441749086015480068401C1349086040
:1077500008460068B0F57A7F0CDB114800684FF4EA
:107760007A71B0FBF1F00F49086000200C49086005
:107770000A490860BDEC068B10BD000064040020BF
:1077800054000020000000000000B0400000000095
:1077900000C8A94058000020082000105C0000200C
:1077A0004C000020500000202DE9F04104460E4618
:1077B000002774B13146204600F0E5F80546B5F5DE
:1077C000003F05D20C2D01D9284600E00C200746C9
:1077D00000BF3846BDE8F0811FB53A200390C420B1
:1077E0000290982001900020009000224FF48071B8
:1077F0001748FBF725F8062000F074F80A2003F07C
:1078000036F9012211021248FBF71AF803AA0121E6
:10781000002000F071F802AA0121084600F06CF87F
:1078200001AA0121022000F067F86A460121032025
:1078300000F062F800224FF480710548FBF700F871
:107840000A2003F014F9082000F04CF81FBD0000D6
:107850000004004810B500224FF480711648FAF772
:10786000EFFF102000F03EF800F02AF813490860FE
:1078700000F026F81149096840EA01200F49086024
:1078800000F01EF80D49096840EA01200B49086024
:107890000846006800F4000030B1084600686FF048
:1078A0007F41401A05490860012211020248FAF797
:1078B000C7FF0248006810BD0004004830000020E7
:1078C0000EB5FF200290002001900A20012301AA9A
:1078D00002A900900248FCF77CFC9DF804000EBD54
:1078E0002005002001B50A23012269460148FCF762
:1078F00073FB08BD200500202DE9F04106460C462B
:10790000154600224FF480710E48FAF799FF0C21BA
:1079100001EA8601621E02F00302114341F04000B9
:10792000FFF7E0FF002704E015F8010BFFF7DAFF8F
:107930007F1CA742F8DB012211020248FAF780FF00
:10794000BDE8F08100040048024600BF481E084020
:1079500018B100BF00BF00BFFEE700BF481E1040C7
:10796000101A704710B502464B1E13444C1E23EAF2
:10797000040000BF4B1E0B401BB100BF00BF00BF87
:10798000FEE700BF10BD024600BF481E084018B108
:1079900000BF00BF00BFFEE700BF481E10444B1EE3
:1079A000984370472DE9F04180460E464446012039
:1079B0006086002500270DE056F8270025A1F8F77E
:1079C000AFFE10B1681C85B202E0608E401C60867C
:1079D000781C87B256F8270020B156F827000078A7
:1079E0000028E9D1208EA84201D1BDE8F081A06A2B
:1079F00020B1A06A1DF0F2FE0020A062E06A20B172
:107A0000E06A1DF0EBFE0020E062E8001DF008FED9
:107A1000A06200BFA06A18B900BF00BF00BFFEE7A8
:107A200000BF68001DF0FCFDE06200BFE06A18B90D
:107A300000BF00BF00BFFEE700BFA06A08B1E06A58
:107A400000B900256900E06A1EF09EF8258600BF97
:107A5000CBE700000A0000002DE9F84F81460E46F2
:107A6000924699F8090000F00700022801D130463B
:107A700000E050468346564501DD304600E0504662
:107A80000746032000EB470020F0030000F110053B
:107A90003948006839490968A0EB0108002405EB62
:107AA000080037490968884206D23348046860688C
:107AB00020F0004060603AE031480068854221D8FB
:107AC00013E04FF0FF300090002269462D4810F07F
:107AD000C7FD002269462C4810F0C2FD2648006808
:107AE00026490968A0EB010800BF08EB05002449FE
:107AF00009688842E5D820480468606820F00040A2
:107B0000606014E028461DF08BFD044600BF1CB9E0
:107B100000BF00BF00BFFEE700BF14B90020BDE8F2
:107B2000F88F606820F0004000F10040606032464D
:107B30005946484602F078FC2060606800F04040FA
:107B4000401C6060606820F080406060A781A4F8FD
:107B50000EB06068C00F20B1204600F11001A16096
:107B600008E0054800681030A06003480068284419
:107B7000014908602046D2E7DC00002038020020DE
:107B8000D800002083370108218A0108F0B585B0AC
:107B900006460D4634460020049003900290654846
:107BA0000088A84202D0FF20634908706148058020
:107BB00094F83C0000F0030020B1012838D00228DE
:107BC00066D000BF94F83C0000F003005A490978E1
:107BD00088421BD02620005D00EB001000EB400027
:107BE000142190FBF1F0554908702720005D00EB4F
:107BF000001000EB4000142190FBF1F05049087098
:107C000094F83C0000F003004B49087002A803A957
:107C1000CDE9001005EB45014FF6FF7202EA410085
:107C200004AB47490A78454909780BF079FA5FE0D7
:107C300094F83C0000F003003F49097888421AD0CC
:107C4000A08C00EB400040024FF4B471B0FBF1F0A7
:107C50003C4908802720005D00EB001000EB40004D
:107C6000142190FBF1F03649087094F83C0000F0C4
:107C700003003149087002A803A9CDE90010E9B258
:107C800004AB2F4802782F4800880BF049FA2FE008
:107C900094F83C0000F003002749097888421AD084
:107CA000A08C00EB400040024FF4B471B0FBF1F047
:107CB000244908802620005D00EB001000EB400006
:107CC000142190FBF1F01D49087094F83C0000F07D
:107CD00003001949087002A803A9EAB204ABCDE970
:107CE000001016480178174800880BF019FA00BFF9
:107CF00000BF9DF810009DF80C109DF80820D708D3
:107D0000BDF8003067F304038F080093BDF800301E
:107D100067F34A13C7080093BDF8003067F3CF2319
:107D20000093BDF800703B460193BDF8041008466F
:107D300005B0F0BD8C0100208A01002088010020E0
:107D4000890100208601002010B501200749087034
:107D50000748FEF749FF20B90648006827F0CCFE27
:107D600003E00448006827F0D3FE10BD1402002091
:107D7000043500201802002010B5044694F8420093
:107D8000C0F3400070B9B4F8400000280ADDB4F830
:107D900040004FF6FF71884204D0B4F84000401E06
:107DA000A4F84000B4F84000D0B9A06B20B194F81A
:107DB0004200C0F3400098B121461A48FEF7CDFFBB
:107DC000FFF7C2FFE06810B12046E16888472069EC
:107DD00010B120462169884720461DF0FFFC1FE0B6
:107DE000E06B40422063A06BD0B194F84210C1F325
:107DF000400111B9616B4942216394F8421049086E
:107E0000C94394F8422061F3410284F84220206A79
:107E1000A16A2162A062E06AA16BE162A06300BF77
:107E200010BD0000043500202DE9F0418046424895
:107E3000006827F0C3FC06464048007880F0010047
:107E40003E4908703E48FEF7CFFE04466BE0002036
:107E50003C49087094F84200C0F380003749097823
:107E6000884253D0354801783034A07C61F38200D9
:107E7000A07420688719A07C303CC0F3C00010BB00
:107E8000206B00281FDC002F1DDB94F8420000F05F
:107E9000010060B9606950B12046616988470546B4
:107EA000206A28442062A06A2844A06200BFA0681B
:107EB00010B12046A168884794F8420020F00800DD
:107EC000083084F84200206B30442063206B002887
:107ED0001BDBD4E90B10884201DDE06A20632046F9
:107EE000E16988470546606AA84206D06562606815
:107EF00018B12946D4E900029047D4E90B10884212
:107F000002DB2046FFF738FF00BF00BF0D480078B6
:107F100020B10B48FEF768FE044604E021460848FD
:107F2000FEF77AFE0446002C91D127F055FC024959
:107F30000860BDE8F081000010020020150200205A
:107F4000043500201402002070B504460D46606818
:107F500018B129466068FFF7F7FF206818B1294675
:107F600020462268904770BD70B505460C46A1B208
:107F7000284611F0F0FF70BD70B505460C46A1B261
:107F8000284612F039F870BD2DE9FF4F8FB01F461B
:107F9000DDF888801C980E901D980D9000200B90A5
:107FA0002398042806D0052809D006280CD01428C8
:107FB0001AD114E000200C904FF0020917E00120C4
:107FC0000C904FF0030912E001200C904FF00209D1
:107FD000FFF7BEF905462868008F0B9007E00120E7
:107FE0000C904FF0020902E013B0BDE8F08F00BF23
:107FF000002489E11E9860430E9901EB20201C901B
:108000001F9860430D9901EB20201D901C980512CC
:108010001D980612002D07DB1098854204DA002E09
:1080200002DB1198864203DB002008F8040069E1B6
:108030001C98C0B20A901D9800F0FF0A0A98802888
:1080400007DA4FF0FF3B0A98C0F17F0040000A902A
:1080500005E04FF0010B0A98803840000A90BAF111
:10806000800F07DA4FF0FF300990CAF17F004FEA26
:10807000400A05E001200990AAF180004FEA400A79
:108080000F98089006FB07F000FB09F005FB0901BB
:1080900008980844089005EB0B0000287EDB05EBF0
:1080A0000B011098401E814278DC0998304400286A
:1080B000F4DB099831181198401E8142F4DC0898CD
:1080C000079008980BFB09000690099800FB07F140
:1080D000089801FB090005900C9800287FD0239B8D
:1080E000052B06D1079B9878059B9978069B9A7873
:1080F0003BE0239B142B18D1DDF844C007FB0CFC9C
:10810000DDF83CE00EEB4C0306FB073C1CF80500D9
:1081100006FB073CAC441CF80B20DDF824C0B4443B
:108120000CFB073C1CF805101FE0239B062B19D104
:10813000079B1B88BDF82CC063450BD0059B1B8893
:10814000BDF82CC0634505D0069B1B88BDF82CC02C
:10815000634503D1002308F80430D3E0FF20FF215A
:10816000FF2202E0FF20FF21FF22814207D001FB16
:108170000AF3CAF5807C00FB0C33C3F3072182426B
:1081800009D00A9B5343DDF828C0CCF5807C00FB66
:108190000C33C3F307228B185B1000E059E008F89A
:1081A000043018F8043003B9ACE0079B93F800C022
:1081B0005B780CEB03239BB20493059B93F800C000
:1081C0005B780CEB03239BB20393069B93F800C0F0
:1081D0005B780CEB03239BB202930CE0FFE707985C
:1081E0000088049006980088029005980088039003
:1081F000FF2008F80400BDF81000BDF80C108842FC
:108200000CD1BDF81000BDF80810884206D12198A5
:1082100000EB4400BDF81010018019E00AF0FF02E5
:10822000DDE9030114F084FC03900A98C2B20499BA
:10823000029814F07DFC02907F22DDE9020114F027
:1082400077FC0190219800EB4400BDF804100180F8
:1082500057E008990A78497802EB01218AB22199FE
:1082600021F814202399052904D0062905D01429C2
:1082700019D10EE00899887817E0219931F8141087
:10828000BDF82C20914201D1002100E0FF210846D9
:108290000BE0119A07FB02F10F9A02EB410106FB7A
:1082A0000711485D01E0FF2000BF00BF15B9BBF119
:1082B000000F06DB1099491EA9420BD1BBF1000F3C
:1082C00008DD0A99C1F1FF014143C1F3072108F814
:1082D000041015E016B90999002906DB1199491E09
:1082E000B1420AD10999002907DDCAF1FF014143D2
:1082F000C1F3072108F8041002E0002108F8041077
:1083000000BF00BF601C04B220988442FFF672AE2A
:1083100000BF69E62DE9F84F04468C469046994621
:10832000109FDDE90A56AA460096002032E00C991B
:1083300041430AEB21250D994143DDF800B00BEBD9
:1083400021262A123312002A05DB624503DA002BAC
:1083500001DB434502DB0021395419E0214603FBD0
:1083600009FB0BEB4B0B02EB420EF344594491F823
:1083700000B091F801E00BEB0E2B1FFA8BFEDDF83D
:108380003CB02BF810E091F802B007F800B000BF45
:10839000411C08B20E998842C9DBBDE8F88F1CB5B4
:1083A000AB200090012201A943F6FF7000F01EF8F7
:1083B0009DF80400AB2801D101201CBD01226946B3
:1083C00043F6FF7000F07CF8012201A943F6FF702C
:1083D00000F00CF89DF80400AB2801D10120ECE777
:1083E0000020EAE710B5FFF7DAFF10BD2DE9FE4FD8
:1083F00005460E4614462846E91705EB916189119A
:10840000A5EB8119C9F14007BC420EDC4FF0FF30EB
:1084100002232A46A021CDE9006402902748FAF7FA
:10842000F1FA052002F023FB37E04FF0FF31B8B23C
:1084300002232A46CDE900600291A0211F48FAF7E5
:10844000E1FA052002F013FBE81985B2E01B84B2C3
:108450003E442046E11704EB91614FEAA11A4FF028
:10846000000817E04FF0FF30402102232A46CDE9F3
:1084700000610290A0211148FAF7C4FA052002F029
:10848000F6FA05F1400085B2A4F1400084B240360E
:1084900008F10108D045E5DB00BF6CB14FF0FF30BB
:1084A00002232A46A021CDE9006402900348FAF78E
:1084B000A9FA052002F0DBFABDE8FE8FCC0400200B
:1084C0002DE9FE4F05460E4614462846E91705EBF2
:1084D00091618911A5EB8119C9F14007BC420EDCFD
:1084E0004FF0FF3002232A46A021CDE9006402901C
:1084F0002748FAF757FB052002F0B9FA37E04FF0AA
:10850000FF31B8B202232A46CDE900600291A021D2
:108510001F48FAF747FB052002F0A9FAE81985B2CF
:10852000E01B84B23E442046E11704EB91614FEA20
:10853000A11A4FF0000817E04FF0FF30402102234E
:108540002A46CDE900610290A0211148FAF72AFBE2
:10855000052002F08CFA05F1400085B2A4F140003C
:1085600084B2403608F10108D045E5DB00BF6CB1AC
:108570004FF0FF3002232A46A021CDE9006402908B
:108580000348FAF70FFB052002F071FABDE8FE8FF1
:10859000CC04002030B591B004462546A88F18B908
:1085A000204629F039F81EE0684610F05BFF2946A6
:1085B000684611F01AF80D49684610F0E1FFA98FDE
:1085C000684610F0F2FF01220021684611F003F81E
:1085D0000749684610F0D8FF0648039000BF684678
:1085E00011F016F800BF11B030BD0000A11603084D
:1085F0004F950108A316030870B504460D4600BF49
:10860000204600F03BF818B100BF00BF00BFFEE7F6
:1086100000BF284600F050F9001D61680844606002
:10862000204600F03AF8204670BD70B505460C466D
:10863000284600F041F904F11001884201D30120DD
:1086400070BD0020FCE70146A1F1080070477CB531
:1086500005460C46204600F02FF906466A4601A959
:1086600028F0CAFB21462846DDE900320FF046FB20
:108670007CBD0146087900F00100704710B5044642
:10868000204600F019F908B9012010BD0020FCE7D0
:108690000146087900F00200704770B50446204694
:1086A00000F097F805462C60284670BD7CB506465C
:1086B0000C4600200190009000256CB16A4601A98B
:1086C000204628F0B6FB01980B2805DA6A4601A976
:1086D00030462AF053FD054685B100BF284600F01C
:1086E000EBF8A04203D200BF00BF00BFFEE700BF0F
:1086F00029463046DDE900322AF084F828467CBD60
:1087000070B504462046FFF7C8FF0546284600F02E
:10871000BEF8204600F0B6F870BD70B5044620469D
:1087200000F057F80546284600F0B6F8204600F05D
:10873000BEF870BD70B506460D46284600F049F8F3
:10874000044600BF1CB900BF00BF00BFFEE700BF6A
:108750002046FFF78EFF90B100BF2846FFF78EFF3F
:1087600018B100BF00BF00BFFEE700BF2146304682
:1087700000F076F821462846FFF73EFF05462846DA
:1087800070BD70B506460D462846FFF781FFF0B173
:10879000284600F057F8044600BF1CB900BF00BFD0
:1087A00000BFFEE700BF00BF2046FFF762FF18B919
:1087B00000BF00BF00BFFEE700BF2146304600F00B
:1087C0004FF829462046FFF717FF054600BF284609
:1087D00070BD2DE9F0410446204600F06DF8061FFB
:1087E000204600F0B8F80746314628F013FE05464B
:1087F00000BF2046FFF742FF18B100BF00BF00BF17
:10880000FEE700BF2846BDE8F0812DE9F0410646AD
:108810000C461546002794B100BF1DB900BF00BF2C
:1088200000BFFEE700BF2A462146304600F097F819
:108830002046FFF772FF204600F08DF807463846C5
:10884000BDE8F08110B5044600BF2046FFF720FFC9
:1088500018B900BF00BF00BFFEE700BF206810BD11
:108860007CB505460C46204600F026F806466A46CA
:1088700001A928F0C1FA21462846DDE9003229F095
:10888000C1FF7CBD416841F0010141607047416812
:1088900041F0020141607047416821F002014160EE
:1088A0007047426802F003030B434360704741681E
:1088B00021F00101416070470146486820F0030043
:1088C00070472DE9F04706460C46304600F043F865
:1088D0008046211F28F09EFD07463046FFF7ECFF3B
:1088E000211D451A00BF384600F035F8814638464C
:1088F00000F031F880460421FFF734F8814503D0B9
:1089000000BF00BF00BFFEE700BF00BF3046FFF75B
:10891000D3FF2919091D884203D000BF00BF00BF43
:10892000FEE700BF29463846FFF7BBFF00BF3846C9
:10893000FFF7C2FF0C2803D200BF00BF00BFFEE755
:1089400000BF21463046FFF7ACFF3846FFF7D8FEA0
:108950003846BDE8F087014601F1080070472DE96F
:10896000F04106460C46154600BF2046FFF781FE43
:1089700018B900BF00BF00BFFEE700BF2946204670
:10898000FFF753FE78B129462046FFF79AFF0746C6
:108990002046FFF782FE3846FFF779FF394630461A
:1089A000FFF755FE00BFBDE8F0812DE9F041064616
:1089B0000C46154600BF2046FFF75BFE18B100BF0E
:1089C00000BF00BFFEE700BF29462046FFF72DFE8F
:1089D00088B129462046FFF774FF07463846FFF75F
:1089E0005BFF39463046FFF7A5FE0746394630465D
:1089F000FFF72DFE00BFBDE8F0812DE9F8430646E4
:108A000034461AF06BFE804640461AF0ACFE78BB46
:108A1000304618F0C2FA38B3304618F03AF9208FD1
:108A2000E18E884212D0E08E2087E08E00906A4668
:108A30001C21304618F0A2FD0746012F02D038460F
:108A4000BDE8F883304621F0B4FA00BF40461AF082
:108A50009AFE0546042D06D130461FF02DF8074634
:108A6000002119F091FC09E0304618F0F9FA05E010
:108A7000FFE7208FE086304621F09BFA0120DFE7F8
:108A80002DE9F0410446204618F072FD05462846BF
:108A90001FF06CF80646284612F098FB07460022A5
:108AA0003946304626F080F8BDE8F0810146C1F332
:108AB000002070470146C1F3C01070470146C1F362
:108AC000002070470146C1F3402070470146C1F3C2
:108AD000001070470146C1F3801070470146C1F392
:108AE000802070470146C1F3C02070470146C1F3A2
:108AF000401070472DE9F04F89B004460D46002123
:108B000020461EF0CDFE30B91C2128461DF03CF851
:108B100009B0BDE8F08F2946204600F00BFB29463E
:108B2000204600F07DF80021204620F0E7F808906C
:108B30000021204620F04AFA0790002120461FF02D
:108B40009CFE012800D100E0002081460021204643
:108B500020F0D6FC0746002120461FF075FF064690
:108B600042F2D170874205D1608CC0F3802008B9F1
:108B7000012000E00020824620461EF031FF0690D2
:108B800000BF4FF00008244802884146204620F0EC
:108B9000DDFA03900398C0B200BF8346AA68296932
:108BA0002868CDE90209CDE900125A465146089BD2
:108BB00006980DF083F8288342F2D170864205D1E1
:108BC000608CC0F3402008B9012000E0002005902F
:108BD00020461EF0E6FE049000BF4FF000080F484C
:108BE00002884146204620F0B1FA03900398C0B2B3
:108BF00000BF83460023EA6869686869CDE902130B
:108C0000CDE900025A46079BDDE904010DF056F854
:108C1000688300BF7CE70000FC000020000100200A
:108C20002DE9F34F87B00C4607980BF077FE80468E
:108C300007981EF0D5FE0690404601F08BFD20619E
:108C4000216948001CF036FD2060216948001CF0B5
:108C500031FDA060002548E05848029038F9150021
:108C600041F69A7188423FD10020019029E0019994
:108C700007981EF015FE00905149009820F0E1FD84
:108C800000B11BE000980BF067FE8246BAF1010FBD
:108C900000D013E000980BF04FFE8346AB4500D0A8
:108CA0000CE0009820F065FD0299884201DA0298F4
:108CB00002E0009820F05DFD029000BF0198401C8A
:108CC000019007981EF00AFE01998842CFD80298B9
:108CD000002804DB0298A16821F8150003E00021B8
:108CE000A06820F8151000BF6D1C2069A842B3D8F9
:108CF0000026B14600251BE038F9150041F69B71AE
:108D0000884202DB411A0E4411E041F69A71884212
:108D100006D1A16831F8151049440FFA81F906E02F
:108D2000A16821F8150009EB00010FFA81F96D1C0B
:108D30002069A842E0D8002107981FF0DFFF0590C6
:108D40002169491EDDE9050200FB112000B20690F1
:108D50000698A0EB090007B2002F00DA00274FF0B9
:108D6000FF30049000200390002513E038F915002F
:108D700041F69B7188420CDB421A11B207FB01F2EB
:108D8000B2FBF6F212B2A36823F815200495039102
:108D900000BF6D1C2069A842E8D8049800280ADBAF
:108DA0000398301A7843B0FBF6F0381A01B2A26883
:108DB000049822F8101009B0BDE8F08F01E0FFFF21
:108DC000010006002DE9FC5F0546002211462846F9
:108DD00022F066FA002128461FF0B7FD81460021E7
:108DE000284620F017F9484407B2002128461FF012
:108DF000F5FE48440FFA80FA28461FF0ABFC3844D1
:108E000050440FFA80FB3B4E28461EF067FD019050
:108E10004FF000085CE0A868006850F82840364928
:108E2000204620F00EFD00B150E0204621F038F938
:108E3000002839D1002120461FF0BDFC0090009889
:108E400030B1012807D0022804D0032815D100E052
:108E500000BF00BF00BFB4F91A10B5F91600081A18
:108E6000401CB04201DA304605E0B4F91A10B5F9F9
:108E70001600081A401C06B214E00021204620F01B
:108E80006FFB70B904F1140011F099F93844B04245
:108E900001DA304604E004F1140011F090F938448E
:108EA00006B200BF00BF10E0B4F91A10B5F9160001
:108EB000081A401CB04201DA304605E0B4F91A1035
:108EC000B5F91600081A401C06B200BF08F10108E7
:108ED000019880459FD30748864209D006EB0A00D7
:108EE00006B25E4502DD3046BDE8FC9F5846FBE712
:108EF0005846F9E701E0FFFF010004002DE9FC5F9F
:108F0000054600221146284622F0AEF900212846E7
:108F10001FF01BFD8246002128461FF0C7FF50446A
:108F20000FFA80F8002128461FF024FF50440FFA62
:108F300080F928461FF01EFC4844404400B20190CE
:108F4000724C28461EF0CAFC8346002128461FF0BA
:108F500070FC012866D100265BE0A868006850F824
:108F600026706B49384620F06CFC00B150E0384662
:108F700021F096F8002839D1002138461FF01BFC5B
:108F80000090009830B1032805D0062804D00828A6
:108F900015D102E000BF00BF00BFB5F91800B7F956
:108FA0001410401A401CA04201DA204605E0B5F931
:108FB0001800B7F91410401A401C04B214E0002144
:108FC000384620F0C1FA70B907F1140011F06AF9BF
:108FD0004044A04201DA204604E007F1140011F0F9
:108FE00061F9404404B200BF00BF10E0B5F91800B9
:108FF000B7F91410401A401CA04201DA204605E0DF
:10900000B5F91800B7F91410401A401C04B200BF9B
:10901000761C5E45A1D33D48844269D004EB09002B
:1090200004B265E000265BE0A868006850F826708E
:109030003749384620F005FC00B150E0384621F0B1
:109040002FF880BB002138461FF0B5FB0090009838
:1090500030B1012805D0042804D0072815D102E03A
:1090600000BF00BF00BFB7F91800B5F91410401ACF
:10907000401CA04201DA204605E0B7F91800B5F916
:109080001410401A401C04B215E00021384620F0AC
:1090900067FA78B907F1140011F004F94844A042C6
:1090A00002DA204605E008E007F1140011F0FAF8B2
:1090B000484404B200BF00BF10E0B7F91800B5F98A
:1090C0001410401A401CA04201DA204605E0B7F90E
:1090D0001800B5F91410401A401C04B200BF761CE9
:1090E0005E45A1D30948844202D004EB080004B2D3
:1090F0000648844202D10198BDE8FC9F0198844251
:1091000001DD2046F8E70198F6E7000001E0FFFFE7
:109110000100040010B5044620681CF047FB60689D
:109120001CF044FBA0681CF041FBE0681CF03EFB17
:1091300010BD00002DE9F34F87B00C4607980CF0E6
:10914000D5FB8046404601F005FB6061616948003F
:109150001CF0B0FA6060616948001CF0ABFAE06096
:10916000002547E05948029038F9150041F69A71F8
:1091700088423ED14FF0000A29E0514607981EF080
:109180008FFB01905249019820F05BFB00B11CE07D
:1091900001980CF06BFC8346BBF1010F00D014E08A
:1091A00001980CF053FC00900098A84200D00CE00D
:1091B00001981EF08BFC0299884201DA029802E0C5
:1091C00001981EF083FC029000BF0AF1010A079883
:1091D0001EF084FB5045D0D80298002804DB02988A
:1091E000E16821F8150003E00020E16821F815008E
:1091F00000BF6D1C6069A842B4D80026B1460025A6
:109200001BE038F9150041F69B71884202DB411AD8
:109210000E4411E041F69A71884206D1E16831F8B6
:10922000151049440FFA81F906E0E16821F81500AC
:1092300009EB00010FFA81F96D1C6069A842E0D8C2
:10924000002107981FF0C2FE069007981EF0A9FBA8
:1092500001466269521E069800FB121000B205908A
:109260000598A0EB090007B2002F00DA00274FF0A5
:10927000FF30049000200390002513E038F915001A
:1092800041F69B7188420CDB421A11B207FB01F2D6
:10929000B2FBF6F212B2E36823F8152004950391AD
:1092A00000BF6D1C6069A842E8D8049800280ADB5A
:1092B0000398301A7843B0FBF6F0381A01B2E2682E
:1092C000049822F8101009B0BDE8F08F01E0FFFF0C
:1092D0000100060038B5044600256E2229462046C6
:1092E0001FF034FF0090009800B208B1022038BD92
:1092F00000256D22294620461FF028FF0090009887
:1093000000B2B0F5807F01D00220F0E70025612295
:10931000294620461FF01AFF00900098C0B2FF288F
:1093200001D00120E3E700256822294620461FF0EE
:109330000DFF00900098C0B208B10120D7E70020CF
:10934000D5E77CB504460D46164628882189084491
:1093500000B2ADF8000068886189084400B2ADF839
:109360000200A8882189084400B2ADF80400E8880A
:109370006189084400B2ADF80600324669462046CD
:10938000636998477CBD0000F8B505460E462C463B
:10939000A06B58B1284625F0F9FF07461149096826
:1093A0008847A16B884201D30020F8BD606B10B1E3
:1093B000606B007808B90120F7E7002000900AE010
:1093C0006946094A606B126890470746B74201D167
:1093D0000120EAE700BF606B0099405C0028EFD1F4
:1093E00000BFE2E7880200207802002070B5044642
:1093F000204618F05CF80546272D0AD102200649C0
:109400000860064A0121064826F05EFA0549086010
:1094100000E000BF00BF70BD08030020580300201B
:109420008D940008C402002030B587B00446204661
:1094300018F03DF80546072D1BD100200F490860A4
:109440000F48006826F06AFA01200021C822029223
:10945000CDE90321059008460A49CDE900100A48E4
:1094600090F8602000F1D80300F15C0131F0F6FEC5
:1094700000E000BF00BF07B030BD000014030020B3
:10948000C4020020E14103085803002070B52DED0F
:10949000068B0646FE48006864282ED1FD48006809
:1094A00032F0B0FB41EC1A0B9FEDFB0B53EC102B91
:1094B00032F0F6FC41EC190B9FEDF90B53EC102B3D
:1094C00032F002FA41EC180B32F056FB0446F64932
:1094D0000022D1F8E000214611F083F9F34800683A
:1094E00026F01CFAF04A6421AFF25F0026F0ECF996
:1094F000EE4908600020E6490860ED480068002851
:109500007ED10120EA490860EA48EB49096850F831
:109510002100401E00EB8000012101EB4000E749E3
:10952000095CE448E44A126850F82200401E00EB4F
:109530008000002202EB4000E04A105C41EA00207B
:1095400000B2DF490880DB48DB49096850F8210098
:10955000401E00EB8000032101EB40001146095C36
:10956000D448D54A126850F82200401E00EB800013
:10957000022202EB4000D14A105C41EA002000B216
:10958000D0490880B1F90010A1F51C50103832F014
:1095900022FB41EC1A0B9FEDCC0B53EC102B32F05D
:1095A00093F941EC190B9FEDCA0B53EC102B32F0E1
:1095B00079FB41EC180B32F0DFFA00B2C1490880A8
:1095C000BC48BD49096850F82100401E00EB8000EE
:1095D000052101EB4000B949095CB648B64A12685A
:1095E00050F82200401E00EB8000042202EB4000F5
:1095F000B24A105C41EA002000B2B749088000E09E
:109600000BE1AC48AC49096850F82100401E00EB62
:109610008000072101EB40001146095CA548A64ADD
:10962000126850F82200401E00EB8000062202EB78
:109630004000A24A105C41EA002000B2A74908801D
:109640009C489D49096850F82100401E00EB8000AD
:10965000092101EB40001146095C9648964A1268C0
:1096600050F82200401E00EB8000082202EB400070
:10967000924A105C41EA002000B29949088099485A
:1096800090F8E903974991F8E81340EA012004B201
:109690009148B0F90000401E40F2E93101EB400072
:1096A0009049095C8C48B0F90000401E4FF47A7272
:1096B00002EB40008B4A105C41EA002005B2AC424C
:1096C00007DA894804608948056089A08A490860EA
:1096D00006E0864804608448056088A086490860E2
:1096E0008248006880490968401A8649086008462F
:1096F0000068B0F5527F0CDA08460068B0F58C7F40
:1097000007DD69490022D1F8F0007FA11BF08AFC37
:109710002EE07C480068B0F5D26F07DA624900227B
:10972000D1F8F00079A11BF07DFC21E075480068BC
:10973000B0F5526F07DA5C490022D1F8F00074A14D
:109740001BF070FC14E06F48006841F6100188427D
:1097500007DA55490022D1F8F0006FA11BF062FC36
:1097600006E051490022D1F8F0006DA11BF05AFC2F
:109770004D490022D1F808015F4909681BF052FCED
:109780004F48B0F9000032F026FA41EC190B9FED7A
:10979000660B53EC102B32F097F841EC180B424952
:1097A00053EC182BD1F8F80061A11BF03BFC4548A5
:1097B000B0F9000032F00FFA41EC190B9FED5A0B93
:1097C00053EC102B32F080F841EC180B364953EC77
:1097D000182BD1F8000158A11BF024FC3E4A128836
:1097E00091B2314AD2F8E80012F09DFB2E49D1F82F
:1097F000E8003B49B1F900303849B1F900200021B7
:1098000012F0D2FB2849D1F8E8003E4909880BB292
:109810000022022112F0C8FB00BF1D4800682E493B
:10982000B1F9001088421BDA21480068012817D1DD
:1098300017490968012303EB41012A4B5B5C14497A
:109840000968002404EB4101264C615C43EA0121D4
:109850000AB21549D1F8E8003949096812F03DFB10
:109860000B4800681C49B1F90010884207D10E4925
:10987000D1F8E80012F0E6FA02200D490860044829
:109880000068401C02490860BDEC068B70BD0000FA
:10989000C802002050000020000000000018904086
:1098A000000000000000084058030020C40200200F
:1098B000CC020020D0020020AC020020302B00207F
:1098C000F8020020FA02002000000000008086401C
:1098D0000000000000D8A340FC020020FE0200208F
:1098E00000030020952B0020B0020020B4020020CD
:1098F000732D3E6500000000BC020020652D3E7304
:1099000000000000B802002023323500233530006B
:1099100023313030000000002332303000000000DE
:109920006E756C6C000000000000000000005940E3
:10993000252E326600000000252E32666D6D000077
:10994000C00200202DE9FF4F8FB00F46209DF87810
:1099500000F0010008B1F94800E0F9480E90F878ED
:1099600000F0010008B1F74800E0F7480D90F878E2
:1099700000F0010008B9F34800E0F3480C90012022
:109980000B90BEE000210B9100206988B5F804C05F
:10999000A1EB0C010AB200261AE006EB860CE9687E
:1099A00001EB8C01097C01F0010141B906EB860C49
:1099B000E96801EB8C018989014408B207E006EBF4
:1099C000860CE96801EB8C010989511A0AB2761CF0
:1099D0002969B142E1D800268EE006EB860CE968E1
:1099E00001EB8C01097C01F0010100297DD100BF50
:1099F00018B900BF00BF00BFFEE700BF92FBF0F840
:109A00000FFA88F306EB8609D5F80C8008EB890875
:109A1000B8F80C8008FB03F80FFA88F106EB86090A
:109A2000D5F80C8008EB8908B8F9049006EB860A93
:109A3000D5F80C8008EB8A08B8F90680884501DD66
:109A4000884607E006EB860AD5F80C8008EB8A0802
:109A5000B8F90680C14508DD06EB8609D5F80C800B
:109A600008EB8908B8F9048013E006EB8609D5F8FD
:109A70000C8008EB8908B8F90680884501DD884626
:109A800007E006EB8609D5F80C8008EB8908B8F9E1
:109A90000680C4468C450BD04FF0010806EB860AC1
:109AA000D5F80C9009EB8A09C9F81080CDF82C8004
:109AB00006EB8609D5F80C8008EB8908A8F808C0E1
:109AC00006EB8609D5F80C8008EB8908B8F80C80FD
:109AD000A0EB08080FFA88F006EB8609D5F80C8091
:109AE00008EB8908B8F8088000E004E0A2EB080859
:109AF0000FFA88F200BF761C2969B1423FF66DAFBC
:109B000000BF0B9800287FF43DAF00210F981EF096
:109B1000A8FE012800D100E000200A900020099052
:109B2000089008A809A9CDE9001029890BB2B5F958
:109B3000022038781E9927F079FCF87800F00100AF
:109B400048B10A9838B10F981DF04AFFBDF82410AB
:109B5000084400B2099011990F981DF0A1FE044627
:109B60008FE17A4920461FF06CFE40B1F878C0F3CF
:109B7000800111AA0F980BF0EAFC044681E1002154
:109B800020461EF039FF07900798002860D000207B
:109B90000390002610E006EB8601E86850F82100EB
:109BA000A04208D106EB8600E96801EB8000B0F91D
:109BB0000800039003E0761C2869B042EBD800BF90
:109BC000F87800F0010050B1608C20F4806000F55E
:109BD00080606084608C20F40070608409E0608C98
:109BE00020F4007000F500706084608C20F48060C8
:109BF000608404F114000D9988470399884226D0A7
:109C0000204620F0D6F900BFA08AADF80400E08A13
:109C1000ADF80600208BADF80800608BADF80A00A7
:109C200000BF04F114000E9A0399904701AA29215C
:109C3000204617F0A3FC20461DF098FF2246222163
:109C4000009017F09BFC204620F0B3F900BF07E01E
:109C5000608C20F480606084608C20F400706084EC
:109C6000002006907878012812D0022819D104F13A
:109C700014000C998847B5F90010491C21F0010126
:109C8000081A039000EBD070401000B2069009E073
:109C900004F114000C9988472988081A00B206902C
:109CA00000E000BF00BFF87800F0010050B10A9852
:109CB00040B104F114000D998847BDF82410081A2A
:109CC00000B20990002003906B22204603991FF0F8
:109CD0003DFA029002980FFA80F800BF002003902E
:109CE0006C22204603991FF031FA029002980FFA75
:109CF00080F900BF20461FF03CFD059020461DF076
:109D0000E5FE049008F4C040B0F5005F01D10120E9
:109D100000E0002030B128F4C040B0F5FA6F01DC5B
:109D2000012000E00020E0B128F4C040B0F57A7FC7
:109D30000EDD28F4C040C0F57A700BE0F1A30108F5
:109D4000E5A3010831A3010813A2010801000600E0
:109D500028F4C04005994843642190FBF1F00FFAC4
:109D600080F809F4C040B0F5005F01D1012000E0A7
:109D7000002030B129F4C040B0F5FA6F01DC0120B9
:109D800000E0002090B129F4C040B0F57A7F04DDF6
:109D900029F4C040C0F57A7001E029F4C04004996C
:109DA0004843642190FBF1F00FFA80F9A18A1C98D6
:109DB000401A40440FFA80FAE18A1D98401A48443C
:109DC0000FFA80FBF87800F0010010B1BDF9240013
:109DD00000E0069850440FFA80FAF87800F001008D
:109DE00008B1069801E0BDF9240058440FFA80FB41
:109DF000BAF1000F02D1BBF1000F1BD0204620F0BA
:109E0000D8F8A08A504400B2A082208B504401B2FE
:109E10002183E08A584401B2E182608B584401B248
:109E20006183204620F0C5F800235A46514620465B
:109E300020F096F9F87800F0010008B10A9870B99E
:109E400004F114000D9988471F990844BDF82010AB
:109E50000844BDF82410084400B2099008E0BDF899
:109E600020101F980844BDF82410081A00B2099069
:109E7000F878C0F3800111AA0F980BF068FB044634
:109E800000BF24B1DDE9111081427FF46AAE13B046
:109E9000BDE8F08F2DE9F04F8DB005468946B9F148
:109EA000000F02D10DB0BDE8F08FA5F8189028681A
:109EB00010B128681BF092FC09EB4901062202EB65
:109EC00041001BF0ADFB286000BF286818B900BF37
:109ED00000BF00BFFEE700BF286868600221286855
:109EE00001FB0900801CE8600421286801FB0900CF
:109EF000001DA860B9F1010F0CD1B4206968087089
:109F00000020E96808800120E96848800020A968ED
:109F10000880C7E709F10101C8001BF0CBFB074629
:109F200009F1010007EB80084FF0000A4FEA8900B1
:109F300002B20BA90CA800F067F90024BDF93000AB
:109F40008010079000200390CCE0002616E00BA9BB
:109F50000CA800F061F90CA800F04BF900B90FE073
:109F6000BDF93000801007A941F82600BDF8300087
:109F700000F0030003A941F82600761C042EE6DB5E
:109F800000BF042E00D0B3E00A990798884219D187
:109F9000079800B227F814000FFA8AF028F8140086
:109FA000DDE90301084405990844069908446968F5
:109FB00008556868005D0007000E69680855601C58
:109FC00004B28DE0DDE9070188422CD0079800B289
:109FD00027F814000FFA8AF028F81400039869682B
:109FE00008556868005D0007000E69680855601C28
:109FF00004B20798401E00B227F814000FFA8AF046
:10A0000028F814000498001D05990844069908448E
:10A01000696808556868005D0007000E69680855A2
:10A02000601C04B25CE00999079888422CD007981C
:10A0300000B227F814000FFA8AF028F81400DDE9BE
:10A0400003010844696808556868005D0007000E50
:10A0500069680855601C04B20798401E00B227F8D2
:10A0600014000FFA8AF028F81400059808300699B1
:10A070000844696808556868005D0007000E696853
:10A080000855601C04B22BE0079800B227F81400B2
:10A090000FFA8AF028F81400DDE903010844059955
:10A0A0000844696808556868005D0007000E696823
:10A0B0000855601C04B20798401E00B227F814002F
:10A0C0000FFA8AF028F8140006980C3069680855D1
:10A0D0006868005D0007000E69680855601C04B2DE
:10A0E0000AF1010A0CA800F084F800287FF42DAFD3
:10A0F00000BF40F2D32109FB01F0029002988012C8
:10A100000190601E37F910100198814205D1601E40
:10A1100038F910100198814226D0DDE90121A1EB28
:10A120008220B0F5007F04DC00FB00F14800001441
:10A1300007E0C0F5806000FB00F148000014C0F1AA
:10A140000F00019909B227F81410019909B228F8F3
:10A1500014106A6810556968095D0907090E6A6874
:10A160001155611C0CB200BFA61E0EE038F8160097
:10A1700027F8140037F8160028F814006868805D86
:10A1800069680855761E601C04B2002EEEDA4FF0A6
:10A19000000B00260020E968088023E0E96821F828
:10A1A0001B6037F81600A96821F81B0010E0A868AA
:10A1B00030F81B0037F91610884203DAA86830F827
:10A1C0001B0001E037F91600A96821F81B00761C76
:10A1D00038F91600584501D1A642E8DB0BF1010021
:10A1E0000FFA80FBA642D9DB38461BF0DFFA00BF2E
:10A1F00058E60146B1F90200B1F90020904201DCB5
:10A20000012070470020FCE7028000234380C2F158
:10A2100001031BB20B807047B1F90020002A07DC54
:10A220000B8842885200D21C1A4412B20A800CE0F9
:10A2300042880388D21A5200521D0B881A4412B267
:10A240000A800288521E12B202804288521C12B248
:10A250004280704737B582B01546022D04DCBDF848
:10A260000C10084605B030BDBDF80C00C00ABDF8A2
:10A27000081000EBD1241F2C01D2204600E01F2043
:10A28000BDF8081060F3CF210291BDF80C00C0F3B7
:10A290004510BDF80810C1F3451144183F2C01D2F8
:10A2A000204600E03F20BDF8081060F34A110291FB
:10A2B000BDF80C0000F01F00BDF8081001F01F01F0
:10A2C00044181F2C01D2204600E01F20BDF80810C2
:10A2D00060F304010291FF2D03D1BDF80810084678
:10A2E000C0E72A46DDE9020112F000FC0190BDF84A
:10A2F00004100846B6E717B581B01446022C04DCFA
:10A30000BDF80810084604B010BDBDF80400C00A2E
:10A31000BDF80810C90A10FB01F04109BDF804009E
:10A3200061F3CF200190BDF8040000F01F00BDF8DC
:10A33000081001F01F0110FB01F04109BDF80400F5
:10A3400061F304000190BDF80400C0F34510BDF8AE
:10A350000810C1F3451110FB01F08109BDF804009C
:10A3600061F34A100190FF2C03D1BDF80410084698
:10A37000C9E72246DDE9010112F0B8FB0090BDF803
:10A3800000100846BFE737B582B01546022D04DC41
:10A39000BDF80C10084605B030BDBDF80C00C00A71
:10A3A000BDF80810A0EBD124002C01DD204600E010
:10A3B0000020BDF8081060F3CF210291BDF80C0019
:10A3C000C0F34510BDF80810C1F34511441A002C24
:10A3D00001DD204600E00020BDF8081060F34A11BE
:10A3E0000291BDF80C0000F01F00BDF8081001F04C
:10A3F0001F01441A002C01DD204600E00020BDF8BA
:10A40000081060F304010291FF2D03D1BDF808107C
:10A410000846C0E72A46DDE9020112F067FB019019
:10A42000BDF804100846B6E708B503460093009847
:10A43000484080EA620008BD2DE9FC5F8246504634
:10A4400017F096F80190504617F031F8064601983B
:10A450001DF08CFB0746BB462B2E09D1384624F055
:10A4600096FB044600222146384624F09DFB5FE01F
:10A470000A2E5DD119F032F98046B8F1000F05D0EF
:10A4800098F80400012801D1BDE8FC9F69460198B5
:10A490001DF0EEFB9BF82C0000F00C00F8B10198C9
:10A4A0001DF09EFA0546002138461EF0F2F90128FB
:10A4B0000AD1284605EBD071BDF90020C2EB61013D
:10A4C00091FBF5F10CB209E0284605EBD071BDF91E
:10A4D000002002EB610191FBF5F10CB20EE0019856
:10A4E0001DF05FFA0546284605EBD071BDF9022044
:10A4F00002EB610191FBF5F10CB200BF002C00DA18
:10A5000000244FF00009384624F041FBA04201D05E
:10A510004FF0010901222146384624F045FBB9F1EC
:10A52000000F04D000221C21384617F027F800BF86
:10A5300000BFA9E710B58060C0600023036100215F
:10A5400010E0002400F1140343F82140002206E04B
:10A5500000F1400303EBC11343F82200521C202AF0
:10A56000F6DB491C0B29ECDB10BD2DE9FF4F87B052
:10A570000546DDE9178ADDF85890149F089CB9F16B
:10A58000040F02D0B9F1060F58D128460FF072FE21
:10A590008346594650461BF02EFBB5F9020078431E
:10A5A0004100B5F9000001EB4000044428460FF0DB
:10A5B0008EFE0590059840000490780000B203904C
:10A5C000CDF80880B5F902600DE02146049A0298A2
:10A5D0001BF058F9039804440599029800EB4100D8
:10A5E0000290701C06B2B5F90600B042EDDAB9F17E
:10A5F000060F22D14FF47F414FF0000C01F47C4E46
:10A600004CEA5E1CC1F3C40E4CEA0E0CCDF800C03F
:10A61000BDF800E0F446CDF804C04246BDF8043071
:10A62000002007E032F81010994202D100210AF808
:10A630000010401C5845F5D300BF88E0B9F1050F64
:10A6400041D1B5F90200784300EB4000B5F90010A4
:10A6500001EB41010844044428460FF038FE381A43
:10A6600000B20590059800EB400000B20490284627
:10A670000FF0BAFD039028460FF029FE834600260E
:10A680001DE00020069010E0A17806980AF800105E
:10A690002078617800EB012081B2069828F810102C
:10A6A000E41C0698401C00B2069006985845EBDB67
:10A6B00008EB4B08DA4404980444701C06B2039873
:10A6C0008642DEDB43E0B9F1140F40D1B5F9020058
:10A6D00078434100B5F9000001EB400004447800E4
:10A6E00000B2059028460FF07FFD049028460FF039
:10A6F000EEFD834600260BE04FEA4B022146404622
:10A700001BF0C0F808EB4B0805980444701C06B217
:10A7100004988642F0DB089C099841000A9801FBE6
:10A720000044B5F90000B5F9021007FB010004442C
:10A73000002608E05A46214650461BF0A3F8DA44AA
:10A740003C44701C06B204988642F3DB00BF0BB099
:10A75000BDE8F08F0146002000E0401C31F91020D8
:10A7600041F6FF739A42F8D170477CB506460D4614
:10A7700034465420005D00F00100A84233D00DB1F2
:10A78000012000E000205421095D60F30001542005
:10A79000015504F1480168460FF001FDBDF80000C5
:10A7A000616A898A084400B2ADF80000BDF8021061
:10A7B000606AC08A084400B2ADF80200BDF8040027
:10A7C000616A898A084400B2ADF80400BDF8061039
:10A7D000606AC08A084400B2ADF806006946304697
:10A7E0001FF011FC00BF7CBD37B582B00546144692
:10A7F0002146039811F0D8FF0190BDF804100846D7
:10A8000005B030BD2DE9FF4F8DB007460D46164609
:10A81000E87A022803DC012011B0BDE8F08F288916
:10A820002A6901460C901098FBF7CCFE04460CB93F
:10A830000020F1E7217D01F01F0017F016FE10B196
:10A840004FF0060818E0207D00F01F000E2801D10F
:10A85000804611E0207D00F01F00142801D18046C1
:10A860000AE0217D01F01F0017F0E2FD10B14FF06A
:10A87000050801E04FF00408B8F10E0F09D128884F
:10A8800018B96888B0F5807F03D04FF00508002024
:10A89000A061206A38B100BF00BF31463846226A45
:10A8A0002DF0EDF8DEE0A069002859D031460BA864
:10A8B0000FF03FFC288818B96888B0F5807F32D047
:10A8C00030460FF020FD834600BFF0887188401AA3
:10A8D000401C00B20890281D6988CDE90010B5F928
:10A8E000003059460BA8089AFBF766FDBDF82C000E
:10A8F0003188084400B2ADF82C00BDF82E007188F4
:10A90000084400B2ADF82E00BDF83000318808448C
:10A9100000B2ADF83000BDF832007188084400B2D2
:10A92000ADF8320000BF0BAA09A8B968FBF743FADB
:10A930008146B9F1000F04D1204601F00EFC012040
:10A940006AE7D7F808A009A8B860CDF800803246B9
:10A9500029463846A36913F0D7F9C7F808A081E063
:10A9600032460BA8B968FBF726FA0A900A9820B974
:10A97000204601F0F2FB01204EE70BA80FF0C3FCCC
:10A9800009900BA80FF0BFFC00EB400003901AF0F9
:10A9900091FE8146D7F808A00BA907A80FF0C9FBC4
:10A9A000012107A80FF01EFDBDF92C00B6F900101B
:10A9B000401A0690BDF92E00B6F90210A0EB010B6B
:10A9C000BDF92E00059042E007AA514602A8FBF708
:10A9D000F2F90A900A9800B936E0CDF8009009988B
:10A9E00003B20FFA8BF2069801B2204618F0A0FAD3
:10A9F0000490049801280ED0204618F0B9F900BF41
:10AA000000BF48461AF0D2FE204601F0A6FBC7F868
:10AA100008A0002000E702A8B8604B4607AA294614
:10AA20003846CDF8008013F06FF9BDF81E00401CC9
:10AA300000B2ADF81E00BDF82200401C00B2ADF817
:10AA400022000BF1010B00BF0598401C0590BDF9D9
:10AA5000321005988142B7DAC7F808A048461AF0C4
:10AA6000A5FE00BF204601F078FB0120D4E601B529
:10AA70000098F7F7E9FD08BDF8B506460C461546FF
:10AA80000095E788BBB2A788BAB26788B9B22788B1
:10AA9000B8B225F01DFD304612F0D5FDF8BD704767
:10AAA000F8B505462C4618F019FE0646206B24F032
:10AAB00085FE3168898B88422CD2606A009094F8B8
:10AAC0003C0000F0030020B1012806D002280CD180
:10AAD00007E00020ADF8000007E064208DF80200D8
:10AAE00003E064208DF8030000BF00BF304618F07B
:10AAF000D3FF2846009912F016FC50B100221C2109
:10AB0000284616F03BFD0746012F01D03846F8BD18
:10AB100000BF00BF24F060FE20630120F7E70000C3
:10AB20002DE9F04F9BB0074689461646BA4617A84E
:10AB300012F065FE4FF4A02138461DF053FE9DF83B
:10AB4000691060F382018DF8691030460FF0F7FB51
:10AB5000054600EBD5704FEA60083088404400B2EB
:10AB6000ADF858007088404400B2ADF85A0000219A
:10AB700038461DF0C9FF1590494603A81CF050FC4B
:10AB800017A80B904FF40030109033480490002029
:10AB900005900AF13000FCF74CF8044657E02079A4
:10ABA000032800D04DE0208BADF85C00208A00B275
:10ABB000ADF85E006079FD2801DD159803E060794D
:10ABC0001599484300128DF868002568B5F92000F2
:10ABD000E98B08440090B5F92030D5E90512A0684A
:10ABE0001AF0FAFC8346B5F92000E98B084400907E
:10ABF000B5F92030D5E90512E0681AF0EDFC0290B5
:10AC0000608B404400B2ADF84800149416A80C9034
:10AC100003AA1A21384616F0B1FC029880B21FFA36
:10AC20008BF1CDE90010BDF8480083B216AA17A930
:10AC3000484612F0C6FD03AA1B21384616F09EFCBA
:10AC400000BF21460AF13000FBF7EDFF0446002C5F
:10AC5000A5D11BB0BDE8F08FCCC8030870B5044681
:10AC60000D4600222946204607F034FE01222946DF
:10AC7000204607F02FFE02222946204607F044FC1A
:10AC800004222946204607F03FFC70BD2DE9F74F0E
:10AC90009EB00C46E078022802DC21B0BDE8F08FBF
:10ACA0001CA820990FF03CFAB4F9200001282EDDF1
:10ACB00094F82200FD282ADB208840B3BDF87000FC
:10ACC00014F8231F4908C1F38001084400B2ADF80D
:10ACD0007000BDF8720021784908C1F340010844B2
:10ACE00000B2ADF87200BDF8740021784908C1F3D4
:10ACF000C001401A00B2ADF87400BDF8760014F837
:10AD00002319C1F34001401A00B2ADF876001E9835
:10AD10001CA982681AA8FBF74EF800B9BDE7E07BD2
:10AD200000F0070616B9A088199001E0E088199094
:10AD3000BDF864106089814200D100261CA813F080
:10AD4000BDFF18901C2111A8F5F7C3FCA0788DF861
:10AD50005D00BDF86400ADF84C00189860B920881B
:10AD600050B94EB91CA81190E0788DF85C0011A97B
:10AD70001E9814F05BFE90E7E078FD2801DBFF20D1
:10AD800000E0E07810901CA80FF0B6FA0F901CA815
:10AD90000FF031FA0E90DDE90E01814201DA0F98D1
:10ADA00000E00E980D90B4F900100D98B1EB600F13
:10ADB00002DAB4F9000001E00D98401007461AA825
:10ADC0000FF09AFA81464FF0FF300C9000200B9064
:10ADD000002F01DC189870B148461AF06BFC0B90FC
:10ADE00000233AB21CA905A814F0E0FA002105A836
:10ADF00013F066FC0C90BDF86800ADF80C00BDF8CF
:10AE00006C00ADF810000B98149003A811901690E8
:10AE1000FF208DF85C00A01DDDE90E2117F024F85D
:10AE20008046B8F1000F0CD0022E0AD1BDF968108F
:10AE3000D8F8080000EB4100BDF97010A0EB41000C
:10AE400012901898A0B3BDF96A502CE028B2ADF862
:10AE50000E0028B2ADF812004A4610990B981AF06D
:10AE600059FEBDF968100FFA89F32AB20B9813F056
:10AE7000D5FE8DF854009DF85400012802D102201F
:10AE80008DF85400012E09D1BDF97210691AD8F855
:10AE9000080000EB41000088ADF84C0011A91E9895
:10AEA00014F0C4FD6D1CBDF96E00A842CEDACCE0F2
:10AEB000FFE700255CE0BDF8720028440FFA80FA35
:10AEC000BDF87600401B0FFA80FBBDF96A005045C3
:10AED00004DDBDF96E00584500DA48E04A46109995
:10AEE0000B981AF017FEBDF90C100FFA89F35246B1
:10AEF0000B9813F093FE8DF854009DF85400012830
:10AF000002D102208DF85400BDF96A00504514DCCE
:10AF1000ADF80EA0ADF812A0012E0AD1BDF9721045
:10AF2000AAEB0101D8F8080000EB41000088ADF859
:10AF30004C0011A91E9814F079FDBDF96E0058451A
:10AF400014DBADF80EB0ADF812B0012E0AD1BDF988
:10AF50007210ABEB0101D8F8080000EB410000884B
:10AF6000ADF84C0011A91E9814F060FD00BF6D1CD7
:10AF7000BD42A0DBBDF87000ADF80400BDF8740060
:10AF8000ADF80800BDF87200384400B2ADF8060014
:10AF9000BDF87600C01B00B2ADF80A0001A813F09E
:10AFA0008DFE00900098B0B9AEB9BDF8720038447B
:10AFB00000B2ADF80E00BDF87600C01B00B2ADF8CF
:10AFC000120010988DF85C000020149011A91E98B2
:10AFD00014F02CFD38E010988DF85C0001208DF8FD
:10AFE0005400BDF97600A0EB070ABDF97200C5193F
:10AFF00027E0009870B14A4610990B981AF08AFD24
:10B00000BDF968100FFA89F32AB20B9813F006FE07
:10B010008DF8540028B2ADF80E0028B2ADF8120039
:10B02000012E09D1BDF97210691AD8F8080000EB99
:10B0300041000088ADF84C0011A91E9814F0F6FCF0
:10B040006D1C5545D5DD00BF00BF0B9810B10B98A6
:10B050001AF0ACFB0C98401C28B10C9814F08EFA36
:10B0600005A813F007FEB8F1000F02D0404616F015
:10B07000F2FE00BF11E62DE9F04F91B006460C46F6
:10B080001546206910B911B0BDE8F08FA07E0228E6
:10B0900000DCF8E729460FA8B268FAF78CFE00B981
:10B0A000F1E7D6F808800FA8B060206918F0B5FA6B
:10B0B0000746022F55D1002041F6FF71CDE900016E
:10B0C000029003460EA8D4E9041224F057FF284644
:10B0D0000FF012F9824600EBDA70298801EB60006C
:10B0E000BDF9389009EBD971A0EB610000B2ADF861
:10B0F0003000BDF83000BDF838100844401E00B2E2
:10B10000ADF8340028460FF076F8824600EBDA708E
:10B11000698801EB6000BDF93A9009EBD971A0EBA9
:10B12000610000B2ADF83200BDF83200BDF83A104F
:10B130000844401E00B2ADF8360004A813F0D0F960
:10B1400060690490208BADF81C00A07E8DF82A0069
:10B15000002000900CAA04A93046236912F008FED2
:10B16000B0E00EA9206917F02FFE8146B9F1010F5A
:10B170007DD108A812F0DFFDA0788DF82C00208B7F
:10B18000ADF82800E07E8DF82A00A07E8DF82B0017
:10B19000207FE8BB28460FF0AFF8834600EBDB705A
:10B1A000298801EB60000E99C1F38A2A0AEBDA7153
:10B1B000A0EB610000B2ADF8180028460FF01BF8B4
:10B1C000834600EBDB70698801EB60000E994FEA63
:10B1D000515A0AEBDA71A0EB610000B2ADF81A0027
:10B1E000BDF818000E99C1F38A210844401E00B230
:10B1F000ADF81C00BDF81A000E9900EB5150401E2E
:10B2000000B2ADF81E0006AA08A93046236900E086
:10B2100002E012F03FFD51E06888ADF81A00BDF879
:10B220001A000E9900EB5150401E00B2ADF81E00FE
:10B230003DE02888ADF81800BDF818000E99C1F35C
:10B240008A210844401E00B2ADF81C0019E006AA8D
:10B2500008A93046236912F01DFDBDF818000E99AB
:10B26000C1F38A21084400B2ADF8180000E026E0DE
:10B27000BDF81C000E99C1F38A21084400B2ADF854
:10B280001C00BDF91800B5F904108842DFDDBDF8D7
:10B290001A000E9900EB515000B2ADF81A00BDF83B
:10B2A0001E000E9900EB515000B2ADF81E00BDF922
:10B2B0001A00B5F906108842BBDD00BF01E000BFEF
:10B2C00000BF00BFC6F8088000BFDCE62DE9F04FE4
:10B2D00087B083460C46164694F82200022802DC0A
:10B2E00007B0BDE8F08F208C00B9F9E794F823008F
:10B2F000C0F3440000B9F3E794F8230000F0010024
:10B3000000B1EDE730460EF0F7FF814630460EF013
:10B3100072FF0746B4F90050B94501DA484600E02B
:10B3200038468246B5EB6A0F01DD4FEA6A053146C1
:10B3300005A80EF0F5FEBDF9141094F8230040089E
:10B3400000F0040010B1B4F9200003E0B4F92000CB
:10B3500028444042084400B2ADF81400BDF918106A
:10B3600094F82300400800F0080010B1B4F9200060
:10B3700003E0B4F9200028444042081A00B2ADF8B6
:10B380001800BDF9161094F82300400800F00200E0
:10B3900010B1B4F9200003E0B4F920002844404281
:10B3A000084400B2ADF81600BDF91A1094F8230055
:10B3B000C0F3400010B1B4F9200003E0B4F920005C
:10B3C00028444042081A00B2ADF81A00208C281A0E
:10B3D0000FFA80F8B8F1000F01DA4FF00008A078FA
:10B3E00094F82210CDE90210E08BADF804002BB2E6
:10B3F00005AA31465846CDF8008000F002F800BF9B
:10B400006EE72DE9FF4FA3B00D4616461F46329852
:10B41000FF2801DBFF2000E032983290284613F02D
:10B420004DFC2290229868B967B9309850B932988B
:10B43000009032462946319B239800F0A9FA27B0A4
:10B44000BDE8F08F23982946826820A8FAF7B3FC5C
:10B4500000B9F4E720A80EF04FFF81461C2119A87F
:10B460001AF092FB48461AF025F91C904FF0FF3075
:10B470001890002F0ADD00233A46294612A813F03F
:10B4800095FF002112A813F01BF9189001233146F3
:10B490000CA8309A13F08AFF00210CA813F010F9C1
:10B4A0000B9009A819901E90BDF8C400ADF86C006F
:10B4B00032988DF87C0033988DF87D00B5F9000046
:10B4C0003844B6F90010884203DDB5F9000038446D
:10B4D00001E0B6F9000000B2ADF81C00B5F90400B7
:10B4E000C01BB6F90410884203DAB5F90400C01B8A
:10B4F00001E0B6F9040000B2ADF82000B5F9020091
:10B500003844B6F90210884203DDB5F90200384428
:10B5100001E0B6F9020000B2ADF81E00B5F9060070
:10B52000C01BB6F90610884203DAB5F90600C01B45
:10B5300001E0B6F9060000B2ADF8220007A80EF04F
:10B54000DBFE0690B5F90200B6F90210884201DC74
:10B55000012000E000208246B5F90600B6F9061089
:10B56000884201DB012000E0002083462298002869
:10B570004CD0BDF88000ADF82400BDF88400ADF8D3
:10B580002800BDF9824029E0BAF1000F04D1BDF9CD
:10B590001E00A04200DD20E0BBF1000F04D1BDF988
:10B5A0002200A04200DA1DE020B2ADF8260020B251
:10B5B000ADF82A0049461C981AF01DFBBDF9801011
:10B5C0000FFA89F322B21C9813F028FB8DF874004F
:10B5D00019A9239814F02AFA00BF641CBDF986004B
:10B5E000A042D1DA00BF0CA813F044FB0B9813F073
:10B5F000C5FF1898401C28B112A813F03BFB1898FF
:10B6000013F0BCFF1C981AF0D1F818E7B5F9000048
:10B61000B6F90010884201DC012000E0002005900E
:10B62000B5F90400B6F90410884201DB012000E0FE
:10B630000020049001200390059860B1049850B157
:10B64000BAF1000F07D0BBF1000F04D006983228E2
:10B6500001DA0020039001208DF87400BAF1000F88
:10B6600015D0039898B1BDF81C00ADF82400BDF8C2
:10B670002000ADF828006888ADF826007088401ECC
:10B6800000B2ADF82A0019A9239814F0CFF9BBF144
:10B69000000F15D0039898B1BDF81C00ADF8240038
:10B6A000BDF82000ADF82800F088401C00B2ADF8CD
:10B6B0002600E888ADF82A0019A9239814F0B6F9F5
:10B6C000059898B12888ADF824003088401E00B253
:10B6D000ADF82800BDF81E00ADF82600BDF8220028
:10B6E000ADF82A0019A9239814F0A0F9049898B18C
:10B6F000B088401C00B2ADF82400A888ADF828003E
:10B70000BDF81E00ADF82600BDF82200ADF82A00F5
:10B7100019A9239814F08AF90398F0BBBDF88000AA
:10B72000ADF82400BDF88400ADF82800B6F9020099
:10B73000B5F90210401AB84201DA384604E0B6F909
:10B740000200B5F90210401A00B20290002442E053
:10B750006888204400B20190E888001B00B2009085
:10B76000BDF982100198814205DDBDF9861000986F
:10B77000814200DA2EE049461C981AF03CFABDF9E5
:10B7800024100FFA89F3019A1C9813F047FA8DF8E8
:10B790007400BDF98210019800E020E0814209DCCC
:10B7A0000198ADF826000198ADF82A0019A9239850
:10B7B00014F03CF9BDF986100098814209DB00982D
:10B7C000ADF826000098ADF82A0019A9239814F0C6
:10B7D0002DF900BF641C02988442B9DBC7E0BDF8B4
:10B7E0008000ADF82400BDF98410BDF91C00401E96
:10B7F000814202DABDF9840002E0BDF91C00401E5E
:10B8000000B2ADF8280009A80EF076FD8046B8F128
:10B81000000F48DD059810B9BAF1000F1ED0BDF930
:10B82000824017E020B2ADF8260020B2ADF82A0021
:10B8300041461C981AF0DFF9BDF92410434622B2A4
:10B840001C9813F0EBF98DF8740019A9239814F0E3
:10B85000EDF8641CBDF91E00A042E3DC059810B9A8
:10B86000BBF1000F1FD0BDF92200441C17E020B22D
:10B87000ADF8260020B2ADF82A0041461C981AF017
:10B88000BAF9BDF92410434622B21C9813F0C6F948
:10B890008DF8740019A9239814F0C8F8641CBDF938
:10B8A0008600A042E3DABDF98010BDF92000401CFB
:10B8B000814202DDBDF9800002E0BDF92000401C9C
:10B8C00000B2ADF82400BDF88400ADF8280009A846
:10B8D0000EF012FD8046B8F1000F48DD049810B953
:10B8E000BAF1000F1ED0BDF9824017E020B2ADF8CA
:10B8F000260020B2ADF82A0041461C981AF07BF9C8
:10B90000BDF92410434622B21C9813F087F98DF834
:10B91000740019A9239814F089F8641CBDF91E005D
:10B92000A042E3DC049810B9BBF1000F1FD0BDF9B1
:10B930002200441C17E020B2ADF8260020B2ADF87A
:10B940002A0041461C981AF056F9BDF924104346C6
:10B9500022B21C9813F062F98DF8740019A923988B
:10B9600014F064F8641CBDF98600A042E3DA0CA868
:10B9700013F080F90B9813F001FE12A813F07AF976
:10B98000189813F0FBFD1C9819F010FF00BF56E546
:10B990002DE9FF4F89B080460C461546DDF85890DA
:10B9A0001C2168461AF0F0F807A80090BDF8300096
:10B9B000ADF808008DF81890B4F90200B5F902103E
:10B9C000884201DC012000E000200646B4F90600B0
:10B9D000B5F90610884201DB012000E0002007468F
:10B9E000B4F90000B5F90010884201DC012000E044
:10B9F00000208246B4F90400B5F90410884201DB46
:10BA0000012000E0002083462088ADF81C00A088BB
:10BA1000ADF820006088ADF81E006888401E00B2B6
:10BA2000ADF822001EB16946404613F0FFFFE888DA
:10BA3000401C00B2ADF81E00E088ADF822001FB136
:10BA40006946404613F0F2FF2088ADF81C002888B4
:10BA5000401E00B2ADF8200016B1B5F9020001E0B9
:10BA6000B4F90200ADF81E0017B1B5F9060001E007
:10BA7000B4F90600ADF82200BAF1000F03D0694610
:10BA8000404613F0D3FFA888401C00B2ADF81C005C
:10BA9000A088ADF82000BBF1000F03D069464046F6
:10BAA00013F0C4FF0DB0BDE8F08F2DE9FF4F93B048
:10BAB0000746904699464FF6FF70804502D117B071
:10BAC000BDE8F08F3E46746A208C1290208C484569
:10BAD00006D0A4F82090608C20F00400001D608443
:10BAE0004FF4802120461DF008FC11904FF4802176
:10BAF00020461DF069FC0546119815F0D8FE8246D7
:10BB0000384609F0A6FA8346BBF81600ADF83E00A9
:10BB1000BDF93E000AEB050108FB010000B2ADF8DB
:10BB20003E00284605EBD071BDF83E20A2EB610136
:10BB300009B2ADF83E10BDF83E0050442844401E06
:10BB400000B2ADF84200706A808AADF83C00706ABD
:10BB5000008BADF8400001A813F03EFD01AA4FF4A0
:10BB6000802120461EF06EF80FAA01A9149813F048
:10BB700017FD12982084608C20F00400608400BFC0
:10BB80009DE72DE9F04F91B007460D469046994646
:10BB90004FF6FF70804502D111B0BDE8F08F1097CD
:10BBA000109F7C6A208C0F90208C484506D0A4F80A
:10BBB0002090608C20F00400001D608407A812F023
:10BBC0008FFC07AA4FF4802120461DF055FF4FF44B
:10BBD000802120461DF0F8FBADF82E00384609F014
:10BBE00038FA064606B9D7E7079815F060FE824690
:10BBF000F08AADF81600BDF91600BDF92E105144BB
:10BC000008FB010000B2ADF81600BDF92E0000EBF4
:10BC1000D071BDF81620A2EB610109B2ADF8161083
:10BC2000BDF816005044BDF82E100844401E00B266
:10BC3000ADF81A00A08AADF81400208BADF81800FA
:10BC400005AA03A8A968FAF7B6F88346BBF1000F66
:10BC500013D0A868029003A8A860304618F08BFCA7
:10BC600001900020009006F1140207A92846019BCC
:10BC700012F07EF80298A86000BF0F982084608CB4
:10BC800020F00400608400BF86E700002DE9F04149
:10BC900005463F48006811F0F1FC04462868C66B71
:10BCA000706B10B13046716B884739480068006886
:10BCB0000088374909680968498810FB01F0E16884
:10BCC000884201D1012000E000200746206898B199
:10BCD000606888B187B90CE02D4800680068806A08
:10BCE00038B12B4A12681068294A12681268916AA2
:10BCF000884720690028EFD101202061244800688E
:10BD00000068C068806900F0010050B120480068F8
:10BD10000068C0688069C0F3400010B10120606114
:10BD200001E000206061606908B1012000E00020AE
:10BD300080462868406998B12868007CC0F30110EB
:10BD400048B12868007CC0F3800020B1D6E900101B
:10BD500000F020F804E0D6E900212868FDF7F1FAA8
:10BD6000206890B1606880B12868007C00F0010014
:10BD700010B1B8F1000F08D02168A068884202D144
:10BD80006068A06001E02068A060BDE8F08100006C
:10BD9000D40000202DE9F34F83B0044688480068A2
:10BDA0000568874800680068007CC0F3400040B127
:10BDB000287CC0F3800020B100BF00BF05B0BDE803
:10BDC000F08F287CC0F3011002280AD121462846B2
:10BDD000049A00F004F921462846049AFDF7B1FAC6
:10BDE000EBE0287CC0F30110012804D0287CC0F3CC
:10BDF00001100328F4D1002002907148006811F06E
:10BE00003DFC824620460EF054FA064620460EF0CF
:10BE1000DDF983464FF4A050B0FBF6F000B2584570
:10BE200005DA4FF4A050B0FBF6F000B200E058463F
:10BE30000190B4F90280287CC0F3011001280BD1D5
:10BE400068882188401A401E00B2E080E088801B8C
:10BE5000401C00B2608006E020886080608830442A
:10BE6000401E00B2E08000279EE0ABEB0701019886
:10BE7000814201DD019801E0ABEB07000FFA80F988
:10BE80000120CAF8100047BBB34526DBB146297C28
:10BE9000C1F30111032901D1012100E0002108466D
:10BEA0003146049A00F00FF9287CC0F301100128F4
:10BEB00007D1A4F8008008EB0600401E00B2A08065
:10BEC0003FE02888401EA0EB080000B2A080A088B8
:10BED000801B401C00B2208033E0029820B94FF450
:10BEE000205019F0E7FB029002980090297CC1F3E2
:10BEF0000111032901D1012100E0002108464A4631
:10BF00003146049B00F0B2F8287CC0F301100128F0
:10BF10000AD108EB070000B2208008EB0700484474
:10BF2000401E00B2A0800CE02888401EA0EB080054
:10BF3000C01B00B2A080A088A0EB0900401C00B28A
:10BF4000208007EB090058450DDBDAF8180000F0F7
:10BF5000010040B1DAF81800C0F3400018B1012028
:10BF6000CAF8140002E00020CAF81400029808B9C8
:10BF7000049800E00298024621462846FDF7E1F9C0
:10BF800004E0A86A10B12846A96A8847DAF81000C8
:10BF90000028F6D106FB09F1049800EB410004905B
:10BFA00007EB090007B200BF5F45FFF65EAF0298DE
:10BFB00010B1029819F0FAFB00BF00BFFEE60000C6
:10BFC000D400002018B5048800940C8804801488DC
:10BFD0000C801C881480BDF800401C8018BD2DE921
:10BFE000FC5F05460C46164620460EF062F9824676
:10BFF00020460EF0EBF883461AFB0BF001900198F7
:10C00000471E4FF0000811E006EB47000088009043
:10C0100006EB470006EB48010988018006EB480063
:10C02000BDF8001001807F1E08F101084745EBD8DC
:10C03000B4F9069068886188401A401E00B2E0801A
:10C040006888A0EB0900401E00B26080B4F904903B
:10C0500028882188401A401E00B2A0802888A0EBC2
:10C060000900401E00B22080BDE8FC9F2DE9F0478A
:10C0700004461D46089F01FB02F0A0F1010C481E7A
:10C0800000FB02F800231AE008EB03000CB1ACEB54
:10C09000000000260FE0A946AD1C07EB400AB9F8E6
:10C0A0000090AAF800900CB1104400E0801A06F14C
:10C0B00001090FFA89F68E42EDDB581C03B2934258
:10C0C000E2DBBDE8F0872DE9F04782460C461546D5
:10C0D00000263BE0002731E0601E801B0FFA80F84D
:10C0E000601EC01B0FFA80F9BAF1000F12D007FBD7
:10C0F000048C05EB4C0308FB049C05EB4C0209FB8C
:10C10000046C05EB4C0106FB047C05EB4C00FFF7CF
:10C1100059FF11E009FB046C05EB4C0308FB049C80
:10C1200005EB4C0207FB048C05EB4C0106FB047C81
:10C1300005EB4C00FFF746FF781C07B2601C00EBD4
:10C14000D071B7EB610FC7DB701C06B204EBD47182
:10C15000B6EB610FBEDBBDE8F08710B504462046A4
:10C1600016F006FE10BD00002DE9F14F9EB01E989E
:10C1700015F0FEF905462C461E9815F0A0F91D9005
:10C18000606A18F0F8F907465420005D00F00100DD
:10C1900010B91FB0BDE8F08F0FA813F01DFA0FAA59
:10C1A0004FF4E02128461DF04DFD04F148010DA893
:10C1B0000DF0F5FFBDF83400616A898A084400B2C9
:10C1C000ADF83400BDF83610606AC08A084400B289
:10C1D000ADF83600BDF83800616A898A084400B2BB
:10C1E000ADF83800BDF83A10606AC08A084400B261
:10C1F000ADF83A000DAA0FA91D9813F0D1F94FF42C
:10C20000E02128461CF0DDFB06464FF4E0212846DD
:10C210001CF034FE30440FFA80F84FF4E021284639
:10C220001CF088FF30440FFA80F900200B900C902E
:10C23000216DC8191F49096888478246206DC119B8
:10C2400052460BA819F01EFBBDF83400404400B262
:10C25000ADF83400BDF83600484400B2ADF8360001
:10C260004FF0000BD4F824A05522594650461CF03C
:10C270006DFF019001980A9002A812F031F902AA0C
:10C280004FF4E02128461DF0F7FB9DF83F000228FF
:10C2900005DCBDF81400BDF82810884207D0002046
:10C2A0000BAB0DAA02A900901D9811F061FD00BF13
:10C2B0006FE700006C0200202DE9F04FBDB005468D
:10C2C0000E4600BF00BFAB460BF13000FAF739FD58
:10C2D00010B13DB0BDE8F08F05F114023BA8B16884
:10C2E000F9F769FD00B9F4E7B0683A903BA8B0608F
:10C2F00035A812F0B8F935AA4FF4E02128461DF010
:10C3000023FC27A813F068F99DF8DC008DF89F0046
:10C3100047F6FF70ADF89C004FF4E02128461DF071
:10C32000FBF8074600EBD7704FEA60094FF4E021B5
:10C3300028461DF0F1F8074600EBD7704FEA600A77
:10C34000314604A81BF06CF824A80A9016A808909F
:10C350004FF4E02011906F480590052006900BF1F6
:10C360003000FAF766FC0446CCE00A2235A924A87E
:10C3700019F088FA382227A916A819F083FAE0885C
:10C38000ADF89000E088ADF85C0039A80D9038A8B1
:10C390000E90607B00F0010020B1B4F90070B4F998
:10C3A000028012E0B4F9040047F6FF71884200D120
:10C3B000A2E0A08882B26B462846A1680FF000FC7C
:10C3C000BDF90070BDF9028000BFA88A384407B2E9
:10C3D000E88A40440FFA80F8B9F1000F04D0BAF1AE
:10C3E000000F01D0012000E0002001900198B0B1C1
:10C3F000A7EB090000B2ADF8080007EB090000B296
:10C40000ADF80C00A8EB0A0000B2ADF80A0008EB8A
:10C410000A0000B2ADF80E0002A8079001E000206B
:10C420000790207B00F0030080B3207B00F0010028
:10C4300010B1B5F9140000E03846ADF8E400ADF8ED
:10C44000E680207B00F0020010B1B5F9180000E092
:10C450003846ADF8E000BDF8E600ADF8E20004AA09
:10C460001A21284615F08AF838AB39AA24A9304693
:10C4700012F0E2F8019820B102AA16A9304613F092
:10C480008FF804AA1B21284615F078F8207B00F0CD
:10C490000C0080B3ADF8E470207B00F0040010B114
:10C4A000B5F9160000E04046ADF8E600BDF8E4003E
:10C4B000ADF8E000207B00F0080010B1B5F91A00DB
:10C4C00000E04046ADF8E20004AA1A21284615F023
:10C4D00055F838AB39AA24A9304612F0ADF80198C6
:10C4E00020B102AA16A9304613F05AF804AA1B215B
:10C4F000284615F043F800BF21460BF13000FAF74B
:10C5000092FB0446002C7FF430AF3A98B06000BF35
:10C51000DFE6000094C303082DE9F14F9AB01A98A2
:10C5200015F026F804461A9814F0C9FF1990204611
:10C530001DF01FF9074620461BF0C8FA834607EB9B
:10C54000D771A28A02EB610109B218910BEBDB7182
:10C550004A10E18A114409B2179107EBD7714E10C6
:10C5600014A812F080F814AA002120461DF0ECFA5D
:10C570004FF41D7016FB00F0552190FBF1F0642183
:10C5800090FBF1F000B2ADF85200BDF85200801CF3
:10C5900000B2ADF8520000201390002120461CF09C
:10C5A00030F90546002347F6FF7204F114010DA887
:10C5B00012F0FCFE00210DA812F082F80C9000BFD2
:10C5C000A08AADF82800E08AADF82A00208BADF8EB
:10C5D0002C00608BADF82E0000BFBDF82800284469
:10C5E00000B2ADF82800BDF82C00401B00B2ADF839
:10C5F0002C00BDF82A00284400B2ADF82A00BDF88E
:10C600002E00401B00B2ADF82E00012347F6FF724A
:10C610000AA904A812F0CAFE002104A812F050F8DA
:10C620000390BDF952804FF0000A4FE0514620467A
:10C63000FBF7ACFA0090BDF80000ADF8500013987D
:10C64000C0F30F290FFA89F023F0AAFB06EB0801CB
:10C650004843189901EBE03000B2ADF804000FFA3E
:10C6600089F023F08CFB06EB08014843179901EB96
:10C67000E03000B2ADF806000FFA89F023F090FB2D
:10C68000711BA1EB08014843189901EBE03000B29F
:10C69000ADF808000FFA89F023F071FB711BA1EBD4
:10C6A00008014843179901EBE03001B2ADF80A10D8
:10C6B00002AB01AA14A9199811F0BEFF0AF10300F8
:10C6C0001FFA80FA139800F587601390BAF5807FFF
:10C6D000ACDD0DA812F0CEFA04A812F0CBFA0C983B
:10C6E00012F04CFF039812F049FF1BB0BDE8F08F29
:10C6F0002DE9F04FA5B004460F46254604F114017C
:10C7000023A8BA68F9F757FB2290229810B925B0F0
:10C71000BDE8F08FB868219023A8B86000212046BA
:10C720001CF02BF91E90002120461CF03BFB01461B
:10C730001E98084400B21D90002120461CF082FC87
:10C7400001461E98084400B21C9020461BF048F990
:10C750007E35E9884843001200B21B9020461BF04A
:10C7600020F929894843001200B21A9017A811F045
:10C770007AFF17AA002120461DF0E6F9394605A8E0
:10C780001AF04EFE002012908C4806900020079070
:10C7900017A80B904FF0FF30139000200E900F90D1
:10C7A00005AA1A21204614F0E9FE0020019031224A
:10C7B000204601991CF0CAFC0090009800F0FF0B85
:10C7C00000BF002120461CF0D8F804900020019002
:10C7D0003322204601991CF0B9FC0090009800F02B
:10C7E000FF0800BF20461BF067FA039020461BF0AD
:10C7F0005DFB029035F87E09002865D0E18A1C981F
:10C8000001440298081A00B20190A08AADF8800095
:10C81000208BADF87C004FF00009B5F87E000FFAD0
:10C8200080FABBF1020F1ADD0498002817DD08F02A
:10C83000020040B1002120461CF004FC18B909F1A7
:10C8400001000FFA80F908F0010040B100212046F4
:10C850001CF0DCF918B9AAF101000FFA80FA4E4673
:10C860002FE01A987043B5F87E10491E90FBF1F046
:10C8700000B2ADF88200BDF882100198084400B201
:10C88000ADF88200BDF88200ADF87E004B480690FE
:10C890000120079020A80E901FA80F90139605AABC
:10C8A0001A21204614F06AFE1FAB20AA17A93846A9
:10C8B00011F0C2FE05AA1B21204614F05FFE701C79
:10C8C00006B25645CDDB00BFB5F88000002865D024
:10C8D000A18A1D9801440398081A00B20190E08AC9
:10C8E000ADF88200608BADF87E004FF00009B5F81E
:10C8F00080000FFA80FABBF1020F1ADD04980028BD
:10C9000017DD08F0040040B1002120461CF04AFA6F
:10C9100018B909F101000FFA80F908F0080040B1D8
:10C92000002120461CF0DAFA18B9AAF101000FFA2A
:10C9300080FA4E462FE01B987043B5F88010491ED0
:10C9400090FBF1F000B2ADF88000BDF880100198C6
:10C95000084400B2ADF88000BDF88000ADF87C005E
:10C96000164806900220079020A80E901FA80F904E
:10C97000139605AA1A21204614F000FE1FAB20AA28
:10C9800017A9384611F058FE05AA1B21204614F0BD
:10C99000F5FD701C06B25645CDDB00BF4FF0FF30F1
:10C9A000139000200E900F9005AA1B21204614F032
:10C9B000E5FD2198B86000BFA9E6000094C3030814
:10C9C0002DE9F14F9AB01A9814F071FD07461A98A4
:10C9D00014F0CEFD05462C46122F7DD11A9814F086
:10C9E000C4FD06463078022802D11BB0BDE8F08FA6
:10C9F00094F8380000F00300032805D094F83800BC
:10CA000000F00300022802D101203070EDE794F815
:10CA10003800C0F38400042808D094F83800C0F32C
:10CA20008400012802D001203070DEE74FF00008BA
:10CA30004622414628461CF089FB19901998C0B23D
:10CA4000FF2802D001203070CFE7208E10B10120E6
:10CA50003070CAE71A9814F088FD8146E08EB0F570
:10CA6000807F09D1002205F114014846F9F7E4F965
:10CA700098BB01203070B8E728461BF027F88046A5
:10CA800028461CF076FE824604F13200E18E002337
:10CA90004246CDE90010514618A8F9F78DFCBDF8C3
:10CAA0006000A98A084400B2ADF86000BDF86210C9
:10CAB000E88A084400B2ADF86200BDF86400A98AB3
:10CAC000084400B2ADF86400BDF86610E88A084476
:10CAD00000B2ADF8660001E00BE009E0002218A901
:10CAE0004846F9F7A9F910B9012030707DE700BF79
:10CAF00010E2152F01D0182FFAD128461CF039FE6C
:10CB0000199028461AF0E2FF18900026322231468A
:10CB100028461CF01BFB1090109800B2804600BF06
:10CB20001222314628461CF011FB10901098404408
:10CB30000FFA80F900BF1322314628461CF006FB8D
:10CB400010901098404400B2179000BF1022314658
:10CB500028461CF0FBFA1090109840440FFA80FA17
:10CB600000BF1122314628461CF0F0FA10901098B0
:10CB7000404400B21690608E484400B2ADF85400B4
:10CB8000A08E504400B2ADF8560094F8390000F081
:10CB90000300012804D113A928461AF040FF26E01B
:10CBA00015A9E08ECDE90001208E03B213A8DDE9BE
:10CBB0001821F9F701FCBDF84C00A98A084400B21D
:10CBC000ADF84C00BDF84E10E88A084400B2ADF84C
:10CBD0004E00BDF85000A98A084400B2ADF85000DC
:10CBE000BDF85210E88A084400B2ADF8520005F1D1
:10CBF000140111A80DF0C1FA13A905F114000DF0EC
:10CC0000BCFAC5481A991AF026FE8346BBF1010FFB
:10CC100000D0EAE611A905F114000DF0AEFA152FC7
:10CC20007DD1E08D08B1A08D00B9DEE6E08E00B9BF
:10CC3000DBE61A9814F043FC064605F114010FA830
:10CC40000DF09BFA284616F0D5FA0E9094F83900AC
:10CC500000F0030001283CD1B4F92C10BDF93820B4
:10CC6000891A481C00EBD071BDF83C20A2EB610191
:10CC700009B2ADF83C10B4F92C10BDF93820891A6E
:10CC8000481C00EBD071BDF84020A2EB610109B255
:10CC9000ADF84010B4F92E10BDF93A20891A481C9D
:10CCA00000EBD071BDF83E20A2EB610109B2ADF8F6
:10CCB0003E10B4F92E10BDF93A20891A481C00EB39
:10CCC000D071BDF84220A2EB610109B2ADF842106B
:10CCD00013E013A80DF04FFBBDF83C100844401EB4
:10CCE00000B2ADF8400013A80DF0B6FABDF83E1042
:10CCF0000844401E00B2ADF84200BDF83C00484474
:10CD000000B2ADF83C00BDF83E00504400B2ADF8B2
:10CD10003E00BDF840101798081A00B200E0F8E095
:10CD2000ADF84000BDF842101698081A00B2ADF8F0
:10CD3000420094F8380000F00300012805D094F870
:10CD4000380000F0030000287ED108A810F0F3FF9F
:10CD500008AA002128461CF027FEE08EADF822002C
:10CD6000208E00B2ADF82000608EADF82400A18EB8
:10CD7000ADF8261094F83800C0098DF83400BDF8DD
:10CD80004C00484400B2ADF81800BDF84E005044C5
:10CD900000B2ADF81A00BDF850101798081A00B28A
:10CDA000ADF81C00BDF852101698081A00B2ADF884
:10CDB0001E00B068059006AA06A8B168F8F7FBFF48
:10CDC00000B912E606A8B060B4F92800B4F92C1036
:10CDD00090FBF1F201FB12000290B4F92A00B4F9C1
:10CDE0002E1090FBF1F201FB12000190BDF83E10F5
:10CDF0000198084400B2ADF80E00BDF90E00BDF96F
:10CE00003E10884206DDBDF80E00E18D401A00B2EA
:10CE1000ADF80E00BDF80E00E18D0844401E00B2D2
:10CE2000ADF812004AE0BDF83C100298084400B288
:10CE3000ADF80C00BDF90C00BDF93C10884208DDCE
:10CE4000BDF80C00A18D00E041E0401A00B2ADF841
:10CE50000C00BDF80C00A18D0844401E00B2ADF8D6
:10CE6000100015E003AA08A93046636A10F012FF0B
:10CE7000BDF80C00BDF83810084400B2ADF80C0045
:10CE8000BDF81000BDF83810084400B2ADF810002D
:10CE9000BDF90C00BDF940108842E3DBBDF80E007F
:10CEA000BDF83A10084400B2ADF80E00BDF812000B
:10CEB000BDF83A10084400B2ADF81200BDF90E00FA
:10CEC000BDF942108842AEDB0598B06020E094F8CE
:10CED000380000F00300022811D106A811F000FB71
:10CEE00006AA002128461CF0C7FD0020009005F18D
:10CEF000140206A93046636A10F03AFF08E000BF4A
:10CF000000BF002305F114021946304610F0C2FE9E
:10CF100000BF00BF00BF68E5980204082DE9F14F8B
:10CF2000DCB05C9814F024FB05462C465C9814F0A9
:10CF3000C6FA5B9059A928461AF071FD0020CDE988
:10CF400010506922DDE910011CF000F90F900F98D4
:10CF500000B258900020CDE910506A22DDE910019E
:10CF60001CF0F4F80F900F9800B25790BDF86411C0
:10CF70005898081A00B2ADF86401BDF868115898C5
:10CF8000084400B2ADF86801BDF866115798081A58
:10CF900000B2ADF86601BDF86A115798084400B2B6
:10CFA000ADF86A0159A80DF0D8F9834659A80DF0DB
:10CFB00045F95690D4E90A10A0EB0109569883452B
:10CFC00001DB012000E0002080460020559094F80D
:10CFD0005C0000F0030001280BD1A06A002808DAE9
:10CFE000E06A002805DDA16A206B884201D101209A
:10CFF0005590002128461BF0F9FE54900021284648
:10D000001BF090FF5390002128461CF03FF85290EF
:10D01000002128461BF01EFE519059A904F134004E
:10D020000DF099F8A18E5498084400B2A086218F83
:10D030005398081A01B22187E18E5298084401B230
:10D04000E186618F5198081A01B26187B8F1000F2B
:10D0500013D004F134000DF0F1F804280DDA5698DD
:10D0600000EBD0714A10E98A1144891E0AB2E286A7
:10D07000E08E001D01B2618715E0B8F1000F12D1FA
:10D0800004F134000DF069F904280CDA58460BEB72
:10D09000D071AA8A02EB6101891E09B2A186A08E15
:10D0A000001D01B2218704F134000DF056F95090B3
:10D0B00004F134000DF0C2F84F90B8F1000F01D028
:10D0C000509800E04F988246B8F1000F05D004F167
:10D0D0003406371DFE484C9004E004F13606371D37
:10D0E000FC484C90A06D401CF8B1A36A216DC91A90
:10D0F00001FB0AF191FBF9F108B2A36A616DC91A4B
:10D1000001FB0AF191FBF9F10AB2131AD4F858C0E5
:10D1100003FB0CF1CB1701EB13631B121BB24D93F6
:10D120004D99014409B24D9108E0A16A206B401A63
:10D1300000FB0AF090FBF9F000B24D90A06C401C8F
:10D14000E0B1A36A216CC91A01FB0AF191FBF9F164
:10D1500008B2A36A616CC91A01FB0AF191FBF9F1EB
:10D160000AB2131AD4F848C003FB0CF1CB1701EB39
:10D17000136300EB23231BB24E9308E0D4E90901AB
:10D18000401A00FB0AF090FBF9F000B24E9000202C
:10D1900011901622284611991BF0D8FF1090109874
:10D1A000C0B24B90B8F1000F0ED04B9801280BD1B4
:10D1B00030463E4607464E99494209B24E914D9936
:10D1C000494209B24D9100BFB8F1000F0AD0318831
:10D1D0004E98084400B2388031884D98084400B217
:10D1E00030800AE039884E98081A401C00B230801E
:10D1F00039884D98081A00B23880559878B3A26AD9
:10D20000524202FB0AF292FBF9F211B2B8F1000F9E
:10D210000CD032880A4410B2B7F90020824201DDF6
:10D2200030801BE03A883280388017E03A88521A02
:10D23000521C10B2B6F90020824201DD388002E0B3
:10D2400032883A803080B7F90020B6F900309A422F
:10D2500004DAB6F900003A883280388000BF559869
:10D2600000BB04F134004C99884701281ADC684659
:10D270005B991AF0D5F84FF400300D909648019064
:10D280000020029004F1340003906A461A212846D7
:10D2900014F074F96A461B21284614F06FF95DB04A
:10D2A000BDE8F08F04F1340149A80CF054FF3BA80D
:10D2B00012F092F93BAA4FF4003128461CF0C2FC50
:10D2C00029A85B991AF0ACF84FF4003036908248E8
:10D2D0002A9000202B903BA82D9004F134002C9034
:10D2E00029AA1A21284614F049F9002011900B228E
:10D2F000284611991BF02AFF1090109800B2289030
:10D300005698834501DA584600E056982790DDE9A3
:10D310002701B1EB600F02DD279840102890BDF97E
:10D32000EC0026904F995098884201DA509800E01E
:10D330004F982790DDE92601B0EB610F02DD2798B9
:10D3400040102690B8F1000F08D004F134000DF021
:10D3500004F801462698B1EB400F0BDCB8F1000F42
:10D3600028D104F134000CF069FF01462698B1EB96
:10D37000400F1FDD9DF8EF0011909DF80601109001
:10D380009DF80E010F9000208DF8EF008DF806013A
:10D390008DF80E0104F134023BA95B9812F000F9FC
:10D3A00011988DF8EF0010988DF806010F988DF800
:10D3B0000E0100BFA98A5498084400B2ADF8780065
:10D3C000298B5398081A00B2ADF87C00E98A52986C
:10D3D000084400B2ADF87A00698B5198081A00B27F
:10D3E000ADF87E0000231EA920A8289A11F0DEFFC8
:10D3F000002120A811F064F91D909DF822011C90D5
:10D400009DF80E011B9000208DF80E018DF8220171
:10D4100059A919A80CF09FFEBDF86410549808444F
:10D4200000B2ADF86400BDF866105298084400B22E
:10D43000ADF86600BDF868105398081A00B2ADF850
:10D440006800BDF86A105198081A00B2ADF86A0079
:10D45000B8F1000F15D019A80CF0F0FE042810DA6E
:10D46000569800EBD0714A10E98A1144891E09B21E
:10D47000ADF86610BDF86600001D00B2ADF86A0098
:10D4800017E0B8F1000F14D119A80CF066FF0428BA
:10D490000FDA58460BEBD071AA8A02EB6101891EA4
:10D4A00009B2ADF86410BDF86400001D00B2ADF81B
:10D4B0006800BDF9EC20002304F1340113A811F039
:10D4C00075FF002113A811F0FBF8129019AA05E0CE
:10D4D0005BA301083DA20108F00104083BA95B9889
:10D4E00012F05EF81B988DF80E011C988DF8220141
:10D4F00000208DF8EF008DF806018DF8220104F16F
:10D5000034023BA95B9812F04BF813A811F0B2FB60
:10D5100020A811F0AFFB129812F030F81D9812F00D
:10D520002DF829AA1B21284614F028F800BFB6E6DA
:10D53000F0B591B00546284614F01AF8044628467E
:10D5400013F0BDFF0746264603A812F045F803AACC
:10D550004FF4403120461CF075FB47F6FF70ADF8E4
:10D560000C002C20805D00F0010038B120460FF047
:10D57000C8FE0090BDF80000ADF81000214601A8DB
:10D5800007F0B4FC01AA03A9384612F009F811B05B
:10D59000F0BD00002DE9F04FB1B08146484613F0D0
:10D5A000E7FF07463C46484613F089FF83460021C3
:10D5B00038461BF07AF9012800D100E000208046AF
:10D5C00038460AF046FE0546002694F85C0000F056
:10D5D0000300012806D1A06A002803DAE06A0028C7
:10D5E00000DD0126B5B138461AF070FA824636B130
:10D5F000606A002803DAA08EADF8BC0019E0B8F12B
:10D60000000F02D0B4F9340001E0B4F93800ADF8ED
:10D61000BC000EE038461CF0ACF8824636B1606AB9
:10D62000002803DA608FADF8BE0002E0E08EADF8AE
:10D63000BE0021A811F0D0FF21AA4FF44031384696
:10D640001CF000FB2B4652462FA9384623F049FF19
:10D650002FA904F168000CF099FD59460FA819F0A4
:10D66000DFFE4FF440301C9038481090002011909D
:10D670001D9004F16800129021A8139038461FF005
:10D680007DFE022810D00FAA1A21384613F076FF2B
:10D6900004F1680221A9584611F082FF0FAA1B214C
:10D6A000384613F06BFF4DE0382221A901A818F08D
:10D6B000E9F80FAA1A21384613F060FF04F1680256
:10D6C00021A9584611F06CFF0FAA1B21384613F010
:10D6D00055FF55B1B8F1000F02D1B4F9340001E0A3
:10D6E000B4F93800ADF8BC0002E0608FADF8BE00C0
:10D6F0002B4652462FA9384623F0F3FE2FA904F1FA
:10D7000060000CF043FD382201A921A818F0BAF8F6
:10D710000120119004F16000129021A813900120C3
:10D720001D900FAA1A21384613F028FF04F1600259
:10D7300021A9584611F034FF0FAA1B21384613F0D7
:10D740001DFF00BF31B0BDE8F08F000024030408C6
:10D750002DE9F04790B08046404613F009FF05469A
:10D7600028461AF003FA064608A810F0B9FE08AADF
:10D77000002130461CF080F9284616F0F3FE28B14F
:10D780009DF83D0040F001008DF83D00404613F04B
:10D7900096FE0446A76806F1140206A8A168F8F7E9
:10D7A0000AFB10B910B0BDE8F08706A8A06004A974
:10D7B000304608F06BF9A88AADF80800E88AADF8A1
:10D7C0000A00288BADF80C00BDF81200ADF80E0071
:10D7D00002AA02A8A168F8F7EEFA98B1D4F8089066
:10D7E00002A8A060284616F0C6FE824600205346D6
:10D7F00005F1140208A90090204610F0B9FAC4F807
:10D80000089000BFA88AADF80800BDF81600ADF872
:10D810000A00288BADF80C00688BADF80E0002AA48
:10D8200002A8A168F8F7C7FA98B1D4F8089002A83E
:10D83000A060284616F09FFE82460020534605F160
:10D84000140208A90090204610F092FAC4F808903B
:10D8500000BFA76000BFA5E72DE9FF4FA1B00646B6
:10D8600014462498807B00F00F052298807E1F903C
:10D87000032D00D10425012D06D0022D0BD0042D3F
:10D8800010D0082D1DD114E0DFF86C834FF0800A12
:10D8900002201E901AE0DFF864834FF0C00A0420D3
:10D8A0001E9013E0DFF858834FF0F00A10201E900E
:10D8B0000CE0DFF850834FF0FF0A4FF480701E90A9
:10D8C00004E000BF00BF25B0BDE8F08F00BF1F9887
:10D8D000FD2823DACC4801781F98814203D1CB4838
:10D8E0000068A84213D000200DE018F80010FF29AE
:10D8F00001D11F9904E018F800101F9A5143091232
:10D90000C34A1154401C1E998842EED300BFDFF871
:10D910000083BD491F980870BC4805602498B0F882
:10D9200006B0249800891B900BFB05F01A90B4F9FF
:10D930000000B168B1F90010884201DB002005E069
:10D94000B068B0F90000B4F90010401A1990B4F9A9
:10D9500000005844B168B1F90410884201DC58460F
:10D9600006E0B068B0F90400B4F90010401A401C99
:10D970001890B4F90200B168B1F90210884201DBD5
:10D98000002005E0B068B0F90200B4F90210401AB6
:10D990001790B4F902101B980844B168B1F9061049
:10D9A000884201DC1B9806E0B068B0F90600B4F9C3
:10D9B0000210401A401C16901A991798484319995A
:10D9C00001FB050015902E99159801EBD0002E90C3
:10D9D000159800F007071C210DA818F0D5F822981B
:10D9E0008089ADF83C002298807E8DF84C0022980A
:10D9F000807FC0F3C2008DF84D00F9F7A9FC0190BB
:10DA00000FF040FE0C901B980BFB00F10C9881422C
:10DA100001DD0C9802E01B990BFB01F00B900B98B9
:10DA200017F048FE8146CDF8409000200A902188EA
:10DA30001998084400B2ADF82000218818980844CD
:10DA4000401E00B2ADF8240061881798084400B267
:10DA5000ADF82200BDF82200ADF8260000BFBDF8E9
:10DA60002400BDF82010401A401C00B2079000BFEF
:10DA7000BDF82000ADF81400BDF82200ADF8160086
:10DA8000BDF82400ADF81800BDF82600ADF81A0066
:10DA900000BFBDF816101698084400B2ADF81A0081
:10DAA00005A811F00BF9049008A80D901290C5F18B
:10DAB0000800039019980BEB00011898081A6843A6
:10DAC000029017981C9078E00A9801902AFA07F0C3
:10DAD000209019981D9028E02E98007820990840F1
:10DAE0000399C91BC8401490149830B1149818F8C1
:10DAF00000100A9809F8001003E000210A9809F8BC
:10DB000000100398874204D22F442098E8402090C8
:10DB100005E00027CDF880A02E98401C2E900A9892
:10DB2000401C0A901D98401C1D9018991D98884211
:10DB3000D2DB0498A0B1BDF92620BDF92010019BCD
:10DB400009EB0300079B11F069F88DF844009DF87C
:10DB5000440028B9019909EB0100079918F014F85D
:10DB6000DDE91801411A0A9801440B98814206D256
:10DB7000BDF82600401C00B2ADF8260012E00220DD
:10DB80008DF844000DA9304611F050FFBDF8260075
:10DB9000401C00B2ADF82200BDF82200ADF826000E
:10DBA00000200A90029807442E9800EBD7002E9090
:10DBB00007F007071C98401C1C9016991C98884277
:10DBC00082DBBDF92200BDF9261088420ED0BDF8D7
:10DBD0002600401E00B2ADF8260002208DF8440059
:10DBE0000DA9304611F022FF00200A90484617F098
:10DBF000DDFD00BF67E60000E0C10308E2C10308E5
:10DC0000EEC10308FEC10308E4000020E800002084
:10DC1000883300202DE9FF4F8FB00C4615461E4675
:10DC2000B4F90200401E0E900E9840100D900E9810
:10DC300000F001010D9808440C90B5F90000B6F908
:10DC40000010884202DAB5F9000001E0B6F90000E0
:10DC5000ADF82800B5F90000B6F90010884202DDE1
:10DC6000B5F9000001E0B6F90000401E00B2ADF8C1
:10DC70002C0069880C98081A00B2ADF82A0069884F
:10DC80000D98084400B2ADF82E000F980AA98268DA
:10DC90000AA8F8F790F88246BAF1000F02D113B043
:10DCA000BDE8F08FE08818B1A08808B1012000E03D
:10DCB00000208346012009900AA810F0FFFF10B150
:10DCC0000020099004E0BBF1000F01D00020099072
:10DCD0001C2102A817F058FF0AA802902088ADF86E
:10DCE0001000207A8DF82000099820B102A90F9821
:10DCF00011F09CFE78E00AA80CF0F7FA0746BDF98F
:10DD00002E000190BDF82A00ADF82E0000200090F2
:10DD1000BBF1000F0BD0B4F90600B4F904100844AD
:10DD2000BDF9281091FBF0F200FB1210009038466C
:10DD300017F0C0FC8046CDF814800AA80790BDF902
:10DD40002A904AE03946404617F055FFBDF92810A1
:10DD50003BB20FFA89F2404610F060FF8DF81800D0
:10DD6000BBF1000F27D09DF8180020B300980021C8
:10DD70001BE0B4F90420824207DBA3881B1A1AB205
:10DD80008B1819B2831818B20BE0B4F90620B4F955
:10DD900004301A44824201DC002002E0002208F82C
:10DDA00001204A1C11B2421C10B2B942E1DB02222E
:10DDB0008DF8182000BF02A90F9811F037FEBDF8AA
:10DDC0002A00401C00B2ADF82A00BDF82E00401C0D
:10DDD00000B2ADF82E0009F1010901988145B1DDCD
:10DDE000404617F0E3FC00BF00BF58E72DE9FF4FA6
:10DDF000C7B08B4691469A46B9F90200BAF90210AB
:10DE0000884210DAB9F80200ADF81A01BAF8020037
:10DE1000ADF81601B9F80000ADF81801BAF8000025
:10DE2000ADF814010FE0BAF80200ADF81A01B9F824
:10DE30000200ADF81601BAF80000ADF81801B9F803
:10DE40000000ADF81401BDF91401BDF91811441A10
:10DE5000BDF91601BDF91A11451A002C01DD204645
:10DE600000E06042002D01DD294600E06942884261
:10DE700001DD012000E000204490BBF90260002099
:10DE80004390449870B1002D01DD284600E06842BF
:10DE90004101002C01DD204600E0604291FBF0F0E2
:10DEA00043900DE0002C01DD204600E0604241017E
:10DEB000002D01DD284600E0684291FBF0F0439020
:10DEC000E0494398085C70433F30C611771006F074
:10DED000010000EB0708BDF91801BDF914118842D3
:10DEE00002DABDF9180101E0BDF91401801B00B28E
:10DEF000ADF80401BDF91801BDF91411884202DD25
:10DF0000BDF9180101E0BDF91401304400B2ADF8CB
:10DF10000801BDF91A01BDF91611884202DABDF9EE
:10DF20001A0101E0BDF91601801B00B2ADF806012F
:10DF3000BDF91A01BDF91611884202DDBDF91A01B9
:10DF400001E0BDF91601304400B2ADF80A0147986E
:10DF500041A9826841A8F7F72EFF4090409810B978
:10DF60004BB0BDE8F08F4498F0B3002C24DD0021C5
:10DF7000BDF81601C01B00B2CDE90001BDF9143196
:10DF8000BDF81A01C01B02B2BDF9181135A810F076
:10DF90008FFF0121BDF81601404400B2CDE9000118
:10DFA000BDF91431BDF81A01404402B2BDF918118F
:10DFB0002AA810F07DFF4AE00021BDF81601404478
:10DFC00000B2CDE90001BDF91431BDF81A01404499
:10DFD00002B2BDF9181135A810F06AFF0121BDF891
:10DFE0001601C01B00B200E00DE0CDE90001BDF953
:10DFF0001431BDF81A01C01B02B2BDF918112AA8CC
:10E0000010F056FF23E00021BDF91601CDE9000113
:10E01000BDF81401404403B2BDF91A21BDF818013E
:10E02000404401B235A810F043FF0121BDF91601AB
:10E03000CDE90001BDF81401C01B03B2BDF91A21DE
:10E04000BDF81801C01B01B22AA810F031FF002151
:10E0500035A810F035FB139000212AA810F030FBF2
:10E0600012904FF0FF30119010909BF80900C0F310
:10E07000001068BB0321BDF81A01204400B2CDE9AD
:10E080000001BDF81801401B03B2BDF91A21BDF90A
:10E0900018111FA810F00CFF0221BDF81601204432
:10E0A00000B2CDE90001BDF81401401B03B2BDF977
:10E0B0001621BDF9141114A810F0FAFE00211FA8B2
:10E0C00010F0FEFA1190002114A810F0F9FA109047
:10E0D00041A80CF00AF90F90F9F73AF901900FF006
:10E0E000D1FA0D9041A80CF0C5F801460D98814277
:10E0F00003D241A80CF0BEF800E00D980C900C98EB
:10E1000017F0D8FA0B90BDF90A010A90BDF8060184
:10E11000ADF80A0100200990DDE90B0117F06BFD55
:10E120001C2102A817F030FD41A80290BBF80000A6
:10E13000ADF810009BF808008DF820000B980590B2
:10E1400041A80790BDF906010E9040E0BDF9041109
:10E15000099B0B9AD0180F9A13B20E9A12B210F0B4
:10E160005DFD8DF818009DF8180028B9099A0B99E3
:10E1700088180F9917F008FD0F990998084409901D
:10E180000F99099801440C98814206D2BDF80A0102
:10E19000401C00B2ADF80A0116E002208DF818000C
:10E1A00002A9479811F042FCBDF80A01401C00B2D8
:10E1B000ADF80601BDF80601ADF80A01002009908E
:10E1C000DDE90B0117F017FD0E98401C0E900A991F
:10E1D0000E988842BADDBDF90601BDF90A118842E0
:10E1E0000CD0BDF80A01401E00B2ADF80A010220B1
:10E1F0008DF8180002A9479811F018FC0B9817F039
:10E20000D5FA35A810F036FD2AA810F033FD119884
:10E21000401C10B11FA810F02DFD1098401C10B12B
:10E2200014A810F027FD139811F0A8F9129811F016
:10E23000A5F9119811F0A2F9109811F09FF900BFFB
:10E240008EE60000FEC203082DE9FF4F91B00C4698
:10E2500015461E46B4F90200401E1090109840105A
:10E260000F90109800F001010F9808440E90298833
:10E270000E98081A00B2ADF8300029880F980844AB
:10E2800000B2ADF83400B5F90200B6F902108842C8
:10E2900002DAB5F9020001E0B6F90200ADF8320089
:10E2A000B5F90200B6F90210884202DDB5F90200A4
:10E2B00001E0B6F90200401E00B2ADF83600119838
:10E2C0000CA982680CA8F7F776FD8146B9F1000F1A
:10E2D00002D115B0BDE8F08FE08818B1A08808B170
:10E2E000012000E00020824601200B900CA810F0D5
:10E2F000E5FC10B100200B9004E0BAF1000F01D052
:10E3000000200B901C2104A817F03EFC0CA80490E0
:10E310002088ADF81800207A8DF828000B9820B1DD
:10E3200004A9119811F082FB66E00CA80BF0DDFF48
:10E330008346BDF936000390BDF83200ADF83600D3
:10E34000584617F0B7F90290029807900CA8099068
:10E3500000200190BAF1000F0BD0B4F90600B4F917
:10E3600004100844BDF9321091FBF0F200FB1210CA
:10E370000190019FBDF9328037E05946029817F0AD
:10E380003AFCBDF930100FFA8BF30FFA88F20298BD
:10E3900010F044FC8DF82000BAF1000F13D09DF866
:10E3A000200070B1B4F90400B84202DA00208DF800
:10E3B0002000B4F90600B4F904100844B84200DCA7
:10E3C0000027781C07B204A9119811F02FFBBDF8A3
:10E3D0003200401C00B2ADF83200BDF83600401CDF
:10E3E00000B2ADF8360008F1010803988045C4DD9D
:10E3F000029817F0DBF900BF00BF6AE72DE9FC5F68
:10E400008046404613F0B4F80746B946D9F8246070
:10E410003446404613F053F80546606A00F1140292
:10E420006846A968F7F7C7FC8246BAF1000F41D0E9
:10E43000D5F808B0C5F808D094F83C00C0F34010F7
:10E4400048B3608FE18E88420CD1628F2123294628
:10E450003046FDF72AFB628F212329463046FDF71F
:10E4600090FB24E0628F202329463046FDF71DFBF8
:10E47000628F202329463046FDF783FBE28E01237D
:10E4800029463046FDF711FBE28E0123294630462E
:10E49000FDF777FB0BE0628F202329463046FDF71E
:10E4A00004FB628F202329463046FDF76AFBC5F83E
:10E4B00008B000BFBDE8FC9F2DE9F14FD0B05098E7
:10E4C00013F056F804462546288E10B951B0BDE821
:10E4D000F08F509812F0F3FF4F90608C20F0040002
:10E4E000001D60844DA9204619F099FA0026B24615
:10E4F000B4F8208000202084608C20F00400001DEF
:10E50000608427A811F068F81FA80FF0E9FF27AA78
:10E510004FF4A02120461BF095FB1FAA4FF4A02129
:10E5200020461BF0A9FA608C20F004006084A4F857
:10E530002080002120461AF0B5FD1E9000212046C3
:10E540001AF094FB1D90002120461AF05BFC1C90F1
:10E55000002120461AF0F2FC1B9009A84F9918F0F0
:10E560005FFF4FF4A0201690D7480A9000200B9030
:10E570003DA80D9035A80E9000BF9BE103E00AF185
:10E5800001001FFA80FA696A51F82A00CFA1F2F758
:10E59000C7F80028F3D0E96A31F81600FAF796FABE
:10E5A00000B181E10027E96A31F81600FAF77EFA36
:10E5B00008B147F00107E96A31F81600FAF78AFA5C
:10E5C00010B147F0800716E0A88EB04213D108F0D2
:10E5D000200008B147F0200708F0020008B147F01A
:10E5E000020708F0040008B147F0040708F008002B
:10E5F00008B147F00807A86A00EBC6014BA80BF06A
:10E60000B3FDBDF82C01BDF83411084400B2ADF8DB
:10E610002C01BDF82E01BDF83611084400B2ADF84A
:10E620002E01BDF83001BDF83411084400B2ADF838
:10E630003001BDF83201BDF83611084400B2ADF822
:10E64000320157B9382227A93DA817F01BF920221B
:10E650001FA935A817F016F91DE02784608C20F05B
:10E660000400001D60843DA810F0B6FF35A80FF02F
:10E6700037FF3DAA4FF4A02120461BF0E3FA35AA4C
:10E680004FF4A02120461BF0F7F9A4F82080608CFD
:10E6900020F004006084E96A31F81600FAF722FAE3
:10E6A0008346BBF1000F06D09DF8F10040F0010059
:10E6B0008DF8F10005E09DF8F10020F001008DF8E3
:10E6C000F1004BA80C90179609AA1A21204612F0C7
:10E6D00055FF9DF81701400800F01000F0B39DF8B9
:10E6E000170120F03E001E308DF81701BDF92C11E6
:10E6F000B4F914201C98104481420AD19DF81701E6
:10E70000400820F004009DF8171160F345018DF8D2
:10E710001711BDF93011B4F918201B98101A814255
:10E720000AD19DF81701400820F008009DF8171144
:10E7300060F345018DF81711BDF92E11B4F91620BB
:10E740001E98104481420CD19DF81701400820F01A
:10E7500002009DF8171160F3450100E014E08DF808
:10E760001711BDF93211B4F91A201D98101A8142FF
:10E770000AD19DF81701400820F001009DF81711FB
:10E7800060F345018DF817114BA80BF05EFD814633
:10E7900007F0200060B1E86A30F8160000F48060ED
:10E7A00030B1BDF82E01A0EB090000B2ADF82E018A
:10E7B0004BAA3DA94F9810F0F3FE35980890BDF98B
:10E7C000E8000790BDF9E6000690686A50F82A0054
:10E7D00005904DA80BF0C8FD03909DF8F11002467E
:10E7E0000698CDE90121009004A8DDE907320599DA
:10E7F00021F0C4FB4BA80BF0B7FDBDF91010401A77
:10E80000039000EBD070BDF82C1101EB600000B25A
:10E81000ADF82C014BA80BF018FDBDF91210401AF1
:10E82000039000EBD070BDF82E1101EB600000B238
:10E83000ADF82E01BDF82C01BDF81010084400B24F
:10E84000ADF83001BDF82E01BDF81210084400B239
:10E85000ADF8320107F02000C0B1E86A30F81600C8
:10E8600000F4806090B1484609EBD071BDF82E21CC
:10E87000A2EB610109B2ADF82E1109EBD071BDF820
:10E880003221A2EB610109B2ADF8321100200090F3
:10E890004BAA35A9059B4F980FF06AFA09AA1B21CC
:10E8A000204612F06BFE00BF701C86B20AF1010018
:10E8B0001FFA80FA288EB0423FF760AE608C20F0DD
:10E8C0000400608400BF01E6280204080A0000007A
:10E8D0002DE9F14FA2B0229812F04AFE04462546D7
:10E8E000229812F0ECFD2190002120461AF051F8F8
:10E8F0008146264600271222394630461AF026FC69
:10E900000A900A98484400B2209000BF132239466A
:10E9100030461AF01BFC0A900A98484400B21F9037
:10E92000002120461AF0D6FB484400B21E9016A8DB
:10E930000FF0D6FD16AA4FF4003120461BF09CF8CC
:10E94000A86A10B1D5F828800AE0802016F0B2FE3F
:10E95000064680223146204612F0E0FAB04600BF5B
:10E960004FF0000A95F83C0000F00F00012800D19C
:10E97000824600261622314620461AF0E7FB0A900E
:10E980000A98C0B2012800D18246E86A00287DD0EA
:10E99000E86A14F042FE0A900A98022814D19DF801
:10E9A000750041F6FF72BDF96A10CDE900120290C0
:10E9B000BDF96C30169A07A8E96A21F0DFFABDF9B3
:10E9C0001C60BDF91E7011E007A9E86A14F0FCF99B
:10E9D0008346BBF1010F05D10798C0F38A2607983B
:10E9E000470D02E04FF0FF36374600BFBAF1000F87
:10E9F0000DD0A18A2098084400B2ADF82000BDF8DF
:10EA000020003044401E00B2ADF824000DE0218B00
:10EA10001F98081A801B00B2ADF82000BDF8200036
:10EA20003044401E00B2ADF824000A98022815D1E7
:10EA3000E18A1E98084400B2ADF82200BDF8220019
:10EA40003844401E00B2ADF826000020009008AA0D
:10EA500016A9EB6A21980FF08BF93FE0204619F0D8
:10EA600035F8A0EB070B0BEBDB704110E08A084494
:10EA700000B2ADF82200BDF822003844401E00B2BA
:10EA8000ADF8260002A80FF056F900E027E002AA30
:10EA90004FF4003120461AF087FF304606EBD07164
:10EAA000491009B2ADF80C10384607EBD071491087
:10EAB0000AB2ADF80E204FF4003B6E2259462046B4
:10EAC0001AF044FB0190019800B2ADF8080008AAC2
:10EAD00002A9EB6A21980FF0DDF800BF00BF0EA875
:10EAE0000FF0FEFC0EAA002120461AF0C5FF9DF88B
:10EAF000550041F6FF72BDF94A10CDE900120290AF
:10EB0000BDF94C3041460DA80E9A21F037FAE18A42
:10EB10001E98084400B2ADF82E00BDF82E00BDF8D6
:10EB20003610084400B2ADF83200E86AB0B92046A9
:10EB30001AF01FFEBDF93410461A06EBD670A18AF2
:10EB400001EB600000B2ADF82C00BDF82C00BDF860
:10EB50003410084400B2ADF8300022E0BAF1000FE2
:10EB600011D0218B1F98081ABDF83410401A00B23A
:10EB7000ADF82C00BDF82C00BDF83410084400B2EC
:10EB8000ADF830000DE0A18A2098084400B2ADF83D
:10EB90002C00BDF82C00BDF83410084400B2ADF8CC
:10EBA0003000002043460BAA0EA9009021980FF0D8
:10EBB000DFF8A86A10B9404616F0F8FD23B0BDE8AA
:10EBC000F08F2DE9F14F90B0109812F0D1FC05466E
:10EBD0002C46109812F073FC06460EA9284618F031
:10EBE000AAFE002794F84800C0F3001008B147F0CF
:10EBF000010794F84800C0F3401008B147F002073D
:10EC0000002128461AF094FC42F2D171884205D1C5
:10EC1000688CC0F3802008B947F0040706A80FF0FD
:10EC20005FFCB4F84400ADF82E004620005BADF860
:10EC300030008DF8357006AA002128461AF01CFF16
:10EC40000DA8411E626A03780BB90123037000BF4F
:10EC5000284615F09CFC0790284615F092FC089079
:10EC60004FF6FF710798884223D00898884220D039
:10EC70004FF4802B5522594628461AF067FA02466F
:10EC8000594601902846F8F703F90290029803903C
:10EC9000BDF80C00ADF8260000BF202259462846DA
:10ECA0001AF054FA029002980390BDF80C00ADF8E7
:10ECB000280094F8480000F00700022805D094F8D6
:10ECC000480000F0070003281FD19DF834000228F7
:10ECD00003D09DF83400032817D141F6FF71BDF928
:10ECE0002A008DE88300BDF92C30069A03A8616ADA
:10ECF00021F044F90EA80BF045FBBDF90C10884239
:10ED000002DA01208DF8340000BF04F1300894F8D5
:10ED1000480000F00700032805D00EA80BF0A3FA66
:10ED2000B0F5806F01DA4FF000080EA904A8B268B0
:10ED3000F7F741F88146B9F1000F02D111B0BDE8F3
:10ED4000F08F94F8480000F0070070B9284619F0D9
:10ED5000ADF88346CBF1000002B200210EA80BF003
:10ED600029FB688BADF83E0000BF94F8480000F026
:10ED70000700022805D094F8480000F00700032897
:10ED80000ED1D6F808B004A8B060CDF800800EAA65
:10ED900006A93046636A0EF0EBFFC6F808B007E03C
:10EDA000CDF800800EAA06A93046636A0EF0E0FF97
:10EDB000D6F808A004A8B06094F8480000F0070056
:10EDC00003284FD141F6FF71BDF92A008DE8830079
:10EDD000BDF92C30069A03A8616A21F0CFF80EA87D
:10EDE0000BF0D0FABDF90C1088421BDA2022114634
:10EDF000069812F047FD00EB4000B4F84410BDF84F
:10EE00000C201144084400B2ADF82E004620005BEF
:10EE1000ADF83000CDF800800EAA06A93046636A2E
:10EE20000EF0A6FF0EA80BF01EFABDF90E108842D8
:10EE300017DAB4F84400ADF82E00069812F03BFD46
:10EE40004621095BBDF80E201144084400B2ADF81C
:10EE50003000CDF800800EAA06A93046636A0EF095
:10EE600087FF00BFC6F808A000BF67E72DE9F14F94
:10EE70009AB01A9812F01BFB19901A9812F078FBAE
:10EE800004461998152816D11A9812F018FB054651
:10EE900017A9204606F0FAFD09A810F09DFB09AA63
:10EEA0004FF4802120461AF0CDFE17AA09A9284662
:10EEB00010F076FBD1E019981828FBD11A9812F0BF
:10EEC000FEFA054611A80FF00BFB11AA4FF48021A2
:10EED00020461AF0D1FD0FA9204606F0D7FD0FAA53
:10EEE0000DA8A968F6F767FF0C900C9800287CD055
:10EEF000204606F0BAF80B900B9815F033FB28B1BA
:10EF00009DF8610040F001008DF8610020461AF084
:10EF100030FC04900B9815F02EFB02220390BDF9F3
:10EF200056100498CDE901020091BDF958300AA8A5
:10EF3000119A039921F022F8204618F0C7FD0646E1
:10EF4000304606EBD0714A10B4F916100A440B99FA
:10EF5000B1F91610891A09910B9818F0B7FD0999A3
:10EF6000890391FBF0F00990002120461AF0DBF9AB
:10EF700008901199B1F908200899B1F90810501AB0
:10EF800000EBD07149100FB2BDF82A00C01B00B2CF
:10EF9000ADF82A00304606EBD0714A10B4F91610CD
:10EFA00002EB0108BDF92A000999484308EBA03893
:10EFB000A8EB07080021204619F0F7FC8146002045
:10EFC00004901222204604991AF0C0F80390039886
:10EFD0000FFA80FA00BF0020049013222046049903
:10EFE0001AF0B4F80390039800E035E00FFA80FBC4
:10EFF00000BFA08A5044484400B2ADF818000FFA90
:10F0000088F0ADF81A00208BA0EB0B00A0EB0900F4
:10F0100000B2ADF81C00BDF81A00BDF82A10084473
:10F0200000B2ADF81E009DF8610040F002008DF8BE
:10F030006100A86805900DA8A8600B9815F09BFAD0
:10F0400004900020009006AA11A92846049B0EF007
:10F050008FFE0598A86000BF00BF1BB0BDE8F08F11
:10F060002DE9F14FA8B0289812F082FA04462546FF
:10F07000289812F024FA27900021204619F0E6FE85
:10F0800026900021204619F07DFF25900021204682
:10F090001AF038F824900021204619F00BFE239036
:10F0A00000BFA08AADF88400E08AADF88600208B0E
:10F0B000ADF88800608BADF88A0000BFBDF8841001
:10F0C0002698084400B2ADF88400BDF88810259851
:10F0D000081A00B2ADF88800BDF8861024980844DC
:10F0E00000B2ADF88600BDF88A102398081A00B265
:10F0F000ADF88A0013A810F06FFA13AA4FF400318C
:10F1000020461AF09FFD21AA13A9279810F048FA6B
:10F110000026204618F0DAFC074600BF208BA18AA3
:10F12000401A401CC01B0FFA80F8686A401C40B1AE
:10F13000696A01FB08F0C11700EB116109120EB2F8
:10F140000CE0204619F026FB00F0010BBBF1000F8C
:10F1500001D0404600E00020064600BF4FF0000B03
:10F1600016225946204619F0F1FF00900098C0B2CF
:10F17000012802D1A8EB060006B2A08A304400B2F2
:10F18000ADF84400BDF84400384400B2ADF8480082
:10F19000E08AADF84600608BADF84A004FF440318C
:10F1A000204619F053FE81464FF44031204619F0B5
:10F1B000E9FE82464FF44031204619F0A3FF10903B
:10F1C0004FF44031204619F075FD0F90BDF8440012
:10F1D000A0EB090000B2ADF84400BDF8480050446F
:10F1E00000B2ADF84800BDF846101098081A00B2F9
:10F1F000ADF84600BDF84A100F98084400B2ADF8CB
:10F200004A0001A810F0E8F901AA4FF44031204665
:10F210001AF018FD11AA01A9279810F0C1F929B018
:10F22000BDE8F08F2DE9F14FE0B0609812F0A0F941
:10F2300004462546609812F042F9804604F1140114
:10F240005EA8D8F80820F6F7B6FD10B961B0BDE8A1
:10F25000F08FD8F808005D905EA8C8F808004FF05D
:10F26000000932224946204619F070FF1390139886
:10F2700000B259900021204619F050FF589000210B
:10F28000204619F023FD57900021204619F0EAFD91
:10F2900056900021204619F081FE5590208C549004
:10F2A00000202084608C20F00400001D608446A8AB
:10F2B00010F092F946AA4FF4A02120461AF0C2FCA1
:10F2C00030A80FF00DF930AA4FF4A02120461AF013
:10F2D000D3FB54982084608C20F0040060840027C5
:10F2E000204618F0F7FD0146E28A58981044401E67
:10F2F000411A5998084400B2ADF86E01204618F042
:10F30000DFFD27900021204619F0DBFA012800D10B
:10F3100000E000202690414614A818F081F84FF430
:10F32000A0202190FE4815900020169038A8189033
:10F3300028A819904FF0000B40E2E86A30F91B0052
:10F340001390BDF86E01401C00B2ADF86A01BDF823
:10F350006A1113980844401E00B2ADF86E01BDF961
:10F360006A01BDF97E11884200DD2BE2269858B172
:10F37000218B5598081A401E2799411A5998081A46
:10F3800000B2ADF868010AE0A18A56980844401E10
:10F390002799411A5998084400B2ADF86C0100262B
:10F3A00004E200201290A86A50F8270020B1A86A51
:10F3B00050F8270000781290269880B1BDF86801B7
:10F3C000401E00B2ADF86C01286B30F81600BDF895
:10F3D0006C11081A401C00B2ADF868010FE0BDF8CE
:10F3E0006C01401C00B2ADF86801286B30F81600C3
:10F3F000BDF868110844401E00B2ADF86C014FF032
:10F40000000900BF2CE007EB0901A86A50F82100B1
:10F410000F900F9808F0F3FE00B127E00F980078E6
:10F420000E900E9800F00100A8B106EB0901491CEE
:10F430002A6B32F91100269931B1BDF86811091A09
:10F4400009B2ADF8681105E0BDF86C11014409B2CC
:10F45000ADF86C1100E009E009F101001FFA80F934
:10F4600009EB0601A88C401E8142CCDB00BFBDF930
:10F470006E01BDF97A11884207DA09F101003844BA
:10F4800087B206EB090086B28EE100BFBDF86801C5
:10F49000ADF84000BDF86A01ADF84200BDF86C015E
:10F4A000ADF84400BDF86E01ADF8460000BF9DF810
:10F4B0003B01400800F0040090B1BDF94010B4F9E0
:10F4C00014205698104481420ADDBDF9380100EB42
:10F4D000D071BDF84020A2EB610109B2ADF8401037
:10F4E0009DF83B01400800F0020090B1BDF94210C8
:10F4F000B4F916205898104481420ADDBDF938014C
:10F5000000EBD071BDF84220A2EB610109B2ADF869
:10F5100042109DF83B01400800F00800B8B1BDF969
:10F520004410B4F918205598101A401E81420EDA82
:10F53000BDF9380100EBD07182B202F0010202EB9A
:10F540006101BDF84420114409B2ADF844109DF8A2
:10F550003B01C0F34000B8B1BDF94610B4F91A2020
:10F560005798101A401E81420EDABDF9380100EB9F
:10F57000D07182B202F0010202EB6101BDF84620B7
:10F58000114409B2ADF846104FF0000AE88E584514
:10F5900023D1A88EB04220D194F8200000F0400082
:10F5A00030B994F8200000F0200008B14AF0200A99
:10F5B00094F8200000F0020008B14AF0020A94F822
:10F5C000200000F0040008B14AF0040A94F820007A
:10F5D00000F0080008B14AF0080ABAF1000F0AD199
:10F5E000382246A938A816F04DF9202230A928A8BB
:10F5F00016F048F91EE0A4F820A0608C20F004006A
:10F60000001D608438A80FF0E7FF28A80EF068FFFF
:10F6100038AA4FF4A02120461AF014FB28AA4FF470
:10F62000A02120461AF028FA54982084608C20F0FB
:10F630000400608410A81790A88C0BFB0060229037
:10F6400014AA1A21204611F099FF10AA38A94046A1
:10F650000FF0A6FFA86A50F8270000285FD04FF4EB
:10F66000A021204619F0FEFB0F904FF4A021204668
:10F6700019F094FC0E904FF4A021204619F04EFD95
:10F680000D904FF4A021204619F020FB0C90002093
:10F690000B90BDF868110F98084400B2ADF8240033
:10F6A000BDF86C110E98081A00B2ADF82800BDF82C
:10F6B0006A110D98084400B2ADF82600BDF86E112D
:10F6C0000C98081A00B2ADF82A001298C0F3400056
:10F6D0000890089808B102200B9000BFBDF82800E0
:10F6E000BDF82410401A401C00B20490BDF9B220AD
:10F6F00004990B98CDE900210290A86A50F82700E0
:10F70000411CBDF9B4305CA8309A20F037FC089851
:10F7100018BB139901EBD172BDF86A3102E036E0F3
:10F720005C03040803EB6202BDF9720100EBD073C5
:10F73000A2EB630212B2ADF82620139901EBD1724D
:10F74000BDF86A3103EB6202BDF9720100EBD073C0
:10F7500002EB630212B2ADF82A205AAA5EA906A8EB
:10F76000F6F729FB0590059880B106A8C8F80800AF
:10F7700000200090A86A50F82700431C09AA28A975
:10F7800040460EF0F5FA5EA8C8F8080000BF14AABB
:10F790001B21204611F0F2FE09F10100384487B226
:10F7A00006EB090086B200BF701C86B2A88CB0427E
:10F7B0003FF7F7AD0BF101001FFA80FBE88C5845CD
:10F7C0003FF7BBAD00BF5D98C8F8080000BF3DE53E
:10F7D0002DE9F04FA3B007468946164622973046DA
:10F7E0000AF0ADFD054600EBD5704FEA60083088A1
:10F7F000404400B2ADF884007088404400B2ADF8D7
:10F8000086001EA80EF02FFF1EAA4FF4A021384636
:10F810001AF09AF918A80EF08EFA18AA4FF4A0213F
:10F8200038461AF0C1F80021384619F06DF91790E2
:10F83000494605A817F0F4FD7148069021A80E90DE
:10F8400022983030F7F7F5F90446D3E0256816948E
:10F85000207901285CD1B5F92000E98B084400909B
:10F86000B5F92030D5E90512E06815F0B5FE8246FD
:10F87000A88B00EB0801608A08440FFA80FB0FFA9E
:10F880008AF020F08DFA10FB0BF047F6FF7190FB29
:10F89000F1F0BDF88610084400B2ADF812000FFA7E
:10F8A0008AF020F074FA10FB0BF047F6FF7190FB22
:10F8B000F1F0BDF88410084400B2ADF81000A08A41
:10F8C000ADF87800208A00B2ADF87A006079FD28A2
:10F8D00001DD179803E060791799484300128DF80D
:10F8E0008000012013901EA80B9004A80F9005AA79
:10F8F0001A21384611F042FE04AB21AA1EA948463F
:10F900000EF09AFE05AA1B21384611F037FE6AE078
:10F910002079002867D1206900B965E0B5F9200099
:10F92000E98B08440090B5F92030D5E90512E0686C
:10F9300015F052FE824604A9206913F045FABDF87D
:10F940008410A08A081A00B2ADF80800BDF886102D
:10F95000E08A081A00B2ADF80A00BDF80800049960
:10F96000C1F38A210844401E00B2ADF80C00BDF876
:10F970000A00049900EB5150401E00B2ADF80E0091
:10F980006079FD2801DD179803E0607917994843F5
:10F9900000128DF86B00A08AADF86400E18A18A807
:10F9A000C1800AEB8A004FEA400ABAF5616F01DDB7
:10F9B000AAF5616A0FFA8AF0ADF860000220139090
:10F9C00018A80C9005AA1A21384611F0D7FD02AAF2
:10F9D00018A9484623690EF05DF905AA1B2138468F
:10F9E00011F0CCFD00BF00BF214622983030F7F760
:10F9F0001AF90446002C7FF429AF23B0BDE8F08F3C
:10FA0000CCC803082DE9F74F8AB00C46904694F80D
:10FA10002A00022802DC0DB0BDE8F08FE08C00B9AE
:10FA2000F9E794F82A90B9F1FD0F01DD4FF0FF09D5
:10FA3000414608A80AF074FB208D401E05B2BDF8AF
:10FA40002000401B00B2ADF82000BDF82200401B92
:10FA500000B2ADF82200BDF82400284400B2ADF891
:10FA60002400BDF82600284400B2ADF8260008A9FD
:10FA700006A80AF055FBBDF81800E18C401A00B248
:10FA8000ADF81800BDF81C00E18C084400B2ADF8D8
:10FA90001C00BDF81A00E18C401A00B2ADF81A0043
:10FAA000BDF81E00E18C084400B2ADF81E0008A8A5
:10FAB0000AF022FC824608A80AF09DFB0746B4F92A
:10FAC0000060BA4501DA504600E038468346B6EB9E
:10FAD0006B0F01DD4FEA6B06E08C304400B20590FD
:10FAE000A07894F82A10CDE90210A08CADF804009B
:10FAF00030B2009008AA06A9059B0A98FBF781FC82
:10FB000000BF88E7F8B50546284611F031FD0646E6
:10FB1000284611F02AFD0446606BB0F5A02F54D1A1
:10FB2000A06B072806D200202169C870216981F8DE
:10FB3000220014E0208F81B2402230460BF04CFBB3
:10FB400068B100202169C870216981F82200122063
:10FB50001CF0E6F90090BDF8001060698181208FEB
:10FB600081B24FF4004230460BF036FB98B166206C
:10FB70002169C87030461FF001FE0090BDF80010EA
:10FB80002069818030460BF021FBA16B884202D1B5
:10FB9000B2202169C870208F81B24FF48042304674
:10FBA0000BF01AFB88B1FF20216981F82200304652
:10FBB0001FF0E4FD0090BDF800102069C1832069AA
:10FBC000008C401C00B221690884F8BD2DE9F04F7B
:10FBD0008BB08146484611F0CBFC05462C46484682
:10FBE00011F06DFC8346606A14F0C5FC82469AF8F9
:10FBF000000000283ED1A06A00283BD0A06A00780F
:10FC0000C0B303A80EF06CFC03AA4FF400212846F1
:10FC100019F032FF94F86000C0F3C00028B19DF8DD
:10FC2000290040F002008DF829000021284619F033
:10FC300025F907460021284619F07CFA8046002164
:10FC4000284618F0BEFE064605F1140101A80AF088
:10FC5000A6FA08EB060002B2B81901B201A80AF030
:10FC6000A9FB0020009001AA03A95846A36A0EF040
:10FC70007FF800BF0BB0BDE8F08F7CB50446A069EB
:10FC800085686089002856D1A089002853D1E08872
:10FC9000218988424FDAE18808B220F081F8B4F96E
:10FCA0000410B4F90E20891A48432168498801EBF1
:10FCB000E03000B2ADF80200E1885A3108B220F01D
:10FCC0006FF8A18810FB01F02168098801EBE03092
:10FCD00000B2ADF80400218908B220F061F8A188D3
:10FCE00010FB01F02168498801EBE03000B2ADF86B
:10FCF000060021895A3108B220F052F8B4F90410F4
:10FD0000B4F90E20891A48432168098801EBE030D4
:10FD100000B2ADF800002A4669466846F6F74BF88F
:10FD200006463EB1A169C1F808D0D4E90412A06921
:10FD30000FF036FCC2E0608910B1A08900287BD1A9
:10FD40006089D0BB20680088ADF80000206840883A
:10FD5000A188084400B2ADF80600E18808B220F09E
:10FD60001FF8B4F90410B4F90E20891A4843216829
:10FD7000498801EBE03000B2ADF80200E1885A3169
:10FD800008B220F00DF8A18810FB01F02168098865
:10FD900001EBE03000B2ADF804002A46694668463F
:10FDA000F6F709F806463EB1A169C1F808D0D4E9D2
:10FDB0000412A0690FF0F4FB00BFA08900287DD1D8
:10FDC00020680088A188084400B2ADF804002068CB
:10FDD0004088ADF80200218908B21FF0E1FFA18838
:10FDE00010FB01F02168498801EBE03000B2ADF86A
:10FDF000060021895A3108B21FF0D2FFB4F904106D
:10FE0000B4F90E20891A48432168098801EBE030D3
:10FE100000B2ADF800002A4669466846F5F7CBFF08
:10FE200006463EB1A169C1F808D0D4E90412A06920
:10FE30000FF0B6FB42E0FFE76089A189884205D157
:10FE4000608918B12089E188884211DB6089022825
:10FE500002D1A08901280BD06089032802D1A08992
:10FE6000022805D06089032828D1A089012825D13E
:10FE700020680088ADF8000020684088ADF80200D6
:10FE800020680088A188084400B2ADF8040020680A
:10FE90004088A188084400B2ADF806002A466946A9
:10FEA0006846F5F788FF06463EB1A169C1F808D05B
:10FEB000D4E90412A0690FF073FB00BFA06985604C
:10FEC0007CBD7CB50446A06985686089012856D14F
:10FED000A089012853D1E088218988424FDAE1883E
:10FEE00008B21FF05DFFA18810FB01F0216849886E
:10FEF00001EBE03000B2ADF80600E1885A3108B2FB
:10FF00001FF04EFFB4F90410B4F90E20891A4843CB
:10FF10002168098801EBE03000B2ADF804002189C6
:10FF200008B21FF03DFFB4F90410B4F90E20891A8D
:10FF300048432168498801EBE03000B2ADF8020087
:10FF400021895A3108B21FF02BFFA18810FB01F064
:10FF50002168098801EBE03000B2ADF800002A46C4
:10FF600069466846F5F727FF06463EB1A169C1F824
:10FF700008D0D4E90412A0690FF012FBC7E0608931
:10FF8000012802D0A08901287ED1608901283AD1B8
:10FF900020680088A188401A00B2ADF800002068EF
:10FFA0004088ADF80200E18808B21FF0F9FEA18890
:10FFB00010FB01F02168498801EBE03000B2ADF898
:10FFC0000600E1885A3108B21FF0EAFEB4F90410C5
:10FFD000B4F90E20891A48432168098801EBE03002
:10FFE00000B2ADF804002A4669466846F5F7E3FE1C
:10FFF00006463EB1A169C1F808D0D4E90412A0694F
:020000040801F1
:100000000FF0CEFA00BFA0890128B7D12068008880
:10001000401E00B2ADF8040020684088A188084462
:1000200000B2ADF80600218908B21FF0B9FEB4F99C
:100030000410B4F90E20891A48432168498801EB5D
:10004000E03000B2ADF8020021895A3108B21FF049
:10005000A7FEA18810FB01F02168098801EBE030C0
:1000600000B2ADF800002A4669466846F5F7A3FEDF
:1000700006463EB1A169C1F808D0D4E90412A069CE
:100080000FF08EFA43E0FFE76089A189884206D12C
:100090006089012803D02089E18888420FDB6089CC
:1000A00010B9A08902280AD0608910B9A089032854
:1000B00005D0608903282AD1A089022827D1206889
:1000C0000088A188401A00B2ADF80000206840887E
:1000D000ADF8020020680088401E00B2ADF80400B0
:1000E00020684088A188084400B2ADF806002A467E
:1000F00069466846F5F75FFE06463EB1A169C1F85C
:1001000008D0D4E90412A0690FF04AFA00BFA06930
:1001100085607CBD7CB50446A0698568608902283D
:1001200056D1A089022853D1E088218988424FDA2C
:10013000E1885A3108B21FF033FEA18810FB01F0AC
:100140002168098801EBE03000B2ADF80000E188D9
:1001500008B21FF025FEB4F90410B4F90E20891A74
:1001600048432168498801EBE03000B2ADF8060051
:10017000218908B21FF014FEA18810FB01F021684C
:10018000498801EBE03000B2ADF8020021895A3114
:1001900008B21FF005FEB4F90410B4F90E20891A54
:1001A00048432168098801EBE03000B2ADF8040053
:1001B0002A4669466846F5F7FEFD06463EB1A16946
:1001C000C1F808D0D4E90412A0690FF0E9F9CCE035
:1001D0006089022802D0A08902287DD16089022886
:1001E0003CD120680088401E00B2ADF804002068B1
:1001F0004088A188401A00B2ADF80200E1885A3167
:1002000008B21FF0CDFDA18810FB01F0216809881C
:1002100001EBE03000B2ADF80000E18808B21FF059
:10022000BFFDB4F90410B4F90E20891A48432168BF
:10023000498801EBE03000B2ADF806002A46694675
:100240006846F5F7B8FD06463EB1A169C1F808D089
:10025000D4E90412A0690FF0A3F900BFA089022815
:10026000B5D120680088A188401A00B2ADF800001E
:1002700020684088401E00B2ADF8060021895A313E
:1002800008B21FF08DFDB4F90410B4F90E20891ADC
:1002900048432168098801EBE03000B2ADF8040062
:1002A000218908B21FF07CFDA18810FB01F02168B4
:1002B000498801EBE03000B2ADF802002A466946F9
:1002C0006846F5F778FD06464EB1A169C1F808D039
:1002D000D4E90412A06900E002E00FF061F944E003
:1002E0006089A189884206D16089022803D02089CB
:1002F000E18888420FDB608910B9A08903280AD001
:100300006089012802D1A089032804D060890128CE
:100310002BD1A08948BB20680088A188401A00B270
:10032000ADF8000020684088A188401A00B2ADF8FE
:10033000020020680088401E00B2ADF8040020686A
:100340004088401E00B2ADF806002A46694668465D
:10035000F5F731FD06463EB1A169C1F808D0D4E9F0
:100360000412A0690FF01CF900BFA06985607CBD74
:100370007CB50446A06985686089032856D1A089A8
:10038000032853D1E088218988424FDAE1885A3125
:1003900008B21FF005FDB4F90410B4F90E20891A53
:1003A00048432168098801EBE03000B2ADF8000055
:1003B000E18808B21FF0F4FCA18810FB01F021686D
:1003C000498801EBE03000B2ADF8020021895A31D2
:1003D00008B21FF0E5FCA18810FB01F02168098834
:1003E00001EBE03000B2ADF80400218908B21FF043
:1003F000D7FCB4F90410B4F90E20891A48432168D7
:10040000498801EBE03000B2ADF806002A466946A3
:100410006846F5F7D0FC06463EB1A169C1F808D0A0
:10042000D4E90412A0690FF0BBF8C7E06089032883
:1004300002D0A08903287ED1608903283CD120689E
:100440000088A188084400B2ADF804002068408804
:10045000401E00B2ADF80600E1885A3108B21FF024
:100460009FFCB4F90410B4F90E20891A484321689E
:10047000098801EBE03000B2ADF80000E18808B275
:100480001FF08EFCA18810FB01F02168498801EB68
:10049000E03000B2ADF802002A4669466846F5F73A
:1004A0008AFC06463EB1A169C1F808D0D4E904121D
:1004B000A0690FF075F800BFA08903287ED12068DD
:1004C0000088ADF8000020684088A188401A00B27A
:1004D000ADF8020021895A3108B21FF061FCA188F1
:1004E00010FB01F02168098801EBE03000B2ADF8A3
:1004F0000400218908B21FF053FCB4F90410B4F9C8
:100500000E20891A48432168498801EBE03000B287
:10051000ADF806002A4669466846F5F74CFC0646E3
:100520003EB1A169C1F808D0D4E90412A0690FF066
:1005300037F843E0FFE76089A189884206D16089E6
:10054000032803D02089E18888420FDB60890228D4
:1005500001D1A08950B16089012801D1A08928B1B9
:10056000608902282AD1A089012827D12068008823
:10057000ADF8000020684088A188401A00B2ADF8AC
:10058000020020680088A188084400B2ADF8040089
:1005900020684088401E00B2ADF806002A46694631
:1005A0006846F5F708FC06463EB1A169C1F808D0D7
:1005B000D4E90412A0690EF0F3FF00BFA0698560C2
:1005C0007CBD000070B5A4B006460D4620AA22A945
:1005D000304617F089FC22A809F04CFE28B920A863
:1005E00009F048FE08B924B070BD12A9304622F0C7
:1005F00019FD0446012C00D0F5E72946684616F09F
:100600000FFF1B4801900220029012A804904FF4A3
:1006100080300D9022A809F02DFE80B122A8039011
:100620006A461A21304610F0A9FF22AA12A92846CC
:100630000EF0B6FF6A461B21304610F09FFF20A83F
:1006400009F018FE90B120A803906A461A2130469E
:1006500010F094FF20A8039020AA12A928460EF0BB
:100660009FFF6A461B21304610F088FF00BFBAE7A3
:10067000BCC103082DE9F04FB3B005460F4605F1A4
:10068000140131A8BA68F5F796FB10B933B0BDE88C
:10069000F08FB868309031A8B8602C460021284609
:1006A00018F080FB2D900021284618F0CBFC2C90F0
:1006B000284617F095F9B4F88410484300120FFA51
:1006C00080FB284617F06DF9B4F8861048430012F5
:1006D00000B22B9004F12400F6F78CFA2990002147
:1006E000284618F017FB823461884843001228908E
:1006F0002188491E289801FB10B0218890FBF1F059
:1007000001B227914FF4A021284618F003FB61881D
:10071000823C4843001226902998421EDDE92601BA
:1007200002FB10112998B1FBF0F00FFA80F9B9F132
:10073000010F01DA4FF001090021284618F01DF9D8
:100740002590284617F0B8FA2D99091A25980844DB
:1007500000B22490284617F0A9FB2C99091A259875
:10076000084400B2239015A80EF036FF15AA4FF4E6
:10077000A021284619F066FA15A8C07B20F00701D1
:1007800015A8C173FF208DF85700688BBDF8541071
:10079000084400B2ADF8BE00394603A816F040FE8A
:1007A0004FF4A02010905C480490042005904FF076
:1007B0000008A7E02798ABEB000000FB08F0B4F8B6
:1007C0008210491E90FBF1F0A98A01442498084444
:1007D00000B20290CDF8448004F12400F6F729FA23
:1007E000064687E0307B00F0010000B17CE0314636
:1007F00028460BF015FB00B201900298ADF8B80046
:10080000BDF8B8004844401E00B2ADF8BC002698C0
:1008100009EB00010298084400B20290BDF9BC0047
:10082000BDF9C410884200DA5EE0BDF9B800BDF938
:10083000C810884200DD60E03089ADF858000198AA
:100840004044B4F8821090FBF1F201FB12000FFA61
:1008500080FA706830F91A10307BC0F3001204F18E
:100860006C0030F91200081A2B9948432A90307B0B
:10087000C0F3001104F1700030F91110307BC0F3A7
:10088000001204F16C0030F91200091A2A9890FB4A
:10089000F1F02A90DDE92A10411AE88A01442398F0
:1008A000084400B2ADF8BA00706830F91A0047F693
:1008B000FF71884217D02EA8069015A807901496AD
:1008C000706830F91A00139003AA1A21284610F014
:1008D00055FE2EAA15A938460EF062FE03AA1B216A
:1008E000284610F04BFE00BF314604F12400F6F715
:1008F0009AF90646002E7FF475AF00BF08F101009B
:100900001FFA80F8B4F8820040453FF753AF3098A3
:10091000B86000BFBAE6000094C303082DE9F34FA6
:10092000B9B083463A980BF11401826837A8F5F7FD
:1009300042FA10B93BB0BDE8F08F3A988068369023
:1009400037A93A9881605D46B5F88200022800DA3E
:10095000F0E70021584618F010F83390002158466F
:1009600018F020FA01463398084400B23290002172
:10097000584618F067FB01463398084400B231909E
:10098000584617F02DF8B5F884104843001200B20D
:100990003090584617F005F8B5F886104843001215
:1009A00000B22F90584617F087F90146BBF8142083
:1009B00032981044401A00B22E90584617F076FA3A
:1009C0000146BBF8162031981044401A00B22D9011
:1009D0003A980BF1140182682BA8F5F7ECF92A90EC
:1009E0002A9800B9A6E727A80DF03DFE27AA4FF4E4
:1009F000A021584619F0A8F819A80EF0EDFD19AA83
:100A00004FF40031584619F01DF94FF400315846A3
:100A100018F082FD064600EBD67047104FF4003107
:100A2000584618F01DF8064600EBD6704FEA600AEB
:100A3000BDF99E00574501DA394600E0514600EB0A
:100A4000D072B1EB620F06DD9DF8A50020F010001A
:100A500010308DF8A500BDF89E00012806D19DF844
:100A6000A50020F0100010308DF8A500B5F8821018
:100A70003098814201DB012000E00020189005F150
:100A80002400F6F7D6F80446D0E1207B00F0010000
:100A900000B1C5E12089ADF89C002089ADF868005F
:100AA000214658460BF0BCF906B217962E98ADF8C1
:100AB000D4002E98ADF8D000179E179EB0466068FF
:100AC00030F91810207BC0F3001205F16C0030F9EA
:100AD0001200081A2F9948431690207BC0F300118A
:100AE00005F1700030F91110207BC0F3001205F100
:100AF0006C0030F91200091A169890FBF1F016906C
:100B000016992F98411A2D98084400B2ADF8D200DA
:100B100004A83A9916F084FCC84805900320069072
:100B20004FF4A020119027A80A9019A808901594B6
:100B3000BDF9D2000390BDF9D20002904FF0000938
:100B400023E1BDF8D000ADF8D400BDF8D200ADF877
:100B5000D600BDF9D4103698B0F904003844401CD2
:100B6000814200DD16E1309800FB09F0B5F88210F3
:100B7000491E90FBF1F12E98084400B2ADF8D00068
:100B800017984844B5F8821090FBF1F201FB12006F
:100B900006B2606830F91610207BC0F3001205F130
:100BA0006C0030F91200081A2F9948431690207BE8
:100BB000C0F3001105F1700030F91110207BC0F373
:100BC000001205F16C0030F91200091A169890FB1A
:100BD000F1F0169016992F98411A2D98084400B2FA
:100BE000ADF8D200BDF9D0103698B0F90000C01BA6
:100BF000401E814201DAB046C3E0B9F1000F58D07F
:100C00001898E8B3606830F9180047F6FF71884219
:100C1000F5D0606830F916008842F0D0BDF9D210E6
:100C20000298814201DA029801E0BDF9D2000290F7
:100C3000BDF9D2100398814201DD039801E0BDF9AE
:100C4000D2000390BDF9D400BDF9D010884230D055
:100C5000BDF9D2000190BDF8D000401E00B2ADF841
:100C6000D000BDF8D000ADF8D4000398ADF8D600A0
:100C70000298ADF8D200BDF9D600BDF9D21000E05F
:100C800018E0884205D1BDF8D200401C00B2ADF892
:100C9000D20034AB35AA27A93A980DF0CDFCBDF8A7
:100CA000D000401C00B2ADF8D0000198039001982C
:100CB000029064E0BDF8D400C01B00B2ADF80000A3
:100CC000BDF8D400384400B2ADF80400BDF8D60039
:100CD000A0EB0A0000B2ADF80200BDF8D600504407
:100CE00000B2ADF80600A9F101001290606830F979
:100CF000180047F6FF71884201D035A800E00020B7
:100D00000D90606830F9160047F6FF71884201D0F7
:100D100034A800E000200E90CDF81CD0606830F9B7
:100D20001800149004AA1A21584610F027FC606895
:100D300030F9180047F6FF7188420AD0606830F930
:100D40001600884205D034AB35AA27A93A980DF091
:100D500073FC77B1BAF1000F0BD0606830F918005E
:100D600047F6FF71884204D06A4619A93A980EF0F6
:100D700017FC04AA1B21584610F000FC00BFB04627
:100D800000BF09F101001FFA80F9B5F8820048455B
:100D90003FF7D7AE00BF1898E8BBB5F882004845CA
:100DA0003DD1606830F9160047F6FF71884236D0B1
:100DB000BDF8D000C01B00B2ADF80000BDF8D000F7
:100DC000384400B2ADF80400BDF8D200A0EB0A0030
:100DD00000B2ADF80200BDF8D200504400B2ADF848
:100DE0000600A9F10100129000200D900E90CDF8A0
:100DF0001CD0606830F91600149004AA1A215846D5
:100E000010F0BCFB6A4619A93A980EF0C9FB04AA77
:100E10001B21584600E002E010F0B0FB00BF00BF0D
:100E2000214605F12400F5F7FEFE0446002C7FF470
:100E30002CAE3A993698886000BF7BE594C30308CE
:100E40002DE9F34FB3B08146349809F1140182685B
:100E500031A8F4F7B0FF10B935B0BDE8F08F349881
:100E60008068309031A9349881604D460021484611
:100E700017F083FD2D900021484617F093FF2C902A
:100E80000021484618F0DEF82B90484616F0A8FDE1
:100E9000B5F884104843001200B22A90484616F074
:100EA00080FDB5F886104843001200B229904846EC
:100EB00016F002FF0146B9F814202C9802442D9830
:100EC0001044401A00B22890484616F0EFFF014641
:100ED000B9F816202B9802442D981044401A00B2FD
:100EE000279024A80DF0BFFB24AA4FF4A021484668
:100EF00018F02AFE16A80EF06FFB16AA4FF4003168
:100F0000484618F09FFE4FF40031484618F004FBA5
:100F1000064600EBD67047104FF40031484617F0F4
:100F20009FFD064600EBD6704FEA6008BDF99200BF
:100F3000474501DA394600E0414600EBD072B1EB9B
:100F4000620F06DD9DF8990020F0100010308DF83A
:100F50009900BDF89200012806D19DF8990020F073
:100F6000100010308DF8990005F12400F5F761FEAE
:100F7000044694E1207B00F0010000B189E1208962
:100F8000ADF890002089ADF85C00214648460AF093
:100F900047FF06B215962898ADF8BC002898ADF822
:100FA000B800159E159EB346606830F816000A28F2
:100FB00047D02A980090236833F91600237BC3F3A7
:100FC000C00C05F1780333F91C20237BC3F3C00C5C
:100FD00005F1740333F91C10002314F0FDFA00B27C
:100FE000ADF8B800BDF8B8102898084400B2ADF8C4
:100FF000B80029980090636833F91600237BC3F387
:10100000001C05F1700333F91C20237BC3F3001C83
:1010100005F16C0333F91C10002314F0DDFA00B263
:10102000ADF8BA00BDF8BA102998401A00B2ADF870
:10103000BA00BDF8BA102798084400B2ADF8BA005B
:1010400005E04EF20100ADF8B800ADF8BA0003A813
:10105000349916F0E5F94FF4A020109094480490CC
:101060000320059024A8099016A8079014944FF027
:10107000000AC8E0BDF8B800ADF8BC00BDF8BA0081
:10108000ADF8BE0015985044B5F8821090FBF1F20F
:1010900001FB120006B2606830F9160047F6FF71D6
:1010A000884247D029980090636833F91600237B63
:1010B000C3F3001C05F1700333F91C20237BC3F339
:1010C000001C05F16C0333F91C10002314F084FAA2
:1010D00000B2ADF8BA00BDF8BA102998401A00B2B3
:1010E000ADF8BA00BDF8BA102798084400B2ADF8C0
:1010F000BA002A980090236833F91600237BC3F3C3
:10110000C00C05F1780333F91C20237BC3F3C00C1A
:1011100005F1740333F91C10002314F05DFA00B2DA
:10112000ADF8B800BDF8B8102898084400B2ADF882
:10113000B80001E0B34662E0BAF1000F5DD0BDF83F
:10114000BC00C01B00B2ADF80400BDF8BC003844C0
:1011500000B2ADF80800BDF8BE00A0EB080000B278
:10116000ADF80600BDF8BE00404400B2ADF80A007C
:10117000AAF101001190606830F91B0047F6FF7179
:10118000884201D02FA800E000200C90606830F960
:10119000160047F6FF71884201D02EA800E000201B
:1011A0000D9001A80690606830F91B00139003AA07
:1011B0001A21484610F0E2F9606830F91B0047F642
:1011C000FF71884213D0606830F9160088420ED053
:1011D0002EAB2FAA24A934980DF02EFA3FB1B8F106
:1011E000000F04D001AA16A934980EF0D9F903AA69
:1011F0001B21484610F0C2F900BFB34600BF0AF1F8
:1012000001001FFA80FAB5F8820050453FF732AF6F
:10121000B5F8820050453BD1606830F9160047F6BA
:10122000FF71884234D0BDF8B800C01B00B2ADF8E1
:101230000400BDF8B800384400B2ADF80800BDF8AD
:10124000BA00A0EB080000B2ADF80600BDF8BA0085
:10125000404400B2ADF80A00AAF10100119000204C
:101260000C900D9001A80690606830F9160013905C
:1012700003AA1A21484610F081F901AA16A9349848
:101280000EF08EF903AA1B21484610F077F900BF33
:1012900000BF214605F12400F5F7C5FC0446002CEB
:1012A0007FF468AE34993098886000BFD4E50000C0
:1012B00094C303082DE9F74FA2B00F46F88D10B97B
:1012C00025B0BDE8F08F97F83600022800DCF7E77C
:1012D000F88D012808D1B7F93400002804DC388ED5
:1012E00010B9788E00B9EBE724980088398E08444D
:1012F000B98E401A00B2ADF8800024988088398EEB
:101300000844B98E084400B2ADF88400249840889F
:10131000798E0844B98E401A00B2ADF88200249844
:10132000C088798E0844B98E084400B2ADF88600B2
:10133000B7F92E0000EBD071BDF88020A2EB61015F
:10134000491E09B2ADF87810B7F92E0000EBD07144
:10135000BDF8842002EB6101491C09B2ADF87C1094
:10136000B7F92E0000EBD071BDF88220A2EB61012D
:10137000491E09B2ADF87A10B7F92E0000EBD07112
:10138000BDF8862002EB6101491C09B2ADF87E1060
:1013900097F836001D901D98FD2801DDFF201D9057
:1013A00022981EA982681BA8F4F705FD00B987E7FB
:1013B00019A8249908F0B4FE4FF0FF32114619A87D
:1013C00008F0E7FFB7F9008019A808F095FF8346F9
:1013D00019A808F010FF834503DA19A808F08CFF5C
:1013E00002E019A808F007FF18901898B8EB600FF2
:1013F00002DD18984FEA6008B7F90000179020A89E
:1014000008F07AFF834620A808F0F5FE834503DA4A
:1014100020A808F071FF02E020A808F0ECFE189068
:10142000DDE91701B0EB610F02DD1898401017904D
:10143000B7F92E1017980C1804FB04F1480014F0AB
:1014400039F98246B7F92E20179803B2514620A8E1
:1014500026F032FA1EA80DF031FC16904FF001096B
:10146000169820B9F878FF2801DBB87808B14FF05A
:1014700000094FF0FF300F90B9F1000F0BD101239D
:101480000FFA88F219A910A80DF090FF002110A8FA
:101490000DF016F90F901EA808F02EFF834614F0E9
:1014A00009F90E901C2102A814F06EFB0CA8029002
:1014B00007900E980590B88DADF8100097F836009B
:1014C0008DF82000B8788DF821001EA808F014FFD0
:1014D000834600EBDB70BDF8781001EB600000B2D2
:1014E00001901EA808F087FE834600EBDB70BDF874
:1014F0007A1001EB600000B20090BDF87C00ADF8FE
:101500003400BDF87C00001B401C00B2ADF8300078
:10151000BDF87A00ADF83200BDF87A002044401ED4
:1015200000B2ADF83600BDF930100198814202DDFD
:10153000BDF9300000E00198ADF83000BDF936107B
:101540000098814202DABDF9360000E00098ADF85B
:10155000360022980CA982680AA8F4F72CFC00280F
:1015600066D00FFA88F219A90AA8F4F765FC0028DA
:101570005ED10AA808F0C0FE83465646BDF92A008F
:10158000BDF97A10401A00FB0466BDF92810BDF9B8
:101590007C00001B401C081A0644B9F1000F09D05A
:1015A0000FFA88F219A90AA8F4F7C1FC10B10120BA
:1015B000099001E0CDF82490BBF1000F37DD0E98C3
:1015C0000590BDF82800ADF83000BDF82C00ADF84E
:1015D000340002208DF81800BDF92A5023E0ADF840
:1015E0003250ADF836500998A8B9224631460E98C7
:1015F00014F048F9BDF928105B462A460E980DF004
:101600000DFB8DF818009DF81800012804D1022068
:101610008DF8180000E0059602A922980EF006FA4F
:101620002644681C05B2BDF92E00A842D7DA00BFD7
:10163000BDF87C00ADF83400BDF87C00001B401CF8
:1016400000B2ADF83000BDF87E00001B401C00B2B7
:10165000ADF83200BDF87E00ADF83600BDF93010AF
:101660000198814202DDBDF9300000E00198ADF83B
:101670003000BDF932100098401C814202DDBDF9F6
:10168000320001E00098401C00B2ADF83200229810
:101690000CA982680AA8F4F78EFB002866D00FFA1E
:1016A00088F219A90AA8F4F7C7FBA8BB0AA808F092
:1016B00023FE83465646BDF93600BDF92E10401A6A
:1016C00000FB0466BDF92810BDF97C00001B401C1E
:1016D000081A0644B9F1000F09D00FFA88F219A9C7
:1016E0000AA8F4F724FC10B10120099001E0CDF81C
:1016F0002490BBF1000F38DD0E980590BDF828004E
:10170000ADF83000BDF82C00ADF8340002208DF8A3
:101710001800BDF92E5024E028E0ADF83250ADF8A5
:1017200036500998A8B9224631460E9814F0AAF806
:10173000BDF928105B462A460E980DF06FFA8DF819
:1017400018009DF81800012804D102208DF8180017
:1017500000E0059602A922980EF068F92644681E5A
:1017600005B2BDF92A00A842D7DD00BFBDF8780058
:10177000204400B2ADF83000BDF87C00001B00B280
:10178000ADF83400BDF87A00ADF83200BDF87A004B
:101790002044401E00B2ADF83600BDF93610009866
:1017A000814202DABDF9360000E00098ADF836005B
:1017B00022980CA982680AA8F4F7FDFA002870D0D4
:1017C0000FFA88F219A90AA8F4F736FB002868D1A5
:1017D0000AA808F091FD83465646BDF92A00BDF9D6
:1017E0003210401A00FB0466B9F1000F09D00FFA5D
:1017F00088F219A90AA8F4F79AFB10B10120099000
:1018000001E0CDF82490BBF1000F49DD099810B933
:101810000E98059001E000200590BDF82800ADF875
:101820003000BDF82C00ADF83400BDF92A5033E08B
:10183000ADF83250ADF836500998C8B931785A46EB
:101840000E9814F067F9BDF928105B462A460E98E9
:101850000DF0E4F98DF818009DF81800012802D168
:1018600002208DF8180002A922980EF0DFF810E08F
:101870001D98FF2801D1307805E0307897F83610B0
:1018800010FB01F000128DF8200002A922980EF042
:10189000CDF82644681C05B2BDF92E00A842C7DA6F
:1018A00000BF97F836008DF82000BDF8780020447E
:1018B00000B2ADF83000BDF87C00001B00B2ADF8FE
:1018C0003400BDF87E00001B401C00B2ADF83200B1
:1018D000BDF87E00ADF83600BDF932100098401C0E
:1018E000814202DDBDF9320001E00098401C00B2E7
:1018F000ADF8320022980CA982680AA8F4F75BFAC6
:1019000000287DD00FFA88F219A90AA8F4F794FAF2
:1019100000287AD10AA808F0EFFC83465646BDF9A4
:101920003600BDF92E10401A00FB0466BBF1000F13
:101930006ADDB9F1000F09D00FFA88F219A90AA8D7
:10194000F4F7F5FA10B10120099001E0CDF82490E8
:10195000099810B90E98059001E000200590BDF897
:101960002800ADF83000BDF82C00ADF83400BDF90A
:101970002E5042E0ADF83250ADF83650B9F1000FBC
:1019800009D00FFA88F219A90AA8F4F7D0FA10B111
:101990000120099001E0CDF824900998C8B9317868
:1019A0005A460E9814F0B6F8BDF928105B462A4640
:1019B0000E980DF033F98DF818009DF818000128E5
:1019C00002D102208DF8180002A922980EF02EF8FC
:1019D00010E01D98FF2801D1307805E0307897F8A5
:1019E000361010FB01F000128DF8200002A9229899
:1019F0000EF01CF82644681E05B2BDF92A0001E06D
:101A000003E001E0A842B5DD00BF97F836008DF88D
:101A10002000BDF87C00001B401C00B2ADF8300077
:101A2000BDF87C00ADF83400BDF87A00204400B267
:101A3000ADF83200BDF87E00001B00B2ADF83600F4
:101A4000BDF932100098401C814202DABDF9320023
:101A500001E00098401C00B2ADF83200BDF936102C
:101A60000098814202DDBDF9360000E00098ADF833
:101A70003600BDF930100198814202DDBDF9300019
:101A800000E00198ADF8300022980CA982680AA8FD
:101A9000F4F791F9E0B30FFA88F219A90AA8F4F75C
:101AA000CBF9A8BB0AA808F027FC83465646601E5F
:101AB00000FB0466BDF92810BDF97C00001B401C2A
:101AC000081A0644B9F1000F09D00FFA88F219A9D3
:101AD0000AA8F4F72CFA10B10120099001E0CDF822
:101AE0002490099808B1304600E00E980590BBF1AB
:101AF000000F33DDBDF82800ADF83000BDF82C0034
:101B0000ADF8340002208DF81800BDF92A5021E00C
:101B100025E0ADF83250ADF836500998A0B95A46D4
:101B200031460E9813F0AEFEBDF928105B462A46EA
:101B30000E980DF073F88DF818009DF81800012824
:101B400002D102208DF8180002A922980DF06EFF34
:101B5000681C05B2BDF92E00A842DADA00BF56466D
:101B6000002515E030463319591E002208E003789D
:101B700091F800C080F800C00B70401C491E521C38
:101B800004EBD47CB2EB6C0FF1DB2644681C05B28D
:101B9000A542E7DBBDF87800ADF83000BDF878006D
:101BA0002044401E00B2ADF83400BDF87A00204455
:101BB00000B2ADF83200BDF87E00001B00B2ADF8F7
:101BC0003600BDF932100098401C814202DABDF99E
:101BD000320001E00098401C00B2ADF83200BDF9BF
:101BE00036100098814202DDBDF9360000E0009811
:101BF000ADF83600BDF934100198401E814202DA7A
